:020000040800F2
:1000000000000120412904088D290408CDA8010819
:100010008D2904088D2904088D290408000000009A
:100020000000000000000000000000008D2904080E
:100030008D290408000000008D290408EDA30108A3
:100040008D2904088D2904088D2904088D290408A8
:100050008D2904088D29040851A901087DAA0108E9
:1000600041AA010805AA0108C9A90108F1B60008BA
:10007000E1B60008D1B60008C1B60008B1B6000864
:100080009DB6000889B600088D2904088D2904084A
:100090008D2904088D2904088D2904088DA90108DB
:1000A0001DA400088D2904088D2904088D29040841
:1000B00061A4000851A400088D29040889B800082B
:1000C000ADB80008C9B70008EDB700088D290408CD
:1000D0008D2904087D9A00088D290408719A00086A
:1000E00015A901088D2904088D2904088D29040803
:1000F0003DA400088D2904082DA4000875B6000849
:100100008D2904088D29040841A400088D290408BC
:100110008D2904088D2904088D29040891190408E3
:1001200061B600084DB6000839B6000825B60008CB
:1001300011B60008000000000000000000000000F0
:10014000000000000000000000000000D14803088B
:10015000FDB50008E9B50008D5B50008659A0008A6
:1001600001B7000829B700088D2904088D29040863
:100170008D2904088D2904080000000000000000FB
:100180008D2904088D2904088D2904088D29040867
:100190008D2904088D290408000000008D29040819
:1001A0000000000000000000000000008D2904088D
:1001B0008D2904088D2904080000000000000000BB
:1001C000000000000000000000000000000000002F
:1001D0000000000000000000000000008D2904085D
:0801E00080240400010000006E
:1001E80002020300D41E0120D01E012000000000DE
:1001F800000000001600080098220120AC2201200F
:100208000000000070060008270004006424012094
:10021800D424012000000000780600080E02020025
:10022800582501205C250120000000007C060008FC
:1002380003123300A72801207428012000000000C1
:100248008006000825005A00C02701201A2801202E
:100258000000000000000000F6110C00B427012087
:10026800A827012000000000B4060008150070004F
:10027800C8260120382701200000000000000000E7
:100288002A006000082601206826012000000000DE
:10029800D53502082C001000EC2E0120DC2E0120A0
:1002A800000000000D1802082B002400202F012058
:1002B800FC2E012000000000DD1702082900500074
:1002C800102E0120442F0120000000000000000033
:1002D80001200800703501209C3501200000000035
:1002E800C00600081A00080058350120A43501206E
:1002F80000000000C806000800020500BC35012007
:100308004839012000000000000000001E00040021
:10031800C43501205039012000000000D006000833
:1003280022000C006438012054390120000000002C
:10033800D40600080B201000043D0120943D012044
:1003480000000000E00600081F000E00003A01202F
:10035800A43D012000000000F0060008050201008D
:10036800283B0120B43D012000000000FE060008E3
:1003780009020100683E0120983E012000000000AB
:100388000007000812200C00D93D01209C3E0120E6
:1003980000000000020700080C002400E63D0120D0
:1003A800A83E0120000000002DBB03081400020035
:1003B800A840012058440120000000000E07000852
:1003C800051006009E450120184601200000000087
:1003D800100700080E20EA007E4401202046012074
:1003E800000000004936020813000400B44501204B
:1003F8000C47012000000000180700080201030054
:1004080069440120104701200000000055BB030883
:10041800FB0101001C580120E058012000000000E9
:1004280005900108FC010900E8560120E458012064
:1004380000000000D18F01080A101200BC560120EC
:10044800F0580120000000001C07000834001000CC
:100458000C4E01200459012000000000FD3502085F
:1004680018102C00384D01201459012000000000FC
:10047800712502080D003400644D01204059012007
:1004880000000000BD00040803010A008C59012087
:10049800DC590120000000002E07000803000100BD
:1004A8009C5B0120A45B012000000000000000000C
:1004B800FE010900C05B0120D45E0120000000009D
:1004C8000D90010804008000807C0120F88F012035
:1004D8000000000000000000F9010400445F012052
:1004E80078900120000000008D900108FD01240093
:1004F8001C5F01207C900120000000001990010879
:1005080006001600887E0120A0900120000000004F
:10051800693602081B00F400C090012090A1012058
:1005280000000000D55E020826000E0094A20120FB
:1005380084A2012000000000658C0308100003005D
:1005480090A301209CA301200000000038070008A8
:100558002800100080A30120A0A3012000000000B3
:10056800D9CA02082300100070A30120B0A30120FB
:1005780000000000F1CA02081900050068A3012064
:10058800C0A30120000000003C070008F81101008A
:1005980064A30120C8A3012000000000420700084E
:1005A8000001040060A30120CCA30120000000008A
:1005B800440700082F00110044A30120D0A3012004
:1005C80000000000480700080101040024A40120DD
:1005D800B8B60120000000000000000008020C006E
:1005E80042B60120BCB6012000000000A590010819
:1005F800060210004EB60120C8B601200000000017
:1006080083B40108070202008CB60120D8B6012085
:10061800000000005A070008FF010100F4B601209D
:10062800DCB60120000000005C07000802000C0096
:1006380060B60120E0B601200000000000000000C4
:10064800F70106003CB60120ECB6012000000000CE
:100658005E0700080A020A0010B8012020B801202D
:08066800000000006407000817
:10067000C409000019012828200300000000000020
:10068000000000000000000000000000000000006A
:10069000000000000000000000000000000000005A
:1006A000000000000000000000000000000000004A
:1006B0000000010000000000000000000000000039
:1006C000E8036400040A00017E05EA05B40532006F
:1006D00000000100C800141E010064002C01280065
:1006E0002B21231E64010200000001000A012900E1
:1006F00000000000000001000000000500000000F4
:1007000037000000000100054E45524F0000030075
:10071000200002010000000008000000003001007D
:10072000005A0000000090012C01C8006400040180
:1007300001006C1600000000000105000000280107
:100740000000040090010000000000000000000014
:1007500000000000000000000000013C000031012A
:0E0760000000000000004A01B400D6010000B5
:10076E00010100005C760408349F040800000000BC
:10077E00000000006C760408747604080000000087
:10078E00012000007876040880760408000000003E
:10079E000140000084760408CC9704080000000095
:1007AE0001200000907604089C76040800000000EA
:1007BE0004000000A0760408AC76040800000000D7
:1007CE0004000000B0760408EC8404080000000069
:1007DE00010000000201FF000000803F0000803F8A
:1007EE00FFFFFFFF0101D601B51102080000000056
:1007FE00000000000000803F00000000000000002C
:10080E00000000000000803F00000000000000001B
:10081E0000000000000000000000000000000000CA
:10082E000000000000000000000000000000803FFB
:10083E0000000000000000000000000001000000A9
:10084E0001AA550B010000AA5507010000AA55097F
:10085E000200000001000000C012AA5503009F0014
:10086E0000010101010000000101010009E7020879
:10087E000000000080020120D0A704080000000044
:10088E00000000000000000000000000349F04087B
:10089E00000000000000000008030120040000001A
:1008AE007CA704080C00000071ED02081015012051
:1008BE0000000000C8A204080C00000099ED020818
:1008CE000415012000000000D0A20408080000005A
:1008DE0000000000F814012004000000D8A2040853
:1008EE000C000000B1E70208EC140120000000002B
:1008FE00E8A2040803000000B1A70308E0140120D9
:10090E0000000000E0A7040803000000B1A70308E0
:10091E00D41401200000000034A1040801000000DE
:10092E0000000000000000000000000000000000B9
:10093E000D0000000000000000000000000000009C
:10094E00D0A7040800000000000000000000000016
:10095E0000000000349F04080000000000000000AA
:10096E00080301200400000028A70408030000006B
:10097E0085EB0208C814012008000000D8A2040864
:10098E000C000000B1E70208EC140120000000008A
:10099E00E8A2040803000000B1A70308E014012038
:1009AE0000000000E0A7040803000000B1A7030840
:1009BE00D41401200000000034A10408010000003E
:1009CE000000000000000000000000000000000019
:1009DE000D000000000000000000000000000000FC
:1009EE00E8A704080000000000000000000000005E
:1009FE0000000000349F040800000000000000000A
:100A0E00080301200400000030A7040803000000C2
:100A1E00B1A703081C1501200000000034A1040832
:100A2E0001000000000000000000000000000000B7
:100A3E00000000000D00000000000000000000009B
:100A4E000000000020700020702D720000000000D9
:100A5E000000000098100120FFFFFFFFFA000000C9
:100A6E0001000000010000002D202D2D202D2D2D28
:100A7E002D202D2D2D000000000000000000000094
:100A8E0000000000000000002CA10408000000007F
:100A9E000000000000000000000000001AA1040881
:100AAE0004000000FDEA0208000000000000000043
:100ABE0034A1040801000000000000000000000046
:100ACE0000000000000000000D000000000000000B
:100ADE000000000000000000327D01200100C4096A
:100AEE0000000000307D01200100C409000000005C
:100AFE002E7D01200100C409000000002C7D012084
:100B0E000100C40900000000287D01200100C40975
:100B1E00000000002A7D01200100C4090000000031
:100B2E00267D01200100C40900000000247D012063
:100B3E000100C409000000000000000000000000D9
:100B4E0028030120D05901209CFF2C010000000039
:100B5E00080101200A000000206204085C44012004
:100B6E00E0150C17000000000A010120080000002B
:100B7E00046504080901012005000000146304083F
:100B8E005E4401200200000038620408A4450120E2
:100B9E000100FF7F010000009D45012002000000C2
:100BAE0044620408724401200300000054620408E9
:100BBE0071440120030000005462040870450120B6
:100BCE000000F401010000006E4501200000F40158
:100BDE00010000006C4501200000F401010000003E
:100BEE006A4501200000F401010000006845012063
:100BFE0000FF010088450120E803D0070A0000002D
:100C0E0086450120006401000A0000008245012093
:100C1E000064010081450120006401008745012028
:100C2E00006401000A0000008045012000640100FC
:100C3E000A00000085450120006401000A00000042
:100C4E0084450120006401000A0000008345012054
:100C5E00006401000A0000007F45012000FF010032
:100C6E000A0000007E45012000FF01000A0000007E
:100C7E007A4401200000F4010100000078440120B4
:100C8E000000F40101000000764401200000F40190
:100C9E0001000000744401200000F4010100000076
:100CAE007A4501201400E803010000007845012078
:100CBE00E8033075010000007745012000C80100EF
:100CCE007645012000C801007545012000C80100CD
:100CDE0074450120006401000A00000073450120E4
:100CEE0000FF01000A0000009345012000C801002A
:100CFE009245012000C801009145012000C8010065
:100D0E009045012000C801008F45012000C8010058
:100D1E008E45012000C801008D45012000C801004C
:100D2E008C45012000C801008B45012000C8010040
:100D3E0060A1040800000000000000000000000098
:100D4E000000000070A1040809000000000000006F
:100D5E00CC0301200400000078A104080900000063
:100D6E0000000000C00301200400000044A5040898
:100D7E000900000000000000B40301200400000080
:100D8E007CA004080900000000000000A803012058
:100D9E000400000080A1040809000000000000000B
:100DAE009C0301200400000088A104080900000033
:100DBE0000000000900301200400000090A1040830
:100DCE000900000000000000840301200400000060
:100DDE0098A104080900000000000000780301201B
:100DEE000400000034A1040801000000000000000F
:100DFE000000000000000000000000000D000000D8
:100E0E00000000000000000000000000A4A2040882
:100E1E0000000000000000000000000000000000C4
:100E2E00B4A2040805000000000000007044012078
:100E3E000000000034A104080100000000000000C2
:100E4E000000000000000000000000000D00000087
:100E5E00000000000000000000000000BCA204081A
:100E6E000000000000000000000000000000000074
:100E7E00349F040800000000000000003815012017
:100E8E000400000078A004080C00000061EB0208CA
:100E9E0020040120000000007CA704080C000000C4
:100EAE00C1E602081404012000000000C8A20408D4
:100EBE000C000000A5E60208080401200000000056
:100ECE00D0A204080800000000000000FC0301206E
:100EDE0004000000D8A204080C000000F1E502088E
:100EEE00F003012000000000E0A204080900000049
:100EFE0000000000E403012004000000E8A2040842
:100F0E0003000000B1A70308D80301200000000071
:100F1E0034A10408010000000000000000000000E1
:100F2E0000000000000000000D00000000000000A6
:100F3E000000000000000000ECA204080000000009
:100F4E00000000000000000000000000FCA20408E9
:100F5E000C0000000000000038040120000000001A
:100F6E0004A304080A00000000000000B845012098
:100F7E000000000010A304080A000000000000009A
:100F8E00C04501200000000018A304080A0000005C
:100F9E0000000000C84501200000000020A3040846
:100FAE0008000000000000002C04012000000000DA
:100FBE0034A1040801000000000000000000000041
:100FCE0000000000000000000D0000000000000006
:100FDE00000000000000000028A30408000000002C
:100FEE000000000000000000000000003CA3040808
:100FFE000C00000000000000500401200000000062
:10100E004CA30408040000000DEE020800000000CE
:10101E000000000054A304080C00000000000000B3
:10102E00440401200000000068A30408040000002E
:10103E00EDED0208000000000000000034A10408DD
:10104E000100000000000000000000000000000091
:10105E00000000000D000000000000000000000075
:10106E000000000070A30408000000000000000053
:10107E00000000000000000084A304080700000028
:10108E00000000008C0401200000000090A3040862
:10109E000800000000000000800401200000000095
:1010AE009CA3040808000000000000007404012046
:1010BE0000000000A8A304080800000000000000C3
:1010CE006804012000000000B4A30408080000001A
:1010DE00000000005C0401200000000034A10408A0
:1010EE0001000000000000000000000000000000F1
:1010FE00000000000D0000000000000000000000D5
:10110E0000000000C0A30408000000000000000062
:10111E00E702012000000000CCA304080B00000031
:10112E00000000000405012000000000D4A3040804
:10113E000B00000000000000F80401200000000079
:10114E00E0A304080B00000000000000EC040120E6
:10115E0000000000ECA304080B00000000000000DB
:10116E00E004012000000000F8A304080B000000BA
:10117E0000000000D40401200000000004A40408B4
:10118E000B00000000000000C80401200000000059
:10119E000CA404080B00000000000000BC04012099
:1011AE000000000018A40408070000000000000062
:1011BE00B40401200000000020A404080700000071
:1011CE0000000000AC040120000000002CA4040864
:1011DE000B00000000000000A00401200000000031
:1011EE0038A4040808000000000000009404012048
:1011FE000000000034A104080100000000000000FF
:10120E000000000000000000000000000D000000C3
:10121E0000000000000000000000000044A40408CC
:10122E0000000000000000000000000000000000B0
:10123E0058A4040808000000000000003405012036
:10124E000000000064A40408080000000000000074
:10125E00280501200000000070A40408080000000A
:10126E00000000001C050120000000007CA4040802
:10127E000800000000000000100501200000000022
:10128E0034A104080100000000000000000000006E
:10129E0000000000000000000D0000000000000033
:1012AE00000000000000000084A4040800000000FC
:1012BE0000000000E40201200000000094A40408D5
:1012CE000B000000000000007C0501200000000063
:1012DE00A0A404080B00000000000000700501200F
:1012EE0000000000ACA4040807000000000000008D
:1012FE006805012000000000B8A4040807000000E3
:10130E00000000006005012000000000C4A40408D5
:10131E00070000000000000058050120000000003A
:10132E00D0A4040808000000000000004C050120B5
:10133E0000000000D8A4040808000000000000000F
:10134E00400501200000000034A104080100000047
:10135E00000000000000000000000000000000007F
:10136E000D00000000000000000000000000000062
:10137E00E0A404080000000000000000E4020120C8
:10138E0000000000ECA404080700000000000000AC
:10139E00C805012000000000F4A4040807000000A6
:1013AE0000000000C005012000000000FCA404089D
:1013BE000700000000000000B8050120000000003A
:1013CE0004A504080700000000000000B00501207D
:1013DE00000000000CA5040807000000000000003B
:1013EE00A80501200000000014A504080700000055
:1013FE0000000000A0050120000000001CA504084C
:10140E000700000000000000980501200000000009
:10141E0024A504080700000000000000900501202C
:10142E00000000002CA504080700000000000000CA
:10143E00880501200000000034A10408010000000E
:10144E00000000000000000000000000000000008E
:10145E000D00000000000000000000000000000071
:10146E000000000045E80208D00501206E4401206E
:10147E001B000000646204086D4401200A32010062
:10148E006C44012001FA01006844012000C80100EB
:10149E0066440120E803D007010000004E45524F7C
:1014AE00000000005BE80208C1ED0208AC06012056
:1014BE002DE6020800000000FC0601200DEF0208D8
:1014CE00B5EA0208D80701207DE8020800000000F6
:1014DE00780801200DE90208DDE802080409012060
:1014EE0099E90208E1E90208A40901207C450120DE
:1014FE0001030100B1E802088DE80208BC0A0120D0
:10150E003DE902082DEE0208480B012011EA0208FF
:10151E0089EE0208100C0120724501200103010022
:10152E0034A50408000000000000000000000000C8
:10153E000000000040A504080800000000000000A4
:10154E00300D01200000000048A50408070000002F
:10155E0000000000280D01200000000058A504081E
:10156E000700000000000000200D01200000000018
:10157E0064A504080700000000000000180D0120FB
:10158E000000000070A504080C0000000000000020
:10159E000C0D0120000000007CA5040803000000D3
:1015AE00B1A70308000D01200000000034A10408BB
:1015BE00010000000000000000000000000000001C
:1015CE00000000000D000000000000000000000000
:1015DE000000000084A504080000000000000000C8
:1015EE00000000000000000094A504080A0000009E
:1015FE0000000000BC760408000000009CA5040852
:10160E000A000000000000003C7604080000000004
:10161E00A4A504080A000000000000009445012063
:10162E0000000000ACA504080A0000000000000045
:10163E003C0D01200000000034A104080100000050
:10164E00000000000000000000000000000000008C
:10165E000D0000000000000000000000000000006F
:10166E00B4A5040800000000000000000000000007
:10167E0000000000C8A5040803000000B1A703087D
:10168E005C0D012000000000D4A50408030000003A
:10169E00B1A703080C01012000000000DCA504081E
:1016AE0003000000B1A70308500D01200000000048
:1016BE00E4A5040803000000B1A70308440D0120AF
:1016CE000000000034A1040801000000000000002A
:1016DE000000000000000000000000000D000000EF
:1016EE00000000000000000000000000F0A504084B
:1016FE0000000000000000000000000000000000DC
:10170E00FCA5040807000000D5EE0208B80D012064
:10171E000000000000AC040803000000B1A703089D
:10172E00AC0D01200000000008A604080300000014
:10173E00B1A70308A00D01200000000010A60408A8
:10174E0003000000B1A70308940D01200000000063
:10175E0018A6040807000000B9EE02088C0D01203F
:10176E000000000098A7040803000000B1A70308BA
:10177E00800D01200000000024A6040803000000D4
:10178E00B1A70308740D01200000000030A6040864
:10179E0003000000B1A70308680D0120000000003F
:1017AE0034A1040801000000000000000000000049
:1017BE0000000000000000000D000000000000000E
:1017CE0000000000000000000DE80208D5E7020846
:1017DE00C00D012081EA020800000000740E0120F5
:1017EE000000000000000000000F012059EA02086E
:1017FE00F1EE02088C0F01203CA604080000000048
:10180E0000000000000000000000000080A004089E
:10181E0003000000B1A703088C1001200000000097
:10182E0048A6040803000000B1A703088010012099
:10183E000000000054A6040803000000B1A703082E
:10184E00741001200000000060A6040803000000D0
:10185E00B1A70308681001200000000068A6040864
:10186E000200000001F0020800000000000000006D
:10187E0070A604080200000001F00208010000003A
:10188E00000000007CA604080200000001F002081F
:10189E000200000000000000000000000D0000002B
:1018AE000000000000000000000000006244012063
:1018BE0088136F17010000006444012088136F170E
:1018CE000000000088A604080000000000000000D0
:1018DE00000000000000000098A6040808000000A8
:1018EE00000000005811012004000000A4A6040806
:1018FE0008000000000000004C1101200000000054
:10190E00E8A2040804000000C5EB02080000000075
:10191E000000000034A104080100000000000000D7
:10192E000000000000000000000000000D0000009C
:10193E0000000000000000000000000060440120D4
:10194E0088136F1701000000203B012088136F17CA
:10195E000000000069E70208000000006411012089
:10196E00B045012001000000D4620408223B012092
:10197E0001000000E0620408183B01200200000094
:10198E00E86204087A7D01200000000000000000DB
:10199E00787D01200000000000000000767D01200F
:1019AE000000000000000000747D01200000000017
:1019BE0000000000727D0120000000000000000009
:1019CE00707D01200000000000000000F8000120E2
:1019DE0000000000000000005F4401200200000033
:1019EE00F4620408E0A604080000000000000000F5
:1019FE00000000000000000098A604080800000087
:101A0E0000000000E811012004000000A4A6040854
:101A1E000800000000000000DC11012000000000A2
:101A2E00E8A20408040000003DE7020800000000E0
:101A3E000000000034A104080100000000000000B6
:101A4E000000000000000000000000000D0000007B
:101A5E00000000000000000000000000F0A60408D6
:101A6E000000000000000000000000000000000068
:101A7E0000A704080C00000015ED02081812012042
:101A8E00040000000CA704080C0000008DE70208FB
:101A9E000C1201200400000018A704080C0000001E
:101AAE00D9EC0208001201200000000024A704084F
:101ABE0003000000A5EB0208F4110120080000004D
:101ACE0030A7040803000000B1A703081C1501206D
:101ADE000000000034A10408010000000000000016
:101AEE000000000000000000000000000D000000DB
:101AFE000000000000000000000000002CA10408FF
:101B0E0000000000000000000000000000000000C7
:101B1E001AA1040804000000E1EB02080000000016
:101B2E000000000034A104080100000000000000C5
:101B3E000000000000000000000000000D0000008A
:101B4E0000000000000000000000000084A7040850
:101B5E000000000000000000000000000000000077
:101B6E00487E04080C0000000000000078120120DE
:101B7E000400000094A70408080000000000000004
:101B8E006C12012004000000A0A704080800000049
:101B9E00000000006012012004000000A8A7040845
:101BAE000800000000000000541201200400000094
:101BBE00B0A7040808000000000000004812012031
:101BCE0004000000B8A70408080000000000000090
:101BDE003C12012004000000C0A704080800000009
:101BEE00000000003012012004000000C8A7040805
:101BFE000800000000000000241201200400000074
:101C0E0034A10408010000000000000000000000E4
:101C1E0000000000000000000D00000000000000A9
:101C2E00000000000000000055E702080000000060
:101C3E00841201200000000000000000FC120120B0
:101C4E0000000000000000009C1301201E3B01203C
:101C5E0004000000006304081C3B0120E0150C1773
:101C6E00000000001B3B0120080000000465040872
:101C7E001A3B012005000000146304080000000058
:101C8E0000000000EC130120010000FFFF00000027
:101C9E000000AA55050100002D202D2D202D2D2DE3
:101CAE002D202D2D2D2D0000000000000000000025
:101CBE0000000000000000001A03000000000000F9
:101CCE000000000000000000000000000000000006
:101CDE00000000000403090412010002020000408B
:101CEE00830440570002010203010000006002401D
:101CFE001060024000000000000B000000002000F9
:101D0E000000000000000000006002402860024059
:101D1E0000000000060C0000000020000000000083
:101D2E000000000000600240406002400000000021
:101D3E00100D000000002000000000000000000058
:101D4E00006002405860024000000000160E0000C5
:101D5E0000002000000000000000000000600240B3
:101D6E007060024000000000200F00000000200004
:101D7E000000000000000000006002408860024089
:101D8E0000000000261000000000200000000000EF
:101D9E000000000000600240A06002400000000051
:101DAE0030110000000020000000000000000000C4
:101DBE0000600240B860024000000000362F0000B4
:101DCE00000020000000000000000000006402403F
:101DDE0010640240000000000038000000004000C7
:101DEE000000000000000000006402402864024071
:101DFE000000000006390000000040000000000056
:101E0E000000000000640240406402400000000038
:101E1E00103A00000000400000000000000000002A
:101E2E00006402405864024000000000163B0000AF
:101E3E0000004000000000000000000000640240AE
:101E4E007064024000000000203C000000004000D2
:101E5E0000000000000000000064024088640240A0
:101E6E0000000000264400000000400000000000BA
:101E7E000000000000640240A06402400000000068
:101E8E00304500000000400000000000000000008F
:101E9E0000640240B86402400000000036460000B4
:101EAE000000400000000000000000000000803F25
:101EBE0000000101FFFF0000A47B040800000000E9
:101ECE000000000069BB0308A086010004000000AA
:101EDE0000000000000000000000000000000000F4
:101EEE0000000000000000000000000000AC04082C
:101EFE00D49D040800000000652B01087D00000041
:101F0E0006000000000000000000000000000000BD
:101F1E0000000000000000000000000000000000B3
:101F2E0020AA04080000000000000000719A0108B9
:101F3E00E8030000030000000000000000000000A5
:101F4E000000000000000000000000000000000083
:101F5E000000000028AA0408000000000000000095
:101F6E00B137020810270000030000000000000037
:101F7E000000000000000000000000000000000053
:101F8E00000000000000000088A00408000000000F
:101F9E0071160208BDE70008204E00000500000083
:101FAE000000000000000000000000000000000023
:101FBE000000000000000000000000003C7D04084E
:101FCE00000000000000000001AB01081027000017
:101FDE0001000000000000000000000000000000F2
:101FEE0000000000000000000000000000000000E3
:101FFE0034AA040800000000000000009D8F0108B4
:10200E00E8030000050000000000000000000000D2
:10201E0000000000000000000000000000000000B2
:10202E000000000040AA04080000000000000000AC
:10203E008DBD0308204E00000300000000000000CC
:10204E000000000000000000000000000000000082
:10205E00000000000000000050AA0408000000006C
:10206E000000000099BB0308204E00000300000092
:10207E000000000000000000000000000000000052
:10208E0000000000000000000000000060AA04082C
:10209E000000000000000000D1900108400D030078
:1020AE00030000000000000000000000000000001F
:1020BE000000000000000000000000000000000012
:1020CE00707C04080000000000000000FD0A0408F7
:1020DE0010270000010000000000000000000000BA
:1020EE0000000000000000000000000000000000E2
:1020FE0000000000447D0408000000000000000005
:10210E0059740208102700000300000000000000B0
:10211E0000000000000000000000000000000000B1
:10212E00000000000000000070AA0408000000007B
:10213E000000000049AE0208A08601000100000068
:10214E000000000000000000000000000000000081
:10215E00000000000000000000000000507D040898
:10216E00000000000000000089BC0008A00F000065
:10217E000100000000000000000000000000000050
:10218E000000000000000000000000000000000041
:10219E007CAA040800000000000000003191030832
:1021AE0010270000010000000000000000000000E9
:1021BE000000000000000000000000000000000011
:1021CE0000000000B47D04080000000000000000C4
:1021DE002D7C020810270000010000000000000006
:1021EE0000000000000000000000000000000000E1
:1021FE000000000000000000C09D04080000000068
:10220E0000000000B1F102081A41000001000000B8
:10221E0000000000000000000000000000000000B0
:10222E0000000000000000000000000088AA040862
:10223E00000000000000000079790108400D030045
:10224E000000000000000000000000000000000080
:10225E000000000000000000000000000000000070
:10226E0090AA040800000000000000001579010883
:10227E00400D030000000000000000000000000000
:10228E000000000000000000000000000000000040
:10229E000000000098AA04080000000000000000E2
:1022AE0069790208A086010003000000000000000A
:1022BE000000000000000000000000000000000010
:1022CE0000000000000000003C7304080508040034
:1022DE000000000014630408046504080063040889
:1022EE00000000006873040805080A0000000000E2
:1022FE00146304080465040820620408000000004A
:10230E000A06000200000040010000000907430019
:10231E00020104C03209040000010202010005247A
:10232E000010010524010001042402020524060008
:10233E0001070582030800FF09040100020A0000DC
:10234E000007050102400000070581024000000061
:10235E0009024300020100C032090400000102021A
:10236E0001000524001001052401000104240202CD
:10237E000524060001070582030800100904010068
:10238E00020A000000070501020002000705810293
:10239E000002000009024300020100C032090400DD
:1023AE0000010202010005240010010524010001B4
:1023BE00042402020524060001070582030800100A
:1023CE0009040100020A0000000705010240000096
:1023DE0007058102400000000000803F0000000061
:1023EE00000000000000000065480308594803087B
:1023FE0099480308AD4803081148030885480308A7
:10240E00714803088DD40308CDD303087DD6030885
:10241E000000000051D10308ADD1030879D10308A3
:10242E0000000000000000000000000039D1030889
:10243E0045D103082DD1030821D1030867180408DC
:10244E004D18040801180408E917040800E6DF0C0B
:10245E0000C2010000000800FC1C0120000000006A
:10246E00000000000000000000000000000000005E
:10247E00000000000000000000000000000000004E
:10248E00000000000000000000000000000000003E
:10249E00000000000000000000000000000000002E
:1024AE00000000000000000000000000000000001E
:1024BE0000000000000000000000000043000000CB
:1024CE0000000000000000000000000000000000FE
:1024DE0000000000000000000000000043000000AB
:1024EE0000000000000000000000000000000000DE
:1024FE00000000000000000000000000430000008B
:10250E0000000000000000000000000000000000BD
:10251E00000000000000000000000000430000006A
:10252E00000000000000000000000000000000009D
:10253E00000000000000000000000000430000004A
:10254E00000000000000000000000000000000007D
:10255E00000000000000000000000000430000002A
:10256E00000000000000000000000000000000005D
:10257E00000000000000000000000000430000000A
:10258E00000000000000000000000000000000003D
:10259E00000000000000000000000000B933040835
:1025AE001D320408000000001FB0040816A1040824
:1025BE0003880408038804080388040803880408B1
:1025CE0003880408038804080388040803880408A1
:1025DE0003880408FFFFFFFFFFFFFFFFFFFFFFFF62
:1025EE00FFFF000001004153434949000000000075
:1025FE0000000000000000000000000000000000CD
:10260E000000000000004153434949000000000053
:10261E0000000000000000000000000000000000AC
:0C262E000000000000000000010000009F
:10800000012380F8493070474FF4006303837047C1
:108010004FF4006303837047D0F8F420034630B474
:108020006AB1C168D0F80C214469881A013A205C11
:1080300008BF0A46C0B2C3F80C2130BC7047006AC2
:108040005D69411CDC68285CA14228BF1146C0B2B2
:10805000196230BC704700BFD0F8F83013B190F807
:108060008C017047836A406A181AB0FA80F04009A0
:10807000704700BF416A836A99420ED3CB1AD0F889
:10808000F810026981B1D0F87811501E0A68526860
:10809000134483420BD2C01A704702691144CB1AB1
:1080A000D0F8F8100029EED1501EC01A70470020F9
:1080B000704700BFD0F8F4306BB1D0F87C31D0F805
:1080C0000C211B685B68934201D3981A7047C06803
:1080D000801A18447047C269036A9A4203D2C06882
:1080E0001044C01A7047D01A704700BFBFF34F8FBB
:1080F0000549064BCA6802F4E0621343CB60BFF344
:108100004F8F00BFFDE700BF00ED00E00400FA055F
:10811000406994302AF048B9416908220023754823
:108120002DE9F043744D01FA02F783B0D0F80080D6
:108130000193EB19B3F8FC3003EB811305EB8303D8
:10814000DC6FD4F85890E36DD9F800609A4016427D
:1081500004D021680868400700F18780674999408A
:108160000E4203D022685269100677D464499940C0
:108170000E4203D022681268920768D410229A40F7
:10818000164203D02168086800074CD420229A4088
:10819000164203D021680868C00631D4636D0BB362
:1081A000636DDA071AD505232168564A84F83530FD
:1081B000A2FB08320B6823F00103920A0B6002E075
:1081C0000B68DB0704D5019B01339A420193F7D278
:1081D0000022012384F8342084F83530E36C0BB19D
:1081E000204698473D446B681B681A6822F00102DC
:1081F0001A60DA6822F48072DA6003B0BDE8F083B6
:10820000C9F8082094F83520052A3FD00B6813F4EC
:10821000802F0B6859D0190364D5E36B002BBDD0B8
:1082200020469847BAE7C9F808200A6812F4802F58
:108230000A6825D1D20503D40A6822F008020A6030
:10824000226C002AA2D020469047E36D9EE7C9F831
:108250000810626D42F0040262658FE7C9F80810E9
:10826000626D42F00202626580E7086820F0040057
:108270000860C9F80820626D42F0010262656DE78E
:108280001103DDD5A26C002ADDD17FE70A68206CDE
:1082900022F016020A604A6922F080024A6128B37D
:1082A0000A6822F008020A603F220020012102FA37
:1082B00003F3226DC9F8083084F8340084F83510CF
:1082C000002A8FD0204690478CE713F48073A4D106
:1082D0000A68012022F010020A6084F8343084F821
:1082E00035009AE7636C002B9AD157E7A26C002AFD
:1082F000D6D1D9E7EC1C0120B07E0120010080001E
:1083000004008000B5814E1B8C4B1A78002A00F0C7
:10831000EB808B4940F20D300B68F0B49F6C002667
:10832000884C894D3C40AB4240EA04009864D868D0
:1083300040F48070D8605E6200F0FA808348834227
:1083400000F0F6801868012A40F00100186000F083
:10835000CA80D1F8283140F20D307A4C00269F6C4B
:10836000794D3C40AB4240EA04009864D86840F440
:108370008070D8605E6200F0D6807448834200F05E
:10838000D2801868022A40F00100186000F0AB802B
:10839000D1F8503240F20D306A4C00269F6C6A4D85
:1083A0003C40AB4240EA04009864D86840F48070D6
:1083B000D8605E6200F0B2806448834200F0AE8014
:1083C0001868032A40F00100186000F08C80D1F892
:1083D000783340F20D305B4C00269F6C5A4D3C4088
:1083E000AB4240EA04009864D86840F48070D860DA
:1083F0005E6200F08E805548834200F08A801868E3
:10840000042A40F0010018606DD0D1F8A03440F289
:108410000D304C4C00269F6C4B4D3C40AB4240EA2B
:1084200004009864D86840F48070D8605E626BD0B5
:108430004648834268D01868052A40F00100186059
:1084400051D0D1F8C83540F20D303E4C00269F6C1B
:108450003D4D3C40AB4240EA04009864D86840F48B
:108460008070D8605E624AD03848834247D018682E
:10847000062A40F00100186035D0D1F8F03640F2FD
:108480000D30304C00269F6C2F4D3C40AB4240EAF3
:1084900004009864D86840F48070D8605E6229D087
:1084A0002A48834226D01868072A40F00100186045
:1084B00019D0D1F8183840F20D32224900249D6CB1
:1084C00021482940834242EA01029A64DA6842F470
:1084D0008072DA605C6208D01C4A934205D01A6848
:1084E00042F001021A60F0BC70475A6C42F400423C
:1084F0005A64F4E7586C40F400405864D3E7586C71
:1085000040F400405864B2E7586C40F400405864AE
:1085100091E7586C40F40040586470E7586C40F4A0
:10852000004058644CE7586C40F40040586428E719
:10853000586C40F40040586404E700BFB086012046
:10854000B4860120E0E0FFFF00000140000401408C
:10855000F8B590F8813190F88221134303F021039C
:10856000212B0FD0436A846AA3420CD802690023EE
:10857000121B92B290F8811100258362202980F8A5
:108580008C5103D0F8BD1A1B92B2F3E78369E34222
:1085900003EB0401F6D0B2FA82F46409002CF1D1A5
:1085A00090F88031012BEDD005460127A0F86A2113
:1085B0001346A0F868214FF0210ED0F87861C0F87A
:1085C0006411C0F88441304685F880710C4A0D4F23
:1085D00085F881E1F76332640B4FD5F818213465D3
:1085E0002832F76429F0C8FFD5F8183140221A6202
:1085F00085F880419A6842F080029A60C2E700BF25
:108600006DD30308A9D3030805D30308426A10B445
:108610008469A154426A04690132D0F8F810A24278
:1086200028BF0022426241B10B68DB0702D55DF82A
:10863000044B70475DF8044B8AE7D0F818215DF8C9
:10864000044B136843F0800313607047426910B510
:108650000832184C54F8220029F0A6FE164B1A884E
:1086600023460C2A0DD8DFE802F0070C0C0C130C83
:108670000C0C190C0C0C1F002168CA6822F4007243
:10868000CA60012283F83D2000220C4B1A7010BDF5
:108690002168CA6822F48062CA60F2E72168CA6869
:1086A00022F40062CA60ECE72168CA6822F48052B2
:1086B000CA60E6E7E4A00120E0A001204392012087
:1086C0002DE9F0470569C3681D4028D00F460646CE
:1086D0004FF000484FF00009B5FA85F328FA03F28D
:1086E0001B3BD24332611540042B16D8DFE803F060
:1086F0003129211903007B6A002B32D003F1FF3AA4
:10870000C7F824901FFA8AFA3C6A34B123682046DD
:10871000514698476468002CF8D1002DDCD1BDE8A3
:10872000F0873868716B036889B29847002DD3D100
:10873000F5E77868B16B036889B29847002DCBD113
:10874000EDE7B868F16B036889B29847002DC3D193
:10875000E5E7F868316C036889B29847002DBBD112
:10876000DDE7F36A1FFA83FACEE700BF2DE9F04F89
:108770008BB090F859300390002B40F07985039B23
:1087800080226B21BE4C1033BE4D4FF0640ADFF8DF
:10879000FC92184602934FF47A7613F0CFF94FF01B
:1087A000100CB948DFF8E8E2D9F80430C3F3080345
:1087B000002B40F05B84EFF31183002B40F05684D4
:1087C0002168826800BF23689942F9D12F6806FBAF
:1087D00007F39B1AB3FBF7F306FB01310127019165
:1087E000D9F80430C3F30803002B40F00584EFF3FD
:1087F0001183002B40F000842368816800BF226849
:108800009342F9D1D5F800B006FB0BF2521AB2FB35
:10881000FBF206FB0323019A9B1AB3F57A7FDFD3A1
:10882000BAF1010AC0D10722682102984FF0640A08
:1088300013F084F9DFF854924FF01008924E4FF481
:108840007A77DFF84CC2D9F80430C3F30803002B61
:1088500040F0F083EFF31183002B40F0EB832168AD
:10886000B26800BF23689942F9D1286807FB00F37A
:108870009B1AB3FBF0F307FB013101200191D9F8FA
:108880000430C3F30803002B40F09983EFF3118306
:10889000002B40F094832368B16800BF22689342A4
:1088A000F9D1D5F800B007FB0BF2521AB2FBFBF27C
:1088B00007FB0323019A9B1AB3F57A7FDFD3BAF142
:1088C000010AC0D152466B2102984FF0640A13F09E
:1088D00035F9DFF8B8914FF0100C6B484FF47A7609
:1088E000DFF8ACE1D9F80430C3F30803002B40F003
:1088F0006984EFF31183002B40F06484216882685F
:1089000000BF23689942F9D12F6806FB07F39B1A31
:10891000B3FBF7F306FB013101270191D9F80430CD
:10892000C3F30803002B40F02D83EFF31183002BDA
:1089300040F028832368816800BF22689342F9D100
:10894000D5F800B006FB0BF2521AB2FBFBF206FBA5
:108950000323019A9B1AB3F57A7FDFD3BAF1010A98
:10896000C0D101226B2102984FF00F0A13F0E6F8F4
:10897000DFF818914FF0100C43484FF47A76DFF887
:1089800010E1D9F80430C3F30803002B40F0FD8355
:10899000EFF31183002B40F0F8832168826800BF59
:1089A00023689942F9D12F6806FB07F39B1AB3FBA2
:1089B000F7F306FB013101270191D9F80430C3F325
:1089C0000803002B40F0C182EFF31183002B40F02D
:1089D000BC822368816800BF22689342F9D1D5F830
:1089E00000B006FB0BF2521AB2FBFBF206FB0323AC
:1089F000019A9B1AB3F57A7FDFD3BAF1010AC0D18D
:108A0000039B1B2102984FF00F0A93F853304FF449
:108A10007A76DFF87890042B34BF18221A2213F0EC
:108A20008DF84FF0100C1848DFF864E0D9F80430E6
:108A3000C3F30803002B40F0FE83EFF31183002BF8
:108A400040F0F9832168826800BF23689942F9D118
:108A50002F6806FB07F39B1AB3FBF7F306FB013104
:108A600001270191D9F80430C3F30803002B40F02B
:108A70004F82EFF31183002B40F04A820AE000BFDF
:108A80003CC2012040C2012010E000E000ED00E007
:108A900038C201202368816800BF22689342F9D15F
:108AA000D5F800B006FB0BF2521AB2FBFBF206FB44
:108AB0000323019A9B1AB3F57A7FD3D3BAF1010A43
:108AC000B4D118221C2102984FF00F0A13F036F887
:108AD000DFF8E0924FF0100CB4484FF47A76DFF8EC
:108AE000D0E2D9F80430C3F30803002B40F08783A9
:108AF000EFF31183002B40F082832168826800BF6E
:108B000023689942F9D12F6806FB07F39B1AB3FB40
:108B1000F7F306FB013101270191D9F80430C3F3C3
:108B20000803002B40F0D781EFF31183002B40F0B6
:108B3000D2812368816800BF22689342F9D1D5F8B9
:108B400000B006FB0BF2521AB2FBFBF206FB03234A
:108B5000019A9B1AB3F57A7FDFD3BAF1010AC0D12B
:108B6000039B1A2102984FF00F0A93F852204FF4FA
:108B70007A7612F0E3FFDFF83C924FF0100C8B484E
:108B8000DFF82CE2D9F80430C3F30803002B40F0DF
:108B9000A682EFF31183002B40F0A1822168826846
:108BA00000BF23689942F9D12F6806FB07F39B1A8F
:108BB000B3FBF7F306FB013101270191D9F804302B
:108BC000C3F30803002B40F06981EFF31183002BFE
:108BD00040F064812368816800BF22689342F9D124
:108BE000D5F800B006FB0BF2521AB2FBFBF206FB03
:108BF0000323019A9B1AB3F57A7FDFD3BAF1010AF6
:108C0000C0D1039B192102984FF0640A93F85420B5
:108C10004FF47A7612F092FFDFF898914FF0100C33
:108C20006248DFF88CE1D9F80430C3F30803002B65
:108C300040F03982EFF31183002B40F03482216839
:108C4000826800BF23689942F9D12F6806FB07F3B9
:108C50009B1AB3FBF7F306FB013101270191D9F809
:108C60000430C3F30803002B40F0FB80EFF31183C3
:108C7000002B40F0F6802368816800BF2268934291
:108C8000F9D1D5F800B006FB0BF2521AB2FBFBF299
:108C900006FB0323019A9B1AB3F57A7FDFD3BAF15F
:108CA000010AC0D11022372102984FF00F0A12F0AA
:108CB00045FFDFF800914FF0100C3C484FF47A76F6
:108CC000DFF8ECE0D9F80430C3F30803002B40F0E0
:108CD0004082EFF31183002B40F03B8221688268D1
:108CE00000BF23689942F9D12F6806FB07F39B1A4E
:108CF000B3FBF7F306FB013101270191D9F80430EA
:108D0000C3F30803002B40F08F80EFF31183002B97
:108D100040F08A802368816800BF22689342F9D1BD
:108D2000D5F800B006FB0BF2521AB2FBFBF206FBC1
:108D30000323019A9B1AB3F57A7FDFD3BAF1010AB4
:108D4000C0D13821029801224FF00F0912F0F6FE2F
:108D5000DFF860804FF0100E14494FF47A70144F12
:108D6000D8F80430C3F30803002B40F0D481EFF3AC
:108D70001183002B40F0CF8122688E6800BF2368EA
:108D80009A42F9D1D5F800C000FB0CF39B1BB3FB52
:108D9000FCF300FB023301930126D8F80430C3F33F
:108DA00008032BBBEFF3118313BB05E010E000E0D9
:108DB00038C2012000ED00E02368D1F808A000BF10
:108DC00022689342F8D1D5F800B000FB0BFCACEB65
:108DD0000A0CBCFBFBFC00FB03C3019A9B1AB3F516
:108DE0007A7FDAD3B9F10109BAD10BB0BDE8F08FBF
:108DF000EFF3118A8EF312888A680B68DB0301D5C2
:108E00003E608A6823685FFA8AFAD7F800C08AF35E
:108E10001188D5F800A09C4400FB0AF39B1AB3FB11
:108E2000FAF300FB0C33D8E7EFF311888CF31288C8
:108E300081680368DB0302D5CEF80070816823687F
:108E40005FFA88F8DEF8002088F31188D5F80080F2
:108E50001A4406FB08F35B1AB3FBF8F306FB023374
:108E600067E7EFF311888CF3128881680368DB03EE
:108E700002D5CEF80070816823685FFA88F8DEF8C2
:108E8000002088F31188D5F800801A4406FB08F307
:108E90005B1AB3FBF8F306FB0233FBE6EFF3118832
:108EA0008CF3128881680368DB0302D5CEF800706A
:108EB000816823685FFA88F8DEF8002088F311885B
:108EC000D5F800801A4406FB08F35B1AB3FBF8F3ED
:108ED00006FB02338DE6EFF311888CF3128881686C
:108EE0000368DB0302D5CEF80070816823685FFA5F
:108EF00088F8DEF8002088F31188D5F800801A443D
:108F000006FB08F35B1AB3FBF8F306FB02331FE61C
:108F1000EFF311888CF3128881680368DB0302D5B4
:108F2000CEF80070816823685FFA88F8DEF80020C8
:108F300088F31188D5F800801A4406FB08F35B1A01
:108F4000B3FBF8F306FB0233B3E5EFF311888CF3C0
:108F5000128881680368DB0302D5CEF8007081684F
:108F600023685FFA88F8DEF8002088F31188D5F8C6
:108F700000801A4406FB08F35B1AB3FBF8F306FB08
:108F8000023335E5EFF311888CF3128881680368AA
:108F9000DB0302D5CEF80070816823685FFA88F899
:108FA000DEF8002088F31188D5F800801A4406FB0B
:108FB00008F35B1AB3FBF8F306FB0233C9E4EFF3E3
:108FC000118E88F31288B1683368DB0302D5CCF8C0
:108FD0000000B16823685FFA8EFEDCF800208EF393
:108FE0001188D5F800E01A4407FB0EF35B1AB3FBB7
:108FF000FEF307FB02335DE4EFF311888CF3128874
:1090000081680368DB0302D5CEF8007081682368AD
:109010005FFA88F8DEF8002088F31188D5F8008020
:109020001A4406FB08F35B1AB3FBF8F306FB0233A2
:10903000FFF7F1BBEFF3118288F31288B068336851
:10904000D90303D50123CCF80030B0682368D2B22D
:10905000DCF8001082F311882A68194407FB02F338
:109060001B1AB3FBF2F307FB013106E4EFF31182A5
:109070008CF3128887680368D90303D50123CEF8DF
:10908000003087682368D2B2DEF8001082F31188BE
:109090002A68194406FB02F3DB1BB3FBF2F306FB61
:1090A0000131FFF79BBBEFF311828CF312888768C5
:1090B0000368D90303D50123CEF8003087682368FD
:1090C000D2B2DEF8001082F311882A68194406FB38
:1090D00002F3DB1BB3FBF2F306FB0131BDE5EFF35B
:1090E00011828CF3128887680368D90303D50123A2
:1090F000CEF8003087682368D2B2DEF8001082F321
:1091000011882A68194406FB02F3DB1BB3FBF2F358
:1091100006FB013150E5EFF311868EF31288D1F88A
:1091200008C00B68DA0303D501233B60D1F808C0FF
:109130002368F6B23A6886F311882E681A4400FB59
:1091400006F3A3EB0C03B3FBF6F300FB023301932E
:1091500022E6EFF311828CF3128887680368D90343
:1091600003D50123CEF8003087682368D2B2DEF839
:10917000001082F311882A68194406FB02F3DB1BF6
:10918000B3FBF2F306FB0131B6E5EFF311828CF38A
:10919000128887680368D90303D50123CEF800300D
:1091A00087682368D2B2DEF8001082F311882A683B
:1091B000194406FB02F3DB1BB3FBF2F306FB0131A0
:1091C000FFF7F9BBEFF311828CF31288876803680D
:1091D000D90303D50123CEF8003087682368D2B2C3
:1091E000DEF8001082F311882A68194406FB02F3A6
:1091F000DB1BB3FBF2F306FB0131FFF78DBBEFF393
:1092000011828CF3128887680368D90303D5012380
:10921000CEF8003087682368D2B2DEF8001082F3FF
:1092200011882A68194406FB02F3DB1BB3FBF2F337
:1092300006FB01316FE4EFF311828CF3128887682B
:109240000368D90303D50123CEF80030876823686B
:10925000D2B2DEF8001082F311882A68194406FBA6
:1092600002F3DB1BB3FBF2F306FB0131FFF7F8BBA4
:109270001C0903F00F03013C032C69D83A4A32F869
:10928000140040FA03F2D70762D5012202FA03F371
:10929000013B184039F0D0F9344B354A1B5D184476
:1092A00012EBC00354D09F8820210024B7FA87F521
:1092B0009971DC71C5F11F052E49039B6E1CD960A5
:1092C0003FF45DAA2C4B05A92C4E52F830000597AF
:1092D0000693775D07940894099434F0CFFB284AED
:1092E000039BD15D0C332748F02940F825307FF7E8
:1092F00046AAF021244B3E44D155DB68317CC3F3B0
:1093000002234AB2C3F107001D1D042828BF042010
:10931000062D88BFDC1E0123002A03FA00F303F1A7
:10932000FF3303F0030303FA04F34FEA031314DBE0
:109330001648DBB2104480F8003301F01F0101230E
:109340005209124803FA01F140F82210FFF717BA48
:10935000084B039AD360FFF712BA01F00F040C48D0
:10936000DBB220440376E8E7187604081476040894
:10937000B0C0012001800008000011106044040802
:1093800014B60120D4B5012000ED00E000E100E0BA
:10939000FCEC00E02DE9F04FA84A83B0436901904E
:1093A000934200F0908102F58062934200F08B813D
:1093B00038211A681027A24C4FF47A7522F0400227
:1093C000DFF888829F4E1A601A6822F038020A433A
:1093D0001A601A6842F040021A6010F0C1FEDFF80D
:1093E00070E2844698490120DEF80430C3F3080394
:1093F000002B40F02F81EFF31183002B40F02A81E6
:109400002368D1F8089000BF22689342F8D1D8F8B9
:1094100000A005FB0AF2A2EB0902B2FBFAF205FB7F
:1094200003239C45E0D0019D2846FFF79FF9EA6998
:109430001AB1938812681B049361019B5A6940F228
:10944000E93302E0002B00F056819168013B11F0F6
:10945000020F9BB2F6D06A2140F2E933117302E0A9
:10946000002B00F05E819168013B11F0010F9BB26F
:10947000F6D0D368019B5A6940F2E93302E0002B31
:1094800000F023819168013B11F0020F9BB2F6D0EE
:10949000102140F2E933117302E0002B00F0158136
:1094A0009168013B11F0010F9BB2F6D0D368019B8C
:1094B000DB6913B11A689B8893614FF0640ADFF887
:1094C00090914FF0100E60484FF47A755D4FD9F8C7
:1094D0000430C3F30803002B40F0DA80EFF311836C
:1094E000002B40F0D5802168826800BF2368994234
:1094F000F9D1D8F8006005FB06F39B1AB3FBF6F32D
:1095000005FB013101260091D9F80430C3F30803AB
:10951000002B5BD1EFF31183002B57D123688168B7
:1095200000BF22689342F9D1D8F800B005FB0BF2D6
:10953000521AB2FBFBF205FB0323009A9B1AB3F508
:109540007A7FE1D3BAF1010AC1D1019B3B4A5B6941
:10955000934205D002F58062934218BF4FF0080A8B
:109560001A684FF47A76384D22F04002354F1A606F
:109570001A6822F0380242EA0A021A601A6842F0B7
:1095800040021A6010F0ECFDDFF8C4C081464FF0D5
:10959000100E0120DCF80430C3F308038BBBEFF39B
:1095A000118373BB2368A96800BF22689342F9D175
:1095B000D8F800A006FB0AF2521AB2FBFAF206FB38
:1095C00003239945E6D003B0BDE8F08FEFF3118C8B
:1095D0008EF3128881680368DA0301D53E608168E2
:1095E00023685FFA8CFC3A688CF31188D8F800C0C5
:1095F0001A4405FB0CF35B1AB3FBFCF305FB0233C7
:109600009BE7EFF311818EF31288D5F808A02B6841
:10961000DB0302D53860D5F808A02368C9B23A68E0
:1096200081F31188D8F800101A4406FB01F3A3EB6C
:109630000A03B3FBF1F306FB0233C2E70038004034
:109640003CC2012038C2012010E000E040C20120ED
:1096500000ED00E0EFF3118987F31288D1F808A03C
:109660000B68DB0302D53060D1F808A023685FFAED
:1096700089F9326889F31188D8F800901A4405FBFB
:1096800009F3A3EB0A03B3FBF9F305FB0233C8E6C6
:10969000EFF311828EF3128886680368D90302D52E
:1096A00001233B6086682368D2B2396882F311884F
:1096B000D8F80020194405FB02F39B1BB3FBF2F31F
:1096C00005FB01311EE7302173E625498A4208D0A7
:1096D000244B9A4241D003F580639A427FF4E7AE6F
:1096E0000223214AD82101FB03239A89013292B235
:1096F0009A819B89DBE61A498A4208D0194B9A4223
:1097000029D003F580639A427FF4B6AE022316494E
:10971000D82000FB03139989013189B299819B8973
:10972000AAE60F498A4208D00E4B9A4211D003F59F
:1097300080639A427FF49EAE02230B4AD82101FB3C
:1097400003239A89013292B29A819B89019B5A69BB
:1097500092E60123F1E70123D9E70123C1E700BF26
:10976000003001400038004050BD0120F8B5D0F86D
:1097700018310446DA69910615D5586AE36AC0B211
:10978000002B00F0A280216B9847D4F818311A689A
:1097900022F480721A609A6822F001029A609A6933
:1097A00042F008029A61DA69D20701D501221A62F1
:1097B000DA69970701D502221A62DA69560701D5DC
:1097C00004221A62DA69150701D508221A62D4F850
:1097D000F820002A00F08580D969490600D4F8BD38
:1097E000D96904F58C701E680F079D6818D18F0623
:1097F00002D5B50600F1F1800F0602D5350600F15D
:10980000CE80480602D5710600F1A880002AE6D075
:10981000626AA36A9A427DD1012384F88C31F8BD33
:1098200015F001057BD116F4907FE5D011F001070A
:1098300000F0D18016F4807775D13D4605EA910796
:109840003FB104271F62D4F8847147F00207C4F8BF
:1098500084710F070AD5B70640F18F8008251D6275
:10986000D4F8845145F00805C4F88451D4F88451E3
:10987000002DCBD08F0605D5B50603D534F032FCCC
:10988000D4F81831D4F8842111076FD51A68202133
:1098900022F490721A609A6822F001029A6084F8A9
:1098A00082119A6852060DD59A68D4F87C1122F07C
:1098B00040029A6031B1574B08460B6528F048FECC
:1098C00000285ED1D4F8F820A0E7E3696269D0549B
:1098D000E369E1680133B3FBF1F201FB1233E361A9
:1098E00053E7D96908067FF577AF94F881112129EC
:1098F0003FF472AFA16A606A814249D0A069405CBE
:109900000131C0B298622569B1FBF5F005FB101179
:10991000A16261E72046BDE8F840FEF719BECF0717
:1099200009D5F70507D501271F62D4F8847147F0E0
:109930000107C4F88471EDB215EA51073FF47EAF18
:109940004FF0020E3D46C1F38007C3F820E0D4F883
:1099500084E14EF0040EC4F884E171E71968202018
:1099600021F04001196084F881014FE79A6812F0F4
:1099700040028BD1C4F88421A4E7002D3FF476AFD8
:109980006CE7D4F87C01036D9847D4F8F8203DE7E4
:10999000A4F86A21196821F0800119601CE794F885
:1099A000811121297FF432AFB4F86A1189B2C9B1AB
:1099B000D4F82011B1F5805F1DD0D4F86411481C93
:1099C000C4F8640109789962B4F86A31013B9BB22A
:1099D000A4F86A311AE73D463BE734F083FBD4F83C
:1099E000F82013E7196821F080011960196841F027
:1099F000400119600AE7D4F828110029DDD1D4F814
:109A0000641131F8020BC0F308009862C4F86411C5
:109A1000DAE700BFF5D20308114B98421ED003F5D8
:109A2000806398421AD0036823F04003036059B161
:109A300041F48071002991FAA1F3B3FA83F108BFD0
:109A40004FF0FF310139C900036823F0380319438F
:109A50000160036843F04003036070474908E2E790
:109A600000380040014B586980E600BF1CB6012059
:109A7000014B98687AE600BF1CB60120014B1868BC
:109A800074E600BF1CB60120F8B510F58C750446CD
:109A900014D0D0F818212421002380F881111168F6
:109AA00021F001011160136053609360C0F88431AC
:109AB00080F8803180F8813180F88231A279A36802
:109AC00012F00401C4F81C3100F0F8804FF4805308
:109AD000C4F8203112F0020300F029814FF4005342
:109AE0004FF48061C4F8243163790020C4F8281150
:109AF00013F00101C4F83001C4F83801C4F82C0196
:109B000002D00420C4F82C0113F0020605D0D4F8CA
:109B10002C0140F00800C4F82C01D0070DD549B144
:109B2000D4F83C014FF4803740F00200C4F844718F
:109B3000C4F83C01002E40F0E88012072AD5002D21
:109B400058D094F8813103F0FF02002B00F0E88038
:109B5000D4F818212423284684F88131136823F08F
:109B60000103136034F04CF9012840D0D4F83C31A3
:109B7000002B40F0D880D4F8183128465A6822F4D7
:109B800090425A609A6822F022029A609A6842F0E3
:109B9000080225E075B394F8813103F0FF020BB998
:109BA00084F88021D4F818212423284684F88131B0
:109BB000136823F00103136034F022F9012816D052
:109BC000D4F83C3113B1284634F0C2F8D4F8183137
:109BD00028465A6822F490425A609A6822F02A0273
:109BE0009A601A6842F001021A6034F07BF86379D7
:109BF00003F0010100292ED0D4F8F420002A75D0FA
:109C00000023D4F8FC004FF4806E4FF4803104F14F
:109C100034074FF48076E3632364A364E364A365AD
:109C2000E365636623666263A0633846C4F844E074
:109C30006165266528F0E4FC384628F01FFD94F89D
:109C40008231C4F87C71202BE5667AD0626B63792F
:109C50005268C4F80C219B072FD5D4F8F820002AAD
:109C60003DD0002340204FF48031C4F8942004F10B
:109C70009406D4F800214FF48067C4F89C00C4F81F
:109C800098203046C4F8A030C4F8A830C4F8AC30EE
:109C9000C4F8B030C4F8B830C4F8BC30C4F8C4302C
:109CA000C4F8C030C4F8A470C4F8B41028F0A8FCFC
:109CB000304628F0E3FC50B1FEE7F8BD12F0020395
:109CC000C4F8201138D1C4F8243119460CE7D4F86F
:109CD0009430C4F87861C4F8CC505860F8BDD4F81A
:109CE0008821136843F080031360F8BDD4F88821FD
:109CF000116841F480711160916841F00101916037
:109D0000116841F020011160A5E7D4F83C014FF43F
:109D1000003640F00100C4F84061C4F83C010CE793
:109D200084F8802114E7284634F012F823E7C4F8B9
:109D300024314FF48061D7E64FF40053C4F8243146
:109D4000D2E6E368626999B2002A3FF47FAFB1FAC4
:109D500081F67609002E7FF479AF94F8800101280E
:109D60003FF474AF0B46A4F8701138461549164FEE
:109D70004FF0010C4FF0220E61672767D4F81811DD
:109D8000124FC4F884612431C4F86C21C4F8846093
:109D900084F880C184F882E1C4F8807028F0ECFB7C
:109DA000D4F8183184F880611A6842F480721A601D
:109DB0009A6842F001029A609A6842F040029A6002
:109DC00044E700BF71D3030875D3030805D3030824
:109DD000417159E6816057E6B0B5BB4BB8B0BB499D
:109DE0001A6C00AFBA4842F08052BA4C1A641A6C2E
:109DF00002F08052C7F8D820D7F8D8201A6B42F466
:109E000080221A631A6B02F48022C7F8D420D7F894
:109E1000D4200A6842F480720A600268A24200F00C
:109E20004882AD4C4FF6FF05AC4AE168AC4829408A
:109E30000A43E2605A6F02601A6B42F480221A638E
:109E40001A6B02F48022C7F8DC20D7F8DC201A6BEA
:109E500042F480121A631A6B02F48012C7F8D02001
:109E6000D7F8D0201A6B42F480021A631A6B02F4FE
:109E70008002C7F8CC20D7F8CC201A6B42F00052F1
:109E80001A631A6B02F00052C7F8C820D7F8C8202E
:109E90001A6B42F080421A631A6B02F08042C7F8D4
:109EA000C420D7F8C4201A6B42F001021A631A6B5F
:109EB00002F00102C7F8C020D7F8C0201A6B42F0A8
:109EC00002021A631A6B02F00202C7F8BC20D7F82C
:109ED000BC201A6B42F004021A631A6B02F00402EF
:109EE000C7F8B820D7F8B8201A6B42F008021A63F6
:109EF0001A6B02F00802C7F8B420D7F8B4201A6B26
:109F000042F010021A631A6B02F01002C7F8B02078
:109F1000D7F8B0201A6B42F020021A631A6B02F0D5
:109F20002002C7F8AC20D7F8AC201A6B42F04002F0
:109F30001A631A6B02F04002C7F8A820D7F8A820CD
:109F40001A6B42F080021A631A6B02F08002C7F8A3
:109F5000A420D7F8A4201A6B42F480721A631A6BFB
:109F600002F48072C7F8A020D7F8A0201A6C42F043
:109F700001021A641A6C02F00102C7F89C20D7F89B
:109F80009C201A6C42F002021A641A6C02F002025F
:109F9000C7F89820D7F898201A6C42F004021A6487
:109FA0001A6C02F00402C7F89420D7F894201A6CB7
:109FB00042F008021A641A6C02F00802C7F89020F6
:109FC000D7F890201A6C42F010021A641A6C02F052
:109FD0001002C7F88C20D7F88C201A6C42F02002AF
:109FE0001A641A6C02F02002C7F88820D7F888207B
:109FF0001A6C42F040021A641A6C02F04002C7F870
:10A000008420D7F884201A6C42F080021A641A6CFB
:10A0100002F08002C7F88020D7F880201A6C42F442
:10A0200080721A641A6C02F48072FA67FA6F1A6C02
:10A0300042F400721A641A6C02F40072BA67BA6FC2
:10A040001A6C42F480421A641A6C02F480427A67F5
:10A050007A6F1A6C42F400421A641A6C02F40042DD
:10A060003A673A6F1A6C42F400321A641A6C02F4BE
:10A070000032FA66FA6E1A6C42F480221A641A6C84
:10A0800002F48022BA66BA6E1A6C42F400221A6494
:10A090001A6C02F400227A667A6E1A6C42F480120C
:10A0A0001A641A6C02F480123A663A6E1A6C42F420
:10A0B00000121A641A6C02F40012FA65FA6D1A6C36
:10A0C00042F480020EE000BF003802400070004001
:10A0D00004400240EFBEADDE00ED00E00005FA05F1
:10A0E000405F01201A641A6C02F48002BA65BA6DEE
:10A0F0001A6C42F400021A641A6C02F400027A65C7
:10A100007A6D1A6C42F000721A641A6C02F00072D6
:10A110003A653A6D1A6C42F000521A641A6C02F0F9
:10A120000052FA64FA6C1A6C42F080421A641A6C9B
:10A1300002F08042BA64BA6C1A6C42F000421A64AF
:10A140001A6C02F000427A647A6C5A6C42F0010296
:10A150005A645A6C02F001023A643A6C5A6C42F04A
:10A1600002025A645A6C02F00202FA63FA6B5A6CE9
:10A1700042F010025A645A6C02F01002BA63BA6BD1
:10A180005A6C42F020025A645A6C02F020027A6340
:10A190007A6B5A6C42F480725A645A6C02F4807280
:10A1A0003A633A6B5A6C42F400725A645A6C02F485
:10A1B0000072FA62FA6A5A6C42F480625A645A6C0B
:10A1C00002F48062BA62BA6A5A6C42F400625A645B
:10A1D0005A6C02F400627A627A6A5A6C42F48052D3
:10A1E0005A645A6C02F480523A623A6A5A6C42F4E7
:10A1F00000525A645A6C02F40052FA61FA695A6CBD
:10A2000042F480325A645A6C02F48032BA61BA69FC
:10A210005A6C42F400325A645A6C02F400327A6189
:10A220007A695A6C42F480225A645A6C02F4802291
:10A230003A613A695A6C42F480125A645A6C02F4D8
:10A240008012FA60FA685A6C42F480025A645A6CBE
:10A2500002F48002BA60BA685A6C42F400025A648E
:10A260005B6C03F400037B607B6827F0DDFF1D4B14
:10A2700002461D491B681D48A1FB03131C49A0FB96
:10A2800002029B09920C013B0A60B3F1807F08D265
:10A29000184AF02500200721536084F8235090606D
:10A2A0001160144AE037136843F004031360BD469D
:10A2B000B0BD114A01F5484102605A6C0F4842F4A2
:10A2C00080425A645B6C03F48043C7F8DC30D7F8F3
:10A2D000DC300A6803680A6083F30888084B1B684F
:10A2E0009847FEE7EC1C0120D34D621083DE1B4330
:10A2F00040C2012010E000E0EDFEFECA0000F01FA9
:10A300000400F01F08B5054B1B6803B19847044BC8
:10A31000044A1A6072B6FDF7E9FE00BFAC400120A6
:10A3200004400240EFBEADDE08B5034B1B6803B12D
:10A33000984772B6FDF7DAFEAC40012030B40D4DFF
:10A34000372400222B4604E001322433092A0DD0A1
:10A350001C79A042F8D19C79214201D10029F3D186
:10A3600002EBC20205EB820030BC7047002030BC1B
:10A37000704700BF2C63040830B5F02287B000217D
:10A38000234839F0FEFF234A0123234C116C04F5C6
:10A39000A27519431164116C194001910199116C56
:10A3A00041F002011164116C01F002010291029965
:10A3B000116C41F008011164116C01F00801039166
:10A3C0000399516C41F002015164516C01F002019A
:10A3D00004910499516C41F480315164526C02F43F
:10A3E00080320592059A2BB92434AC420DD0A37962
:10A3F000002BF9D02079243410F038F914F81C2CF3
:10A40000022110F0FDF9AC42F1D107B030BD00BF20
:10A4100004B70120003802402C63040801490248B7
:10A42000FEF74EB9A4B7012000400140014902489F
:10A43000FEF746B97CB7012000040140FFF7F6BFE4
:10A4400001490248FEF73CB954B70120000C004016
:10A4500001490248FEF734B92CB70120000400403E
:10A4600002494FF08040FEF72BB900BF04B701202E
:10A470000368134A9B0A93421FD010D8B3F5801F7C
:10A4800019D0023A934213D1012142790223890162
:10A490000C48DA4041589340DB430B6170470A4A4D
:10A4A000934206D00F32934201D10421EDE7704769
:10A4B00070470321E9E70021E7E70221E5E700BF54
:10A4C00003001000545D01204100100003681B4A86
:10A4D0009B0A93422FD013D8B3F5801F29D0023A9C
:10A4E000934222D10123A1B99B0141790222144850
:10A4F000D140C0588A40C36823EA0203C360704752
:10A50000104A934213D00F3293420FD104230029F3
:10A51000EAD002229B0141790948D140C05802FA91
:10A5200001F3C2681343C360704770477047032349
:10A53000D9E70023D7E70223D5E700BF03001000C7
:10A54000545D01204100100003682DE9F0439B0A8F
:10A55000554CA34200F0918028D8B3F5801F00F03D
:10A560009080023CA3427CD1407901244F4F860861
:10A5700041BBA5014FF0020E4FEA840C57F805804D
:10A5800020FA0EF00CEB04050EFA00FED8F80C00D1
:10A5900006EB450520EA0E00DFF818E12E1DC8F88D
:10A5A0000C004EF825104EF8262025E0404CA34222
:10A5B00065D00F34A34256D1042440793B4F86081E
:10A5C0000029D6D04FEA841E02254FEA840C57F8A2
:10A5D0000E8005FA06F00CEB040ED8F80C9006EB92
:10A5E0004E05DFF8D0E040EA09002E1D4EF8251098
:10A5F0004EF82620C8F80C002B4A934247D034D896
:10A60000B3F5801F41D0023A934248D101260CEBAA
:10A610000403DB0003F120007044EFF311855022A6
:10A6200082F312881033002273441968013211B189
:10A63000016018680430042A03F10403F5D10023F3
:10A64000EDB2036085F311886444B6010EEBC404D7
:10A65000BA59236AEBB1D36843F00103D360BDE874
:10A66000F083BDE8F083BDE8F083114A93420AD03D
:10A670000F32934215D10426C9E702249DE7032433
:10A680009BE7002499E70326C1E70026BFE70226DF
:10A69000BDE7D36823F00103D360BDE8F083BDE8D4
:10A6A000F083BDE8F08300BF03001000545D01207B
:10A6B0004100100004B70120F0B5830A544C85B066
:10A6C000A34200F0A08040D8B3F5801F00F099802D
:10A6D000023CA34237D10125AD014E4E7359771983
:10A6E000984230D04C4B01394FF0000E04461B68A5
:10A6F00089B270513846F960C7F810E0C7F808E031
:10A70000C7F814E0B3FBF2F2013A7A6028F02EF9B0
:10A710004249B4F1804F18BF8C420CBF0121002187
:10A720001BD03F4B9C4218D003F580639C4214D051
:10A730003C4A03F57C439C4218BF94420DD003F57C
:10A7400070539C4209D005B0F0BD374CA34256D09F
:10A750000F34A342F7D10425BEE7721900234FF44A
:10A76000805792F83C0001930128029303930097CD
:10A77000E9D070590227DFF8B8E04FF0010C82F8F9
:10A780003D70876807EA0E0E284FC0F808E0D0F841
:10A7900008E00EEA0707876082F83C3082F83DC087
:10A7A000B9B91F4B9C4214D003F580639C4210D072
:10A7B00003F580639C4203D003F578439C42C2D1E9
:10A7C0007219002392F83C200093012A019302930E
:10A7D000B9D0735911485A688342996815D000F569
:10A7E0008060834211D022F0700221F08001354454
:10A7F00000205A60996085F83C0005B0F0BD032543
:10A800006AE7002568E7022566E722F47002EAE7B6
:10A8100003001000545D0120EC1C012000000140E9
:10A8200000040040000C004041001000F8FFFEFF53
:10A830008800FEFFF8B50668324CB30AA34239D04F
:10A8400007D8B3F5801F37D0023CA3422ED1012593
:10A8500006E02D4CA3422BD00F34A34227D1042570
:10A8600004463046FFF728FF284AAB010220216842
:10A870000127D518D658264A002385F83D003468AC
:10A8800024483C43346085F83D7001E050F83320A3
:10A89000914213D001330E2BF8D10020012136F064
:10A8A00031FB0020BDE8F84032F02CBFF8BDF8BD08
:10A8B0000325D5E70225D3E70025D1E7154A012175
:10A8C00002EBC3035C7965B2284636F01BFB2846D1
:10A8D00032F018FF1B2C0AD02E2C11D101212C2074
:10A8E00036F010FB0C4B4FF480525A60F8BD01213A
:10A8F000192036F007FB084B4FF000721A60F8BDC4
:10A90000F8BD00BF0300100041001000545D01209D
:10A9100000000140686D040800E100E0800A0E4B71
:10A92000984216D007D8B0F5801F10D0023B98424D
:10A9300009D10A4870470A4B984206D00F33984213
:10A9400001D1084870470020704707487047074802
:10A9500070470748704700BF03001000945D012056
:10A9600041001000545E0120145E0120545D01205E
:10A97000D45D0120F8B5464F05027C196368002BB1
:10A980003ED09B69002B3BD0227C0646414B0020E9
:10A9900042EA4101207420468AB21B68111281EA02
:10A9A0001211514001F00F0141EA021189B298479A
:10A9B00063685B799B08B0B194F8FE104A2200EB03
:10A9C000861412FB0131344A053405F1140302EBFD
:10A9D000810207EB84043B4453F8041B1032A3426A
:10A9E00042F8081CF8D13D44B5F8FC3003EB86165C
:10A9F00007EB8607FA6F92F83530DBB2012B00D0F7
:10AA0000F8BD92F834100129FAD092F8351095F873
:10AA1000FE600129EC6D956D82F8343003D000237F
:10AA200082F83430ECE74FF0020E002703B21168D1
:10AA300082F835E04C34576503FA0EF3174F4FF4A4
:10AA4000947E08680EFB0676976820F48020402FDD
:10AA500008604B6018D08E60CC60D06D3F23126CC4
:10AA60008340AB600B6843F016030B604B6943F007
:10AA700080034B611AB10B6843F008030B600B684D
:10AA800043F001030B60F8BD8C60CE60E5E700BFCA
:10AA9000B07E0120A47E0120B4860120BC86012066
:10AAA00030B44468012B24F4805444601CDD40F22F
:10AAB000E93401E0013C35D08568AD07FAD50029BD
:10AAC0003DD031F8024B848140F2E93401E0013C91
:10AAD00028D08568ED07FAD5C468A4B20AB122F877
:10AAE000024B023B012BE2DC446844F48054446096
:10AAF00013B340F2E93301E0013B37D08468A40787
:10AB0000FAD5002936D00B78037340F2E93301E01F
:10AB1000013B2BD08168C907FAD5C368DBB25AB1B3
:10AB2000137009E0144B98420CD0144B984219D082
:10AB300003F58063984217D0012030BC70474FF670
:10AB4000FF74C0E723460E4AD82101FB03239A89EC
:10AB5000013292B29A81988980B2003030BC18BF1D
:10AB6000012070470123EEE70223ECE7024A9042FE
:10AB7000DBD1E8E7FF23C7E70030014000380040A1
:10AB800050BD012070B5C36982B004461BB19A88DC
:10AB9000196812048A6107236A4611496069FFF740
:10ABA0007FFFE36913B11A689B8893619DF80130B8
:10ABB00001209DF802109DF8036041EA03219DF8F1
:10ABC00004209DF805509DF8063042EA0622A18730
:10ABD00043EA0523E287A4F8403002B070BD00BF0D
:10ABE000784404082DE9F04F037C85B00446012B1E
:10ABF0004CD0022B45D1C3691BB19A881968120445
:10AC00008A61606940F2E93301E0002B63D0826819
:10AC1000013B12F0020F9BB2F7D0C32240F2E9339E
:10AC2000027301E0002B6DD08268013B12F0010F2E
:10AC30009BB2F7D0C3686069062302AA0021FFF720
:10AC40002FFFE36913B11A689B8893619DF8083060
:10AC500001259DF809109DF80C0041EA03219DF89B
:10AC60000A609DF80B209DF80D3042EA0622A1876C
:10AC700043EA00232846E287A4F8403005B0BDE847
:10AC8000F08F0025284605B0BDE8F08F90F91460DC
:10AC9000042ED4BF00250125B6F1FF3F08BF45F0C3
:10ACA0000105002DEDD17700DFF81C83BA1908EB00
:10ACB0004212D2F814E0BEF1000FE3D092F8551022
:10ACC000202935D0B64A2846138801339BB2138019
:10ACD00005B0BDE8F08FB34A904207D0B24B98421E
:10ACE0000ED003F580639842A6D10223AF4AD82143
:10ACF00001FB03239A89013292B29A819B899BE7D7
:10AD00000123F3E7A74A904207D0A74B98426AD0A5
:10AD100003F5806398428ED10223A44AD82101FB17
:10AD200003239A89013292B29A819B89606983E7F1
:10AD300092F854100129C5D09D4894F81590D0F888
:10AD400000A082F8543004E00368A3EB0A03192B37
:10AD50003DD8DEF8181011F40041F5D1B8194FEACA
:10AD600049034FF0220C402240010093019208EB6E
:10AD70000009143089F855C043F4903C4FF00603A5
:10AD800089F8562008EB000BC9F85810A9F83E3096
:10AD900002ABDEF80400C9F848108649C9F838301B
:10ADA000014058464CEA010C5146CEF804C02AF046
:10ADB00075FFD0B1D9F85830374408EB47139A6D76
:10ADC000042A00F0C680002283F854207AE7374432
:10ADD0000023202208EB471888F8552088F85430C3
:10ADE00088F856306EE7012397E7019A4323D9F894
:10ADF000140011465246836258462AF079FF002813
:10AE0000DAD1B9F83E2092B2FF2A40F28580602163
:10AE1000009B694A4FF0FF0E01FB06811A43486907
:10AE2000A1F83CE0436823F07F7323F4593323F403
:10AE30007F7323F003031A434260604B3744009A48
:10AE400008EB4719019513435546BA4627461C4659
:10AE500005E0B9F83E2092B2002A00F081802A462F
:10AE6000042158462AF044FF002853D1D9F838204D
:10AE7000D9F81410501C496AC9F838001170B9F893
:10AE80003C20B9F83E10013A013992B289B2A9F8D2
:10AE90003C20A9F83E10002ADBD1B9F83E2092B23E
:10AEA000002AD6D080212A4658462AF021FF009B4E
:10AEB000FF2143F0007E68BBB9F83E2092B28A427F
:10AEC0000FD9D9F81400A9F83C10426822F07F721B
:10AED00022F4593222F47F7222F0030222434260AC
:10AEE000B7E7D9F81410B9F83EC04A681FFA8CFCCD
:10AEF00022F07F725FFA8CF0A9F83CC022F459323C
:10AF000022F47F7222F0030242EA0E0242EA004279
:10AF10004A609EE7019DD5E64FF0600E009B284AEF
:10AF20000EFB068E1A43DEF81400BEF83E1043688E
:10AF300089B223F07F73AEF83C10C9B223F45933C1
:10AF400023F47F7323F00303134343EA0143436075
:10AF500073E76023002203FB068686F85420B1E6DF
:10AF60003C465746AA465846019D51462AF0E0FE07
:10AF700020B1602303FB0686B36DA3E6D9F8143035
:10AF80002021104D08EB4717D9615A682A405A60B2
:10AF900089F8551087F8540089F8560056E600BF26
:10AFA000883E0120003001400038004050BD0120A3
:10AFB000A85B0120009800FC0024FF010000FF01B5
:10AFC0000024000200E800FED45B01202DE9F04FD0
:10AFD000037A85B00446012B4BD0022B44D1436940
:10AFE0001BB19A88196812048A61E06840F2E9335B
:10AFF00001E0002B62D08268013B12F0020F9BB28D
:10B00000F7D0BB2240F2E933027301E0002B6CD091
:10B010008268013B12F0010F9BB2F7D0C368E06871
:10B02000062302AA0021FFF73BFD636913B11A68EA
:10B030009B8893619DF8083001259DF809109DF8C3
:10B040000C0041EA03219DF80A609DF80B209DF851
:10B050000D3042EA0622618343EA00232846A28398
:10B06000E38305B0BDE8F08F0025284605B0BDE8B4
:10B07000F08F90F90C60042ED4BF00250125B6F1A5
:10B08000FF3F08BF45F00105002DEDD17700DFF847
:10B090001C83BA1908EB4212D2F814E0BEF1000F7B
:10B0A000E3D092F85510202935D0B64A28461388A7
:10B0B00001339BB2138005B0BDE8F08FB24A9042D5
:10B0C00007D0B24B98420ED003F580639842A7D1C7
:10B0D0000223AF4AD82101FB03239A89013292B29D
:10B0E0009A819B899CE70123F3E7A74A904207D006
:10B0F000A64B98426AD003F5806398428FD1022311
:10B10000A34AD82101FB03239A89013292B29A8182
:10B110009B89E06884E792F854100129C5D09D48C6
:10B1200094F80D90D0F800A082F8543004E0036841
:10B13000A3EB0A03192B3DD8DEF8181011F40041D7
:10B14000F5D1B8194FEA49034FF0220C40224001D3
:10B150000093019208EB0009143089F855C043F4BC
:10B16000903C4FF0060389F8562008EB000BC9F815
:10B170005810A9F83E3002ABDEF80400C9F84810B8
:10B180008549C9F83830014058464CEA010C51460F
:10B19000CEF804C02AF082FDD0B1D9F85830374437
:10B1A00008EB47139A6D042A00F0C680002283F84A
:10B1B00054207AE737440023202208EB471888F808
:10B1C000552088F8543088F856306EE7012397E709
:10B1D000019A3B23D9F8140011465246836258461F
:10B1E0002AF086FD0028DAD1B9F83E2092B2FF2A73
:10B1F00040F285806021009B684A4FF0FF0E01FB02
:10B2000006811A434869A1F83CE0436823F07F7344
:10B2100023F4593323F47F7323F003031A4342606A
:10B220005F4B3744009A08EB471901951343554685
:10B23000BA4627461C4605E0B9F83E2092B2002ADD
:10B2400000F081802A46042158462AF051FD00284A
:10B2500053D1D9F83820D9F81410501C496AC9F8CC
:10B2600038001170B9F83C20B9F83E10013A0139A4
:10B2700092B289B2A9F83C20A9F83E10002ADBD18D
:10B28000B9F83E2092B2002AD6D080212A465846EC
:10B290002AF02EFD009BFF2143F0007E68BBB9F829
:10B2A0003E2092B28A420FD9D9F81400A9F83C1076
:10B2B000426822F07F7222F4593222F47F7222F027
:10B2C000030222434260B7E7D9F81410B9F83EC030
:10B2D0004A681FFA8CFC22F07F725FFA8CF0A9F8A2
:10B2E0003CC022F4593222F47F7222F0030242EA77
:10B2F0000E0242EA00424A609EE7019DD5E64FF009
:10B30000600E009B274A0EFB068E1A43DEF81400DF
:10B31000BEF83E10436889B223F07F73AEF83C104C
:10B32000C9B223F4593323F47F7323F00303134387
:10B3300043EA0143436073E76023002203FB068670
:10B3400086F85420B1E63C465746AA465846019D29
:10B3500051462AF0EDFC20B1602303FB0686B36D55
:10B36000A3E6D9F8143020210F4D08EB4717D96117
:10B370005A682A405A6089F8551087F8540089F8AD
:10B38000560057E6883E012000300140003800405A
:10B3900050BD0120A85B0120009800FC0024FF01A3
:10B3A0000000FF010024000200E800FED45B012041
:10B3B000F8B5D823604D614A044603FB00F3E95811
:10B3C0002B44914200F09580D823661C03FB045364
:10B3D000F6B218790FF04AF9074610B11223C67178
:10B3E0008371D82303FB045358790FF03FF910B150
:10B3F0001323C6718371D82303FB045398790FF08C
:10B4000035F910B11423C6718371D82303FB04539B
:10B410009A7B002A5CD0DA7938464E210FF0F0F999
:10B42000D82606FB04F6AF1978790FF01FF93A7A9F
:10B430002E210FF0E5F9B8790FF018F97A7A0E217C
:10B440000FF0DEF9AB593E491A688B4222F04002F8
:10B450001A6051D03B4A934258D0384A934260D048
:10B46000394A93423AD0394A934209D102F56842A7
:10B47000516A41F480115162516A21F48011516284
:10B48000D822596802FB045441F48051A27B5960D0
:10B49000002A196814BF0024022449060FD41D682D
:10B4A00082F001022A482B492840024342F44572A7
:10B4B00022431A605A68114041F4E0615960DA6928
:10B4C00022F40062DA611A6842F040021A60F8BDA4
:10B4D000DA7938462E210FF093F9A1E702F582328E
:10B4E000516A41F400515162516A21F40051516294
:10B4F000C6E701229A7367E7174A516A41F48051FF
:10B500005162516A21F480515162B9E702F500326B
:10B51000116A41F480411162116A21F48041116283
:10B52000AEE702F5FE32116A41F400411162116A80
:10B5300021F400411162A3E750BD0120003C00400E
:10B54000003001400038004000340140005001400C
:10B550004000FFFFFBF0FFFF0038024070B5C0EB7A
:10B56000C0000D4C0D4E82B004EB8004306B256999
:10B5700028433063366B94F90D003540A160636158
:10B5800091090195019B35F0BDFC94F90D0032F055
:10B59000B9F802B070BD00BF8C1501200038024020
:10B5A0000A4BC0EBC00030B403EB8000084C82B003
:10B5B000256B03691D432563246B01762340427686
:10B5C0000193019B02B030BC704700BF8C15012075
:10B5D000003802400348D0F8AC3113B100F5D27006
:10B5E000184770478C1501200348D0F8903113B1EB
:10B5F00000F5C470184770478C1501200348D0F837
:10B60000743113B100F5B670184770478C150120DE
:10B610000348D0F8583113B100F5A87018477047A7
:10B620008C1501200348D0F83C3113B100F59A7015
:10B63000184770478C1501200348D0F8203113B10A
:10B6400000F58C70184770478C1501200348D0F81E
:10B6500004310BB1FC301847704700BF8C15012036
:10B660000348D0F8E8300BB1E0301847704700BF0E
:10B670008C1501200348D0F8CC300BB1C4301847EA
:10B68000704700BF8C1501200348D0F8B0300BB1D3
:10B69000A8301847704700BF8C1501200348D0F828
:10B6A00094300BB18C301847704700BF8C150120C7
:10B6B0000248836F0BB17030184770478C1501201A
:10B6C0000248C36D0BB15430184770478C150120E8
:10B6D0000248036C0BB13830184770478C150120B5
:10B6E0000248436A0BB11C30184770478C15012083
:10B6F0000248836803B11847704700BF8C150120CA
:10B70000084810B4D0F8D430D0F8084199691A68C4
:10B7100024B12346D4305DF8044B18475DF8044B40
:10B72000704700BFD45B0120254BD3F8D4108A6941
:10B73000086810B4D4051FD504062DD5D3F8180118
:10B740004FF4807440F00100C3F818015005CC613B
:10B7500032D5D3F818014FF48064920540F0080008
:10B76000C3F81801CC611DD4D3F8182112F00B0FC7
:10B770000BD15DF8044B704754050FD50006E8D493
:10B78000D3F8182112F00B0FF3D0D3F818110D488D
:10B790005DF8044B31F0C2BF5405E5D49405E3D500
:10B7A0000206E1D5D3F818214FF4007042F00202EE
:10B7B000C3F81821C861D7E79205F3D4D4E700BFD6
:10B7C000D45B0120A85C0120074810B4436FD0F877
:10B7D000A84099691A6824B1234674305DF8044B77
:10B7E00018475DF8044B7047D45B0120244B596F18
:10B7F0008A69086810B4D4051FD504062DD5D3F87E
:10B80000B8004FF4807440F00100C3F8B800500550
:10B81000CC6132D5D3F8B8004FF48064920540F083
:10B820000800C3F8B800CC611DD4D3F8B82012F0DA
:10B830000B0F0BD15DF8044B704754050FD5000674
:10B84000E8D4D3F8B82012F00B0FF3D0D3F8B81027
:10B850000C485DF8044B31F061BF5405E5D4940504
:10B86000E3D50206E1D5D3F8B8204FF4007042F0DA
:10B870000202C3F8B820C861D7E79205F3D4D4E731
:10B88000D45B0120485C0120074810B44369846CF4
:10B8900099691A6824B1234614305DF8044B18479F
:10B8A0005DF8044B704700BFD45B0120204B596901
:10B8B0008A69086810B4D4051AD5040626D5986D8F
:10B8C0004FF4807440F0010098655005CC612BD591
:10B8D000986D4FF48064920540F008009865CC6143
:10B8E0001AD49A6D12F00B0F0AD15DF8044B704711
:10B8F00054050DD50006EBD49A6D12F00B0FF4D061
:10B90000996D0C485DF8044B31F008BF5405E8D43C
:10B910009405E6D50206E4D59A6D4FF4007042F026
:10B9200002029A65C861DCE79205F5D4D9E700BF49
:10B93000D45B0120E85B0120A54A0021A54BA64865
:10B9400070B5D2F888404FF00065A44EA4B044F41E
:10B950007004C2F888401C6844F001041C609960BF
:10B960001C68204018605E60186820F48020186011
:10B97000D9609560BFF34F8FBFF36F8FC2F850123D
:10B98000516941F400315161BFF34F8FBFF36F8FA5
:10B99000196C934A41F080511964196C01F080517F
:10B9A00002910299116841F440411160126802F459
:10B9B00040420192019A9A6802F00C02042A52D085
:10B9C0009A6802F00C02082A4AD0824B854C1A6809
:10B9D000194642F480321A60226803E023689B1AF9
:10B9E000642B3CD80B689803F8D57A4B9A6802F020
:10B9F0000C02082A33D01A68184622F080721A60A6
:10BA0000226803E023689B1A022B28D803689B0155
:10BA1000F8D447F6C07393FAA3F34FF44031B3FA66
:10BA200083F291FAA1F14FF0706191FAA1F1092628
:10BA3000B1FA81F14FF4D8736B4D8E406549934054
:10BA400033431D434560036843F0807303602268FD
:10BA50000B689E010BD423689B1A022BF8D9FEE7D2
:10BA60005B685C02B1D55B4B5E4C1B68BDE7086C44
:10BA70005B4A40F0805013460864096C01F0805125
:10BA800003910399116841F48031116021685A686B
:10BA9000D50305D42268521AB2F57A7FF7D9FEE7AA
:10BAA0001A684F4942F400321A60226804E02368A1
:10BAB0009B1AB3F57A7FF2D84B689803F7D54FF409
:10BAC00000164FF000654FF4C0710722032304A84D
:10BAD00004962195089109920A9336F07FFF00B1F0
:10BAE000FEE7424A136803F00F03062B1BD9394BBC
:10BAF0009A6822F0F0029A601A68920167D59A68F3
:10BB0000184641F2883122F0030242F002029A60A4
:10BB10002268836803F00C03082B10D023689B1A5B
:10BB20008B42F6D90AE0136823F00F0343F00703B2
:10BB30001360136803F00F03072BD8D0FEE72B4ADE
:10BB4000136803F00F03072B35D8224CA36823F4A6
:10BB5000E05343F4A053A360A36823F4604343F489
:10BB60000043A36026F060FBA368F02292FAA2F2E1
:10BB7000B2FA82F203F0F0031D4ED3401D4D334460
:10BB800093F8203020FA03F32B6035F0EFF900230F
:10BB9000194A04A8049213931493159316931793B8
:10BBA000189319931A931B931C931D931E9336F0AD
:10BBB00015FF18B3FEE7136823F00F0343F00703E4
:10BBC0001360136803F00F03072BB7D1BDE7B5E788
:10BBD00000ED00E000380240FFFFF6FE10300024C8
:10BBE00000700040A85B012008004020003C02409B
:10BBF00060440408EC1C0120C0FF0300D4F88C3022
:10BC000023F08073C4F88C30D4F88C3043F0807308
:10BC1000C4F88C30A36803F00C03042B27D0082B46
:10BC20000DD0154B154A16499268C2F303121644FB
:10BC300096F82020D3408B422B601AD0FEE7616833
:10BC400062684B02616802F03F024CBF0D4B0A4B29
:10BC5000B3FBF2F3C1F3881203FB02F3074A526805
:10BC6000C2F3014201325200B3FBF2F3DAE7054BB3
:10BC7000D8E724B070BD00BF0024F40000380240B3
:10BC800000E6DF0C00127A002DE9F04F2DED028B5B
:10BC900093B006462DF032FFB24B1D7825B113B09C
:10BCA000BDEC028BBDE8F08FAF4B1B685805F6D595
:10BCB000AE4F3A68002A00F01A81AD4CAD4BD4F873
:10BCC00028110B449E42C0F0128194F82C31DFF809
:10BCD00000830133C4F82861D8F80010DBB289076B
:10BCE00084F82C3101F1BF8513F0070901F00485B8
:10BCF000282B01F0FB86A04B03935E2090479F4BBF
:10BD00001B78002B6AD09A4C9D4AD4F83431F31A30
:10BD1000934201F2A783DFF8BC9299F800A0BAF130
:10BD2000000F32D1DFF86882D8F800000EF0BEFBB9
:10BD3000C0B201280ED9022841F09587914F3B7877
:10BD4000002B42F0F780D4F83C31F31AB3F57A6F48
:10BD500082F0A8818C4F3A68002A3FD099F80030D1
:10BD6000B3B98A4B0221D8F800001B689B781E3BB0
:10BD7000012B42F2F28004301DF078FB01220023F7
:10BD800089F8002084F8483126E07F4F3A682AB3CA
:10BD9000D4F8443140F6B731F31A8B421ED994F8E7
:10BDA0004031002B01F05587013BDBB284F8403174
:10BDB000002B01F0C48594F848E194F8493112F859
:10BDC000011B734801338E443A60006884F848E1EF
:10BDD00084F849310EF06EFBC4F84461039B6D4A50
:10BDE0001B6812780133012A0A9301F063826A4BBF
:10BDF0001B786BB1694F3B6853B1039B5C4CD3F824
:10BE00000090D4F85C31A9EB0303632B01F2888125
:10BE1000DFF8C48198F80090B9F1020F01F069854C
:10BE2000584F97F87430032B01F02E845C4B1B782D
:10BE300073B15C4D2B685BB14D4C0EF091F944F63B
:10BE40001F620490D4F86831C31A934200F2D8807C
:10BE5000554B1B78002B4DD1544B1B7843B1444CB0
:10BE600048F2E803D4F8B82213449E4281F09A8243
:10BE70004F4B1B78002B3FF412AF3D4E4D4C06F25A
:10BE8000C1274D4D20680EF011FB00283FF407AF8D
:10BE900020680EF003FB2B7880465A1E33B12068D1
:10BEA0002A700EF003FB0028F2D1F8E6032239468F
:10BEB000781E38F04CFA96F8C0124FF6FF7396F8D9
:10BEC000C12286F8C3821FFA88F84B409B1A9BB2A6
:10BED000B8EB132FD6D1DBB296F8C2229A42D1D159
:10BEE000781E1CF06DFC2B7818442870CAE7224B92
:10BEF000039304E7314C2278002A41F0D281DFF825
:10BF0000DC8098F80040002C6AD12D4D297800295A
:10BF100041F094872B4D2C4B2A78154C93FBF2F370
:10BF2000D4F8B02213449E4296D3284A94F8B432EF
:10BF3000C4F8B062D75CF80702F1F880B90702F1E3
:10BF4000BF817A0702F185813A0702F10A8094F8ED
:10BF5000B4322978013393FBF1F201FB123384F8F8
:10BF6000B43279E7C7370120E0560120903D012027
:10BF7000E01E012048E801003CC201203693012068
:10BF80003F0D030000000120883D0120843D012079
:10BF9000803D01203793012044930120FC3C012087
:10BFA0004C93012050930120BC930120CD9301209C
:10BFB000569301205C930120609301202893012077
:10BFC000C4930120CC930120A0860100C8930120D6
:10BFD000143D01208C3D0120962D0120C5930120A8
:10BFE000054F386E002841F038858246034B88F8AB
:10BFF00000A0C3F8B0622FE7D4930120E01E012017
:10C0000094F86E31002B41F0AA84DB4A48F60340D5
:10C010004AF60B4E4BF60F43126849F6074702F0FB
:10C02000080100294FF0190104BF0746734612F0BA
:10C03000040F84F86E1118BF1F46900603D547F40D
:10C04000804747F020072FF0A5FFC7F3090A002813
:10C0500042F05782C94B9B79002B42F0D882984618
:10C0600064204FF0FF3900230122FE210DF1280E3C
:10C070000A974FF01F0C0B97CDF830A0ADF8368023
:10C08000ADF838908DF84600ADF83430CDF83A3040
:10C09000CDF83E30CDF842306371E271A170B84FF7
:10C0A00084F803C0BEE80F000FC79EE80F0007C763
:10C0B0001A0C27F8023BC8233946781CA37101F8F3
:10C0C0001E2994F87E2182F0F103571C227183EA25
:10C0D000031384F87E71DAB2130983F0E70343EAAD
:10C0E000022383EAC2031BB283EA0312C3F30723CA
:10C0F000D2B283EA121343EA022383EAC2031BB2D9
:10C1000083F0C802C3F3072382EA0212D2B283EAA1
:10C11000121343EA022383EAC2031BB283F001072E
:10C12000C3F3072287EA0713DBB282EA131242EA5B
:10C13000032282EAC3021746228011F8013B7B40AA
:10C14000814283EA0313DBB24FEA131282EA172219
:10C1500042EA032282EAC3031BB29FB22780ECD1DA
:10C1600083F07C03DFF830C204F1220883EA031372
:10C170000CF5D379DBB24FEA131E8EEA172E8EEA46
:10C18000032E8EEAC30E0FFA8EFE1FFA8EF35FFAAD
:10C190008EFE4FEA132A238084F827E084F828A033
:10C1A000DCF800000CF1100C5CF80C1C4F465CF83D
:10C1B000082C09F110095CF8043CC4450FC7EFD105
:10C1C000DCF800006F4FC9F8000007F127089CF861
:10C1D000043089F8043084F8CDE184F8CEA117F852
:10C1E000011F28680EF066F9B845F8D194F86F1170
:10C1F000002941F0B983644B0A2203981B78006838
:10C2000084F86F210590002B01F04F855F4A012BC8
:10C21000B2F8008042F2F381022B578802F0898144
:10C220009088032B069002F0B282042BB2F806C06D
:10C2300002F0A882052BB2F808B002F09F82062B0C
:10C24000B2F80AA002F0D881072B908900D0D189DA
:10C2500094F87E914FF0000E4D4A89F0300368F358
:10C260000F0E12884FF0000867F31F4E83EA031386
:10C27000059FC2EB0222DBB2CDF82CE00A97454FB6
:10C280004FEA131E059387FB0273069F8EF07A0E0A
:10C2900084F8049067F30F081F46059B17446CF35E
:10C2A0001F484EEA032E4FF0000CD217CDF8308015
:10C2B0008EEAC3034FF01608C2EB672267461BB233
:10C2C0006BF30F0C60F30F078DF83D206AF31F4CE2
:10C2D00009F1010261F31F4783EA0311C3F3072346
:10C2E000CDF834C0C9B24FF0C80C84F87E214FF0AD
:10C2F000230A83EA111384F80380002084F806C01F
:10C3000043EA01230DF1280E0E974FF0FE0983EA50
:10C31000C1038DF83C0060711BB2194F84F807A06F
:10C3200083EA0C02C3F3072384F8029082EA021125
:10C33000C9B283EA111242EA012282EAC10212B2B0
:10C3400082EA0A03C2F3072C83EA03185FFA88F82B
:10C35000BEE80F008CEA181C0FC74CEA08239EE8C1
:10C36000030083EAC80347F8040BB81C238027F8AE
:10C370001419194612E000BF143D0120043D0120AC
:10C38000E81E012087200120543E0120247D012049
:10C390007092012003082080E21E012017F8012B73
:10C3A0004A40874282EA0212D2B24FEA121383EA6B
:10C3B000112343EA022383EAC20212B291B221801E
:10C3C000ECD182F0F402DFF80C9404F2A71704F227
:10C3D000C51882EA0212D9F8000009F5D37CD2B25E
:10C3E0004FEA121E8EEA112E8EEA022E8EEAC20E3D
:10C3F0000FFA8EFE1FFA8EF35FFA8EFE4FEA132AB3
:10C40000238084F81EE084F81FA0D9F80410D9F81E
:10C410000820D9F80C30ACE80F00D9F81000D9F892
:10C420001410D9F81820ACE8070084F8C5A184F8E6
:10C43000C4E117F8011F28680EF03CF8B845F8D1A0
:10C4400094F87231002B41F09F82DF4B19221B6858
:10C4500084F87221990640F11B83DC4B1B789A0704
:10C4600041F14486DFF8788398F81430042B8CBFB0
:10C470004FF0030A4FF0020A0DF072FEB8F81030C8
:10C48000B8F808204FF47A7103EB83030A900AAFDF
:10C4900001FB02F2D8F800005B000E92BE46ADF838
:10C4A00042304FF000090C904FF0FF31B8F80E30D9
:10C4B0004FF0C80C98F81420D8F804008DF844A068
:10C4C0004FF0180A0D90ADF840308DF84520CDF8AA
:10C4D0002C900F910597BE4FBEE80F000FC79EE846
:10C4E0000F0007C73A461E20B91CFE2722F81C3948
:10C4F00094F87EE1E0708EF07803A77084F804E091
:10C500000EF1010E83EA031384F807A084F8059066
:10C51000D8B284F87EE184F806C0030983F0F603FC
:10C5200043EA002383EAC0031BB283EA0310C3F388
:10C530000723C0B283EA101343EA002383EAC0034F
:10C540001BB283EA0C00C3F3072380EA0017FFB293
:10C5500083EA171040EA072080EAC70000B280EAA9
:10C560000A07C0F3072387EA0710C0B283EA101353
:10C5700043EA002383EAC0031F46238012F8010B1D
:10C5800078408A4280EA0010C0B24FEA101383EA72
:10C59000172343EA002383EAC00000B287B2278052
:10C5A000ECD180F018008B4A04F1220980EA0010D7
:10C5B0000692964602F5D37CC0B24FEA101A8AEA78
:10C5C000172A8AEA002A8AEAC00A0FFA8AFA1FFAA8
:10C5D0008AF35FFA8AFA1A0A238084F826A007925F
:10C5E00084F82720DEF800000EF1100E5EF80C1C17
:10C5F00067465EF8082C0CF1100C5EF8043CCE4542
:10C600000FC7EFD1744BDEF800001F4603F1260977
:10C61000CCF800009B469DF81C3084F8CCA184F82F
:10C62000CD311BF8011F28680DF044FFD945F8D122
:10C630000DF096FD694BDFF8ACC1B946B3F9043093
:10C640004FF47A7EB8F8082000218CFB037CDB17BE
:10C650000EFB02F2D8F80070C3EBAC03DDF814C097
:10C660000B97ADF842302123D8F804704FF01C0826
:10C670000D920E92FE220C974F460A90ADF83C1098
:10C68000ADF83E10ADF840106171E371A270DFF8B3
:10C6900040E184F80380BCE80F00AEE80F00C82238
:10C6A0000EF10C03A271A3F11C089CE807008EE8B0
:10C6B000070094F87E1181F06A02481C217182EA19
:10C6C000021284F87E01D1B20A0982F0D50242EA50
:10C6D000012282EAC10212B282EA0211C2F30722E7
:10C6E000C9B282EA111242EA012282EAC10212B2FE
:10C6F00082F0C801C2F3072281EA0110C0B282EAC7
:10C70000101141EA002181EAC00109B281F0210043
:10C71000C1F3072280EA0011C9B282EA111242EA8B
:10C72000012282EAC1021046228018F8011B414012
:10C73000984581EA0111C9B24FEA111282EA10222A
:10C7400042EA012282EAC10109B288B22080ECD11A
:10C7500081F06801DFF87CE004F1220881EA011130
:10C760000EF5D379C9B24FEA111B8BEA102B8BEA75
:10C77000012B8BEAC10B0FFA8BFB1FFA8BF35FFACD
:10C780008BFB1A0A238084F824B0079284F82520B2
:10C79000DEF800000EF1100E5EF80C1CCC465EF8C0
:10C7A000082C09F110095EF8043CC645ACE80F00FE
:10C7B000EED1BEF80030BA46DFF82C80A9F8003080
:10C7C0009DF81C3012E000BF143D01206E3D012099
:10C7D000E81E0120E21E012087200120183D0120D3
:10C7E0004C5F012067666666AB20012084F8CAB101
:10C7F00084F8CB311AF8011F28680DF05BFED04594
:10C80000F8D194F87E110023DFF848C64FF0310EBE
:10C8100081F0EB020C936371BB4682EA0212DCF8F2
:10C82000043021710131D2B20B9384F87E11C821FA
:10C83000130984F807E0DCF80070FE2083F0C503DC
:10C84000DFF814860A974FF00C0C43EA0223A8F590
:10C85000D077A07083EAC203A17184F803C01BB231
:10C8600083EA0312C3F30723D2B283EA121343EA23
:10C87000022383EAC2031BB283EA0102C3F3072344
:10C8800082EA0212D2B283EA121343EA022383EA53
:10C89000C203059A1BB283EA0E0EC3F307238EEA86
:10C8A0000E1E5FFA8EFE83EA1E1343EA0E2307CAAA
:10C8B00083EACE0387E807001BB294F808E0607AA9
:10C8C0008EEA030EC3F30723A17A8EEA0E1EE27AE4
:10C8D00094F80CC05FFA8EFE94F80D9094F80EA0B8
:10C8E00083EA1E1343EA0E2383EACE0394F80FE093
:10C8F0001BB25840C3F3072380EA0010C0B283EA9A
:10C90000101343EA002383EAC003207C1BB2594082
:10C91000C3F3072381EA0111C9B283EA111343EA81
:10C92000012383EAC103617C1BB25A40C3F307238E
:10C9300082EA0212D2B283EA121343EA022383EAA2
:10C94000C203A27C1BB28CEA030CC3F307238CEA5C
:10C950000C1C5FFA8CFC83EA1C1343EA0C2383EA69
:10C96000CC0394F813C01BB289EA0309C3F307236D
:10C9700089EA09195FFA89F983EA191343EA092355
:10C9800083EAC9031BB28AEA030AC3F307238AEACC
:10C990000A1A5FFA8AFA83EA1A1343EA0A2383EA35
:10C9A000CA031BB28EEA030EC3F307238EEA0E1EE0
:10C9B0005FFA8EFE83EA1E1343EA0E2383EACE0358
:10C9C0001BB25840C3F3072380EA0010C0B283EAC9
:10C9D000101343EA002383EAC0031BB25940C3F398
:10C9E000072381EA0111C9B283EA111343EA012343
:10C9F00083EAC1031BB25A40C3F3072382EA02123F
:10CA0000D2B283EA121343EA022383EAC2031BB2BF
:10CA10008CEA030CC3F307238CEA0C1C5FFA8CFC32
:10CA200083EA1C1343EA0C2383EACC031BB283F092
:10CA3000270EC3F307238EEA0E12D2B283EA121E28
:10CA40004EEA022E8EEAC20E0FFA8EFE1FFA8EF307
:10CA50005FFA8EFE23804FEA132C069F84F814E0C1
:10CA600084F815C038687968BA68FB68B7F8109020
:10CA70005F46A8E80F0028F8039B84F8BBC184F840
:10CA8000BAE117F8011F28680DF014FDB845F8D178
:10CA900094F87621002A40F07287E54F052094F83B
:10CAA0007E810DF1280CB7F902E0B7F9001088F08B
:10CAB0006A0362711E2206EE901ACEF1000183EA2B
:10CAC0000313E27107EE901AB7F90410FE22F8EE94
:10CAD000E66A07EE101AD9B2039BF8EEE77AA27065
:10CAE0001C221F680B09E270C82283F0D5030A9745
:10CAF000A271B8EEC77A43EA01239FEDCE6A4FF0E8
:10CB0000000E84F8760183EAC10366EE866A67EE5A
:10CB1000867ACDF838E01BB227EE067ACDF83CE0F5
:10CB200008F1010983EA0311C3F30723CDF840E0BC
:10CB3000C9B2CDED0B6ACDED0C7A83EA11138DED00
:10CB40000D7ADFF808E343EA012383EAC1031BB24D
:10CB50005A40C3F3072382EA0212D2B283EA1213C5
:10CB600043EA022383EAC2031BB283F01E07C3F326
:10CB7000072387EA071A5FFA8AFA83EA1A17BCE8DA
:10CB80000F0047EA0A27AEE80F0087EACA070EF14E
:10CB90000C039CE80700AEF1100C8EE8070084F847
:10CBA0000480278084F87E911CF8012B7A409C45F4
:10CBB00082EA0212D2B24FEA121181EA172141EA47
:10CBC000022181EAC20212B297B22780ECD182F030
:10CBD0002702DFF87CC204F1220882EA02120CF577
:10CBE000D379D2B24FEA121E8EEA172E8EEA022EA7
:10CBF0008EEAC20E0FFA8EFE1FFA8EF35FFA8EFED9
:10CC00004FEA132A238084F824E084F825A0DCF876
:10CC100000000CF1100C5CF80C1C4F465CF8082C62
:10CC200009F110095CF8043CC4450FC7EFD1824FED
:10CC3000BCF8003007F12408A9F8003084F8CAE1F4
:10CC400084F8CBA117F8011F28680DF033FCB84514
:10CC5000F8D194F877A1BAF1000F40F08A86774BAB
:10CC600005221B6884F877219B0641F11880744BDC
:10CC7000DFED746ADA891B8907EE902A07EE103A15
:10CC8000F8EEE77AB8EE477A67EEA67A94F87E7106
:10CC90000AAB6D4A4FF0640E87F022011846B2F9D4
:10CCA000062081EA01110593B2F5FA6F604BC9B213
:10CCB0008446A8BF4FF4FA62B3F904000B09DFF809
:10CCC0009C81B2F57A7F277183F0590307F1010740
:10CCD000B8BF4FF47A72CDED0B7A43EA012384F8A2
:10CCE0007E71A2F57A728DED0C7A83EAC1030EFB98
:10CCF00002F2DFF86CE11BB288FB0278D2178EFBE0
:10CD0000001E83EA0311C2EBA812C3F30723C9B2C2
:10CD10000027ADF83A204A2283EA11130A97E271FC
:10CD2000FE2243EA01230D97A270142283EAC10375
:10CD3000C821E27000221BB2A1716271C01783EAA0
:10CD40000102C3F30723C0EBAE00404F82EA021298
:10CD5000ADF83800D2B283EA121343EA022383EA21
:10CD6000C2031BB283F04A0EC3F307238EEA0E18E8
:10CD70005FFA88F883EA181EBCE80F004EEA082E16
:10CD8000DCF800C08EEAC80E0FC7A4F800E03A1D18
:10CD900047F810C917F8013B83EA0E03974283EA6C
:10CDA0000313DBB24FEA131181EA1E2141EA03218A
:10CDB00081EAC3031BB21FFA83FEA4F800E0E9D1A5
:10CDC00083F01403224A04F2C31983EA03131146C1
:10CDD000069204F2A712DBB20868174601F5D37C6D
:10CDE0001A09B846039782EA1E2E0F468EEA032ED2
:10CDF0008EEAC30E0FFA8EFE1FFA8EF35FFA8EFED6
:10CE00004FEA132B238084F81CE084F81DB0FB68E4
:10CE10004968BA68ACE80F00386979693B8B4746C6
:10CE2000ACE80300ACF8003084F8C3B11AE000BFEE
:10CE3000183D012088C3E43A87200120143D0120D9
:10CE40004C5F01200AD7233C247D0120E81E0120ED
:10CE5000E21E0120C837012088200120D34D621036
:10CE60006766666684F8C2E118F8011F28680DF04D
:10CE700021FBC145F8D1A54BA54A1B781278013B8F
:10CE8000039712F00101DBB214BF4FF0C00C4FF05A
:10CE9000400C172B03D89F4A134493F80CA09E4BC9
:10CEA0001B889F0701F043804CF0100C002213F404
:10CEB000027F18BF022213F0100F18BF062213F0D2
:10CEC000200F18BF1022002941F0DC804FF0030E24
:10CED00094F87E0103230A92002180F046028DF827
:10CEE000303000F10109207182EA0212C8208DF869
:10CEF0002EC04FF0090CD2B28DF82CA084F803C0DC
:10CF00004FF0FE0813098DF82FE08DF82D1083F0F7
:10CF10009203E171617143EA0223A071DFF8FCE141
:10CF200083EAC20384F87E9184F802801BB283EA0C
:10CF30000312C3F30723D2B283EA121343EA022394
:10CF400083EAC2031BB283EA0002C3F3072382EA27
:10CF50000212D2B283EA121343EA022383EAC20323
:10CF6000059A1BB283EA031CC3F307235FFA8CFC08
:10CF700083EA1C1343EA0C2307CA83EACC03AEE816
:10CF800003001BB2207A617A0EF5CC7C5840C3F3C3
:10CF9000072394F80A900EF5D47880EA00108EF8F2
:10CFA0000020E27AC0B294F80CE094F80DB083EA65
:10CFB0001013A77B94F810A043EA002383EAC00370
:10CFC000E07B1BB25940C3F3072381EA0111C9B2C8
:10CFD00083EA111343EA012383EAC1031BB289EAFE
:10CFE0000309C3F3072389EA09195FFA89F983EA78
:10CFF000191343EA092383EAC9031BB25A40C3F356
:10D00000072382EA0212D2B283EA121343EA02230E
:10D0100083EAC2031BB28EEA030EC3F307238EEA30
:10D020000E1E5FFA8EFE83EA1E1343EA0E2383EA86
:10D03000CE031BB28BEA030BC3F307238BEA0B1B54
:10D040005FFA8BFB83EA1B1343EA0B2383EACB03D0
:10D050001BB287EA0302C3F3072382EA0212D2B2A9
:10D0600083EA121343EA022383EAC2031BB2584045
:10D07000C3F3072380EA0010C0B283EA101343EA27
:10D08000002383EAC0031BB28AEA0302C3F3072327
:10D0900082EA0212D2B283EA121343EA022383EA3B
:10D0A000C2031BB283F03202C3F3072382EA0212E7
:10D0B000D2B283EA121343EA022383EAC2031BB209
:10D0C0009AB2DBB24FEA122E2280637484F812E027
:10D0D000069F38687968BA68B7F80C90039FACE887
:10D0E00007008CF802A0ACF8009084F8B8E184F84E
:10D0F000B73117F8011F28680DF0DCF9B845F8D1F1
:10D10000049BC4F86831FEF7A3BE00BFA84001200D
:10D1100083590120904404086C3D0120E81E012041
:10D12000DFF8288341201BF0E9FDDFF81CB3B8F9D4
:10D130000230DFF81CA38BFB0320DB17C3EBA0003E
:10D1400080B21BF0BFFDB8F900308BFB0320DB176A
:10D15000C3EBA00080B21BF0B5FDB8F904308BFB27
:10D160000320DB17C3EBA00080B21BF0ABFD9AF8E5
:10D17000001038680DF09EF994F860B11BF00108BA
:10D1800000F00784A44B1B689A0679D5A34B1B7843
:10D190009B0740F1DC86DFF8BC8298F81430042B42
:10D1A0008CBF4FF0030B4FF0020B47201BF0A6FD86
:10D1B000D8F800001BF04EFDD8F804001BF04AFD23
:10D1C000B8F80E30964A3868A2FB0323C3F347131E
:10D1D000194604930DF06EF99AF80010049B642030
:10D1E000B8F808204B4000FB02F08AF800301BF032
:10D1F00031FD98F8148038684BEA88085FFA88F89F
:10D2000041460DF057F99AF80030386888EA03086B
:10D2100041468AF800800DF04DF994F860B1BBF1F9
:10D22000000F2DD1DFF830824F201BF067FDD8F8BA
:10D2300000001BF00FFDD8F804001BF00BFD584652
:10D240001BF008FD012138680DF034F9734B9AF892
:10D2500000201B7882F00102386803F001088AF888
:10D26000002041460DF026F99AF80030386888EA27
:10D27000030319468AF800300DF01CF994F860B1E8
:10D280000BF10103674AC4F85C91DBB2A2FB031205
:10D29000D20802EB8202A3EB420384F86031FEF76E
:10D2A000B7BD614B614918680DF0CCF800232370BD
:10D2B000FEF725BE5E4F386800283EF498AD4FF06B
:10D2C0000009DFF898815B4C0DF0F0F8B9F1000F20
:10D2D00022D108B34FF001094FF0000A38680DF071
:10D2E000DDF883B27E2B00F01B8398F80120002A22
:10D2F0004AD194F84C11B1B11B2B84F84C2100F0A9
:10D30000E7820D2B46D0386888F801900DF0CEF8F2
:10D310000028E3D14FF0000948460AAA46491BF00D
:10D3200007FDFEF764BD7D2B00F0AF8494F850211B
:10D3300022B180F0200384F85011DBB294F84B2125
:10D34000062A10D8B4F84E11501C2244194484F80F
:10D350004B013868A4F84E1182F854310DF0A6F84C
:10D360000028BBD1D6E7B4F84E2188F801901344C9
:10D370009BB21A0A52FA83F3FF2BA4F84E3103D161
:10D380003868DFF8DC909FE738680DF08FF80028E8
:10D39000A4D1BFE73868A4F84E210DF087F8002823
:10D3A0009CD1B7E794F8BC32C4F8B862012B40F2C4
:10D3B000548494F8BD2221499818013201EB800170
:10D3C00002F001024F6A84F8BD22C7B11C4B12A8BB
:10D3D0004FF0A50E8022A3F112050B9315233146C1
:10D3E00040F8205D84F810E1059084F8112184F85C
:10D3F0001231B847002840F0B28394F8BC320133B0
:10D40000104A82FB0312A2EBE37202EB42029B1A68
:10D4100084F8BC32FEF72CBD143D01206E3D012086
:10D420001F85EB51CDCCCCCCC0930120E8920120DC
:10D430007C3D0120E01E01202A20012090440408A8
:10D44000052001205655555567666666183D012032
:10D45000003D01204C5F0120C83701200000012061
:10D4600034200120934A4FF47A71934B4FF0000E11
:10D47000D07A1B8801FB00F10398904A5FFA83FC85
:10D4800007681B0AD4F8380182F81EC0381AD3770F
:10D4900082F814C08842537582F802E082F804E0F2
:10D4A00080F0C88386494FF0F40E864801270B6848
:10D4B0004FF03009896880FB038CDB1780FB01800B
:10D4C000C917C3EBAC0382F81AE0C1EBA0017E4898
:10D4D00013774FF0750C1B12DFF808824FEA212AF0
:10D4E00000784FF0780E537782F8201082F821A050
:10D4F00098F81410754BD77682F8229082F823C0E2
:10D5000082F824E08207997640F19183D8F800C030
:10D510000529D8F804206E4F4FEAEC701146DFF869
:10D52000C89187FB0CE287FB01E74FEAE17EC0EB85
:10D53000A250684ACEEBA75E049109FB00C700EB3E
:10D54000800009FB0E1B0EEB8E0E07EB47070BEB63
:10D550004B0B4FEA47074FEA4B0B82FB079100EB5F
:10D5600080004FEAE77982FB0BA24FEAA1410590C8
:10D57000B8F808A04FEAA242B8F80E00A1EB0908DB
:10D5800006920EEB8E024146DFF860E14FEAEB793E
:10D5900007920EFB1171069A059F4FFA88F80AF55B
:10D5A000FA7A00EBC00008EB8708A2EB09074FEA04
:10D5B00080003A461FFA8AF90EFB17B7DFF830A150
:10D5C0004FFA82FE079A1FFA88F883F815900EEB3F
:10D5D000820E8AFB002A404A4FEAE0704FEADC7C68
:10D5E00083F80A8082FB012B3B4A05901FFA8EFECE
:10D5F00082FB07024FEAE77705984FEA1828C7EB46
:10D600006212364F83F809C04FEAE1713F88C0EBE0
:10D61000AA10DFF8E0C0C1EB6B11ADF81470C0F3D5
:10D62000072B049FBCF800C04FEAD77A83F80B8021
:10D630004FEA1E2883F80FE083F80EA04FEA222E4F
:10D640004FEA212A83F8108019734FEA19284FEA0C
:10D650001C2183F80DA05A7434BF4FF0320A4FF0EA
:10D66000330A83F812E083F81680D87183F808B083
:10D6700083F813C019759DF8142083F81BA01A773E
:10D68000C4F83461FEF747BB154B049318680CF0DF
:10D69000FDFE00283EF4CAAB049B012118680CF083
:10D6A000F1FE0222002387F8742088F80030FEF78C
:10D6B000BDBB00BF003A0120383B0120649301202C
:10D6C000D83A0120676666666E3D0120909301207E
:10D6D0006BCA5F6B83DE1B431F85EB51183801203B
:10D6E000B02E01204C5F0120806967FF40420F008F
:10D6F000D34D6210783D01205E2090473B680220A8
:10D700009847FF201AF0E2FF0378FF2B00F01C84FB
:10D7100090F901304FEAE379D8B25FFA89F91BF04A
:10D72000F9FE48461BF0F6FE3B685E2098473B68D2
:10D7300003209847FF201AF0C9FF0378FF2B00F061
:10D74000FF83B0F90830D8B2C3F307291BF0E2FE1B
:10D7500048461BF0DFFED24B1B78042B79D0DFF854
:10D7600078B34FF0640CB4F82E215E209BF80030A3
:10D77000DFF858A392FBF3FEBAF8001003FB1E2E4D
:10D780005A000CFB01311FFA8EFE3B684FEA0E195E
:10D79000A4F82EE1B1FBF2F11FFA89F9C1F30322DB
:10D7A00049EA01291FFA89F949EA020998473B68C1
:10D7B000062098475FFA89F01BF0ACFE4FEA19206B
:10D7C0001BF0A8FEB74AB4F82E31517A0133BAF8EB
:10D7D00000A00129A4F82E3100F0CF860AEB8A0AB6
:10D7E000537B1FFA8AFA002B40F056843B685E2078
:10D7F00098473B683A209847AB4BA3FB0A394FEA5E
:10D8000059191FFA89FB5FFA8BF01BF083FE4FEA70
:10D810001B201BF07FFE3B685E2098473B683B2047
:10D8200098476423A14803FB19A39BB2053380FBEF
:10D830000320DB17C3EBA000C0B21BF06BFE00207F
:10D840001BF068FEDFF8949299F80630002B40F048
:10D85000D883D8F800309A0600F13A8294F82C3137
:10D860003A68FEF745BADFF878924FF0240B9FED47
:10D87000908A5E20904758463B680BF1010B984711
:10D880008C4BF9EC016A5FFA8BFB1B8BF8EEE66AB6
:10D8900007EE103AB8EEC77AC6EE877A67EE887A56
:10D8A000FDEEE77ACDED037ABDF90CA05FFA8AF0C0
:10D8B0001BF030FECAF307201BF02CFEBBF1270F34
:10D8C00001D03A68D5E794F82C313A68FEF70CBAE3
:10D8D00038680CF0EBFD00287FF415AD386884F84B
:10D8E0004A9188F801900CF0E1FD00287FF4F6AC35
:10D8F00010E50CF035FC704A40F6B8331268A0EB26
:10D90000020A9A4500F2B681DFF8D8B19BF80430DC
:10D910003A2B00F03985002388F80030FEF786BAEC
:10D92000386884F84AA184F84BA184F84C9188F8AF
:10D9300001A00CF0BBFD00287FF4D0ACEAE494F821
:10D94000481194F849315D484A1C0133006884F855
:10D95000482184F849310CF0ADFDFEF73DBA013B9A
:10D9600084F86E31FEF742BC013984F86F11FEF77E
:10D9700067BD0AF1FF3A84F877A1FFF7C1BB013A0E
:10D9800084F87621FFF765B9013B84F87231FFF71F
:10D990007FB84B4B1B88D80515D4D90600F163839B
:10D9A0009A0600F1CD85580600F10586190700F1A9
:10D9B0000686DA0700F11C8613F0020F0CBF4FF049
:10D9C00004084FF00C083F4B3F4A1B78D27803F015
:10D9D00001030AB143F00203532048EA03081BF095
:10D9E0008DF93A4B1B8803EB830303EB8303980009
:10D9F00080B21BF067F900201BF064F9344B354A04
:10DA00001B883868C3EBC3135B0082FB0312D91772
:10DA10001344C1EB63235FFA83FB59460CF04AFDC4
:10DA20009AF80030002138688BEA03038AF8003046
:10DA30000CF040FD414638680CF03CFD9AF800308F
:10DA4000386888EA0303DBB219468AF800300CF024
:10DA500031FD94F860B1FFF7E2BB0024DFF8889055
:10DA60004FF0500BA24601E081F311883D5D601C30
:10DA7000294638441AF0EAFF002840F020816B1C48
:10DA80001C44EFF311838BF312883A6ED9B294429F
:10DA9000EADB00223A6681F31188FEF7A7BA00BFDD
:10DAA00076920120003A01201F85EB516766666679
:10DAB00000007A44203D01209C2D0120803D012062
:10DAC0006C3D0120835901207C920120383B0120CC
:10DAD00070920120030820803E3B0120043D01207C
:10DAE000543D0120842D0120799A0308C24B4FF048
:10DAF00000095E20DFF83483039384F82C911C68BE
:10DB000090473B681720984748461BF003FDBB4BE6
:10DB1000A3FB04239B0BA8FB03125209C2EB0212C6
:10DB2000A3EB8203D8B21BF0F5FC3B685E2098475C
:10DB30003B6818209847B24BA3FB04239B09A8FB22
:10DB400003125209C2EB0212A3EB8203D8B21BF0FC
:10DB5000E1FC48461BF0DEFC3A68FEF7CEB80A9EB0
:10DB60000021AE424FD941F2210015F8013B81EA74
:10DB70000323590013F4004F80EA010289B292B2E4
:10DB800008BF0A46530012F4004F80EA03029BB21A
:10DB900092B218BF1346590013F4004F80EA0102F5
:10DBA00089B292B208BF0A46530012F4004F80EACD
:10DBB00003029BB292B208BF1A46530012F4004F00
:10DBC00080EA03029BB292B208BF1A46530012F4D5
:10DBD000004F80EA03029BB292B208BF1A4653007C
:10DBE00012F4004F80EA03029BB292B208BF1A46B9
:10DBF000530012F4004F80EA03019BB289B208BFC0
:10DC00001946B542B1D105980EF09EFD7D4B0A9D97
:10DC100019467D48ED1A152DA8BF15252A4635F061
:10DC20001CFA7A4A94F8BC321570FFF7E8BB2D2233
:10DC3000DA7625E5764B03991B780968013BC4F831
:10DC40003811012B3FF62EAC102102239170137175
:10DC500028E41BF041FCFEF7BFB86E4A02EB8302DA
:10DC6000576AFFF7B2BB1BF027FC6B4F01233B70D9
:10DC7000FEF770B8694A0021B2F8623188F80010E6
:10DC80000133A2F86231FEF7D1B8386884F85091B8
:10DC90000CF00CFC00287FF421ABFFF73BBBDFED61
:10DCA000607AB0EE677AFEF7F1BF18469A469B4657
:10DCB0009C4606931F4698461946FEF7C9BA494640
:10DCC0003A201AF01DFE40EA0A0A5FFA8AFAD6E6FE
:10DCD000DFF85C9199F800309B0700F17382DFF860
:10DCE00054814FF0000AD3463B685E2098473B685A
:10DCF0000120984758461BF00DFC50461BF00AFCCB
:10DD00003B685E2098473B680920984700201BF03D
:10DD100001FC00201BF0FEFBB8F8123098F814B09C
:10DD2000B3F5967F0AD994F82C2102F00F02072A46
:10DD300004D842F20F7B9B4528BF9B463B685E2080
:10DD4000DFF8F4A098473B68052098479AF8083018
:10DD5000002B00F0F983ABF120039FED326AF6EE61
:10DD6000006A07EE903ABEEE007AF8EEE77A67EEC8
:10DD7000867AF5EEC07AF1EE10FA58BFB0EE667A08
:10DD800077EE877AFDEEE77ACDED037ABDF90CB038
:10DD90005FFA8BF01BF0BEFBCBF307201BF0BAFB46
:10DDA00099F80020002391070893099300F15E8100
:10DDB00094F83031012B00F05981BAF900300AA8EB
:10DDC000DFED196A07EE103ABAF9023007EE903A21
:10DDD000B8EEC77AF8EEE77A27EE267A67EEA67AEB
:10DDE000BDEEC77AFDEEE77A8DED0A7ACDED0B7ABE
:10DDF0001BF0B2FB32E500BF3CC2012073B2E74525
:10DE0000D34D6210F01F01202C2B0120412B01204B
:10DE1000769201209044040800000120E01E0120B9
:10DE200000000000E4380E3F0050C347898888880E
:10DE30006E3D01204C5F0120003A0120AE490AA846
:10DE4000AE4BA1F13F07AE4A00930991AD4B01F8EB
:10DE5000404CAD4908970EF05BFD089F2920EA2150
:10DE6000C8227B1C08933C70089B03F1010ECDF87F
:10DE700020E018700AA8089B03F1010ECDF820E0FD
:10DE80001970089B591C08911A7033F0DBFE00F1E1
:10DE900001080AA90898424635F0DFF808990122DE
:10DEA00012A801EB08031344089301F80840089BEB
:10DEB000991808911C70089B991808911C70089B70
:10DEC000991808911C70089B991808911C70089B60
:10DED000991808911C70089B991808911C70089B50
:10DEE000991808911C70089B991808911C70089B40
:10DEF000991808911C70089B991808911C70089B30
:10DF0000991808911C70089B991808911C70089B1F
:10DF1000991808911A7050F8283DDB1B3B702BF0C4
:10DF20008FFD7A4B2C70C3F8B062FDF795BF0122CC
:10DF3000FEF7BDBFC4F83C6187F800A0FDF70ABF3B
:10DF40004FF00009484601E44846FFF7E8BB4FF0B0
:10DF5000010BDFF8D081FFF728B90CF093FAFDF739
:10DF60000DBF654B12A90020DFF8B8810F46A3F161
:10DF70003D01A3F1400203F8400C47F8201D112198
:10DF80000B930223517038469370D8F80010059710
:10DF90000EF0A0FB3846D8F804100EF09BFBB8F842
:10DFA0000E305B49384603EBC3039B00053381FB0E
:10DFB0000321DB17C3EBA10189B20EF0A1FBB8F876
:10DFC0001030384603EB8303590089B20EF098FBFA
:10DFD000504B1B789B0740F1C982B8F8081001F537
:10DFE0007A7189B2059F38460EF08AFB0A9B98F831
:10DFF00014203846591C0A911A702BF021FDFDF7A8
:10E00000A6BF3B685E20DFF820A198473B68282028
:10E0100098473F4ADAF800304FEAE37B82FB03235C
:10E02000CBEBA30B5FFA8BF01BF074FACBF307205A
:10E030001BF070FA3B685E2098473B6804209847C5
:10E04000B9F80830002B40F08882DAF8083083F302
:10E0500010095FFA89F01BF05DFAC9F307201BF085
:10E0600059FAFFF7F6BB4FF03408ACE498E80C001F
:10E07000012108A8089284F8301109931BF06CFA6A
:10E08000FFF7ECBB244BDB78002B0CBF4FF0040EEA
:10E090004FF0050EFEF71CBF9BF800309AFBF3FA19
:10E0A000FFF7A4BB0123D8F800003B700CF0F6F991
:10E0B0000746D8F800000CF0F1F97F0602D080285E
:10E0C0007DF448AE8A2800F07E828E287DF442AE30
:10E0D00099F80030002B7DF458AE104F2D22104BD4
:10E0E00084F840213B603A68FDF738BE4FF0010AE2
:10E0F000DFF83080FEF7C0B9E8920120DF3D012053
:10E10000447604083C76040850760408E01E01209A
:10E11000676666666E3D01207C920120883D012085
:10E12000649301204C5F0120D83A0120DFF8489227
:10E1300008229FED878A0DF14808B9F9023007EEF1
:10E14000903A844BF8EEE77A03F8401C03F83F2C32
:10E15000A3F13D011E220B9367EE887A48F8201D3B
:10E1600003F83E2C4046FDEEE77ACDED037ABDF88C
:10E170000C100EF0C5FAB9F90030404607EE903A9F
:10E18000F8EEE77A67EE887AFDEEE77ACDED037A6E
:10E19000BDF80C100EF0B4FAB9F90430404607EEA1
:10E1A000903AF8EEE77A67EE887AFDEEE77ACDED01
:10E1B000037ABDF80C100EF0A3FA40462BF040FC99
:10E1C000FDF7BCBEDFF8B4815E203B684FF4F36A14
:10E1D00098473B681120DFF8A8B19847B8F80E308F
:10E1E0000AFB03F38BFB032BDB17C3EB6B3B5FFAE1
:10E1F0008BF01BF08FF9CBF307201BF08BF93B68FA
:10E200005E2098473B6819209847B8F80E30524A6C
:10E2100064210AFB03F382FB03E0DB17C3EB60130B
:10E2200082FB0320DA17C2EB601201FB1233D8B273
:10E230001BF070F900201BF06DF999F80030B8F868
:10E2400008A098077FF54DAD5FFA8AFB4FEA1A2ABE
:10E250004AE5424A00203F4B21211268A3F14009C0
:10E260000B9303F8400CD30089F8021040F195811C
:10E270004FF003083A493B4B1B88580500F1798160
:10E28000DA0700F1B181980702D54FF0030836494B
:10E29000DFF8F0A04246504634F0DFFE08EB0A03F8
:10E2A000AAF102020021013312A808F80A109A1AF2
:10E2B00040F8203D89F801202BF0C2FBFDF744BE59
:10E2C000244B4FF000090DF148084FF00A0C4FF0B5
:10E2D000080EA3F13D00254903F8409CDFF8949017
:10E2E00048F8200D404603F83FCC03F83EEC09887F
:10E2F0000B930EF005FAD9F8003040461C49DA17A6
:10E3000081FB0313C2EBA30399B20EF0F9F9D9F81C
:10E3100008902DF04DFE0A9B4FEA194103F1010EC2
:10E320004FEA1922CDF828E019700A9B591C0A916E
:10E330001A700A9B5A1C0A9283F800900A9B5A1C76
:10E340000A92187040462BF07BFBFDF7FABD00BF28
:10E3500058A08B41E89201201F85EB51F43E01202B
:10E36000287604086C3D012038760408383B0120EB
:10E3700067666666D83A0120183D01204C5F01208F
:10E3800089B5F814AB9201209BF80210584615F09D
:10E3900003F900287FF4BFAAA04AA14F1288A14B1D
:10E3A000A149FA61A14C1A6804919B68B4F8621102
:10E3B000FA629D4AF863C7F86CA01068FB64F965BF
:10E3C000F9F778FE824600287DF42BAD964B49463E
:10E3D00018680CF057F894F8643104229BF8031085
:10E3E000642B069187F8742040F03A8194F86531E7
:10E3F000072B8F4B08BF84F865A194F865B107938C
:10E4000007EB0B19D9F804A0504633F01BFCD9F8E0
:10E4100008305FFA80F91846059333F013FC514633
:10E420005FFA80FA079B2BF00F020BF00F0B09EB42
:10E430000A0E0AEBC9009A724A460EF1080E98734A
:10E4400083F80DB003F10F0083F807E034F005FE08
:10E45000784B09F1090052460599184434F0FDFD46
:10E46000079BDA7902F1010AFAB102F1FF3903F1EF
:10E47000070E0022DFF8E4C15FFA89F909F1080903
:10E4800099441EF8011B5140F1454FEA81024FEAC1
:10E49000D10082EA410200F0180082EA01024CFA3F
:10E4A00000F182EA0102D2B2EBD10593614B0698EA
:10E4B0000AF8032034F076FD94F865210021059BCD
:10E4C000013284F8641184F865219A7899465AB12A
:10E4D000049B19F80510013518680BF0EBFF99F84B
:10E4E0000230EDB2AB42F3D894F864310322013329
:10E4F00087F8742088F8002084F86431049BFFF7C3
:10E50000C5B8464B4C4A1B88927903EB830303EB57
:10E5100083034FEA83081FFA88F8002A00F03D8140
:10E52000404B1B680FFA83F92DF042FD40B2FDF716
:10E530009ABD08468A468B468C460691FDF788BEF2
:10E540004FF02408FFF73FBA5FFA8BF01AF0E2FFB2
:10E550004FEA1B201AF0DEFF22E42DF029FD1AF00D
:10E56000D9FF00201AF0D6FFFFF773B94FF47A7184
:10E5700038E54FF0030831498AE63B685E2098474A
:10E580003B68392098475FFA8AF01AF0C3FF4FEAD8
:10E590001A201AF0BFFFFFF755B9294B294A1B680B
:10E5A000294903F48003834216BF11464FF0040843
:10E5B0004FF003085FE64FF01008FFF704BA4FF082
:10E5C0002008FFF700BA214B1B6899067DF5C2AB06
:10E5D00099F80030002B7DF4D8AB1D4F2D221D4B38
:10E5E00084F840213B607EE54FF004081A494FE66D
:10E5F0004FF00808FFF7E7B90846FDF729BE0846BF
:10E600008A468B468C4606910F46FDF721BE054B88
:10E6100080466420B3F90090FDF725BD383B01200A
:10E6200000000120D83A0120B02E0120E01E012078
:10E63000887101208E710120043D01202C76040890
:10E64000E05601202876040820760408143D0120B5
:10E65000883D012090930120307604080007090EC0
:10E6600097F8759019F00F0F03D109F101095FFABE
:10E6700089F9B9F1070F4C4B4FF0000228BF4FF05A
:10E68000010903F10D0B9A724FEA091A07EB0A020E
:10E690005FFA8AF1107C454A0591115C059A0129BF
:10E6A0000BF1010C40EA020007EB0A028BF80000B4
:10E6B000D2680DD9881E6146C0B200F1020EDE4458
:10E6C00001F8012B71454FEA1222F9D1013084443F
:10E6D000BA4409F1010922F060020CF1010B9AF829
:10E6E00011105FFA89F90A43B9F1080F8CF800207C
:10E6F00056D005984FEA091A2D4A103007EB0A0147
:10E70000ABEB0202C0B20590087C2849095C02EB21
:10E71000010EBEF1130FC1DDD2B2DFF89CC0911D16
:10E72000C9B241F0400001F1010AD871E1B10532EE
:10E730000CF1010E0021D2B2083203EB020B1EF8DD
:10E74000010B4840F3454FEA80014FEAD00281EACD
:10E75000400102F0180281EA0001164840FA02F274
:10E7600081EA0201C9B2EAD106980AF80C100593B1
:10E7700087F8759034F016FC059BA6E608468A4695
:10E78000FDF766BD08468A468B46FDF761BD084623
:10E790008A468B468C46FDF75BBD4FF0FF33C1E6E2
:10E7A000034AABEB0202B7E78871012090440408EA
:10E7B000957101200007090E8E71012044F6206337
:10E7C0001A465C4B2DE9F04F82182DED088B97B05F
:10E7D00011461C780C92584A08901160002C00F0E9
:10E7E0004287564A08991268914240F28A80544AF8
:10E7F000013C544916681C70534B06F4805607922E
:10E800000593524B06910993002E40F08880504B9F
:10E810001B78022B01F08381042B01F0EE81012B88
:10E8200001F0A2814B4B089A9A42099B9B7800F217
:10E830001986002B40F01A86474B0893079B1E68E9
:10E8400016F4805740F0D486DFF83891059BB3F971
:10E850000610069B5D8BA942B4BF00250125DFF899
:10E860002081D8F8003013F0805300F08D80089A92
:10E87000127812F0010200F08E800698408C8842D7
:10E8800041F32983002D40F08D80344C94F88C1096
:10E89000002940F0878032480024324900680C602B
:10E8A00090F82D004C608C602F4900287BD10870B7
:10E8B000002A7CD0F1067AD52C4A1278D20676D47A
:10E8C000002F74D1002B72D1740270D4284B1B78A6
:10E8D000002B02F0A183274B9B78002D42F0C383CD
:10E8E0003BB1254A254B12681B689B1A002BC2F2CC
:10E8F000A3831020194C32F0BDF8012384F88D3029
:10E9000055E00F4B0F4A1E6807930F4B06F48056D5
:10E91000069205930D4B0993002E3FF478AF00212A
:10E9200017480EF0E1FB00287FF471AF30F050FA89
:10E930006DE700BFA82D0120202C0120A42D01206F
:10E94000E0560120384D0120247D01207C920120D9
:10E95000F62C0120404B4C0083590120A4210120BA
:10E96000703D0120083F0120342401206E3D01202C
:10E97000DC00012090A301203CC20120F4B701205B
:10E98000F43E0120602E012070023FF570AF089A1E
:10E99000127802F00102574C002184F88C10002DEF
:10E9A0003FF479AF544901200870002A82D1534BBB
:10E9B0001978002940F0C283069A059C568BB4F959
:10E9C00000702346908BBE42B4BF80220022B3F970
:10E9D00004E0B4F9024042F0400CB842CCBF6346B8
:10E9E0001346059A9B08B2F9067043F08002A642CE
:10E9F000B8BF134643F04002A042D8BF1A463D4C70
:10EA0000920894F88EC042F080037645B8BF1A464B
:10EA100042F040037045D8BF13469B0843F0800284
:10EA2000B742C8BF134643F040028742ACBF184606
:10EA30001046844501F0D4840B46A4F8901084F865
:10EA400092102F4A84F88E001678002E01F0B083C1
:10EA50005F2801F01F846F2801F06584089B1B78F4
:10EA6000DB0700F16B8394F89210002940F0668375
:10EA7000B4F99030322B40F3618394F88E2001205A
:10EA8000572A84F8920001F0DD87079B1B685D0719
:10EA900041F102835A2A41F0FF8294F89430002B0E
:10EAA00042F0B18294F8963083F0010384F89630F6
:10EAB000002B42F0E3820C20124E31F0DBFF079B6B
:10EAC000114A1B680A9203F00403002B40F04083B4
:10EAD0000E4B0DF1500B0B9640F6330A1D460D936D
:10EAE0000023192740F28334059ECBF80430149399
:10EAF00011E000BFA421012034240120433901206A
:10EB0000DC0001206C3D0120743D0120102E01200D
:10EB100004354D4522D0A978EB7817FB0140994286
:10EB2000F6D295F801E017FB03410EF1040336F924
:10EB300013305345A8BF5346B3F5617FB8BF4FF4B8
:10EB400061739842E4DA9942E2DB29782729DFD819
:10EB5000043558460EF0B8FA4D45DCD1664B0B9E95
:10EB60001B789BE8030088E80300002B40F0A08797
:10EB7000624B1B78002B00F01B87012160480EF0D0
:10EB8000B3FA002840F02683099BDB78002B40F085
:10EB90002183DFF8889133881CB224F00104A7B2E6
:10EBA000BB42378001F04180564C4FF002084FF0D5
:10EBB000140B4FF0FF0A0E2084F8008084F801B097
:10EBC00084F802A031F056FF41464D4837880EF0D8
:10EBD0008BFA002841F02A8327F002039BB2BB4244
:10EBE00033800AD0474B02201421FF2218700E20D8
:10EBF00059709A7031F03EFF3788434BBC07434A47
:10EC00001978506808BF81F002010C930B92C1F390
:10EC100040010BF009FE242139480EF065FA30B9A5
:10EC2000089A1378590702D523F004031370D9F812
:10EC3000003013F00A0F1DD0052131480EF054FAB0
:10EC4000002801F018813488620741F1C68206214C
:10EC50002B480EF049FA002801F0FA80630641F1D2
:10EC6000B482072126480EF03FFA002841F02480A4
:10EC7000D9F800309F0600F14087B6F80080244F95
:10EC80000C211F480EF030FA002800F0C08248F432
:10EC900080734345338009D01A4B02201421FF2290
:10ECA00018700E2059709A7031F0E4FE194B1B78E1
:10ECB0000E2B00F0B882082B00F0B582079B1C6871
:10ECC000600568D5144B1B79002B00F06582142178
:10ECD0000B480EF009FA002840F063822AF00EFF7C
:10ECE000012031F009FE00240246DFF834B04FF075
:10ECF000CC0AA9460E9616E0AC7E0120C73701204B
:10ED0000F43E0120E428012044C2012048C2012031
:10ED1000403B0120A8400120003A0120143D012081
:10ED20001C7A0120DCB20AFB04F8631C7AB3022CC3
:10ED30002DD85BF80850002DF4D1032192F9020080
:10ED4000E34E2B4601910121029592F803E02A46F9
:10ED500056F82E60009631F019FA0346CC2204EBE7
:10ED6000440029460F9353B100EB001001340BEB24
:10ED7000800035F006FB0F9BE4B24BF8083021F021
:10ED800027FE02460AFB04F8631C002ACFD14D4639
:10ED90000E9E079B1C68089B93F800A0CD4B1AF0B1
:10EDA000010A00F0968201221A700A9B4FF0010EB0
:10EDB00005991868B1F906104289C74B914283F84A
:10EDC00000E080F26C824FF07E52C44B1A60C44A5D
:10EDD000069B0598B3F81880B0F900E092F904306A
:10EDE0001078002BAEEB080392F801C014BF01228B
:10EDF0004FF0FF32002BB8BF5B42B3F5FA7FA8BFDC
:10EE00004FF4FA73984280F247821B1A07EE903A49
:10EE1000F8EEE77AC645C7ED007A03DAF1EE677AD5
:10EE2000C7ED007A059BB3F902E0AEEB0803002BB7
:10EE3000B8BF5B42B3F5FA7FA8BF4FF4FA739842AC
:10EE400080F227821B1A07EE903AF8EEE77AF04537
:10EE5000C7ED017A03DDF1EE677AC7ED017A059B14
:10EE6000B3F90400A0EB0803002BB8BF5B42B3F575
:10EE7000FA7FA8BF4FF4FA736345CCBFA3EB0C0332
:10EE80000023404502FB03F307EE903AF8EEE77AE1
:10EE9000C7ED027A03DAF1EE677AC7ED027A14F46D
:10EEA000805400F0D381B1F5FA6F8E4BA8BF4FF4B8
:10EEB000FA611A78B1F57A7FB8BF4FF47A71A1F58B
:10EEC0007A71002A40F0DB818748CA17DFF830E208
:10EED0006FF0630380FB019CC2EB6C1202F1010C2A
:10EEE00003FB02133EF912203EF91C10891A03FBA2
:10EEF00001F380FB0310DB17C3EB60131A4412B25B
:10EF000007EE902AB8EEE78A87ED038A002C40F0DE
:10EF1000E58433885A0640F1FA807449B6EE000A57
:10EF2000734A13F0030391ED011AD2ED014AD2EDB9
:10EF3000025A91ED035A74EEE57A92ED038A31EEAE
:10EF4000457AD1ED028AD2ED001A71EE05AAD1ED13
:10EF5000000A34EEA5AA27EE274A97ED012A70EEA3
:10EF6000A89A644A31EEC89A97ED003AB0EE446A26
:10EF700008BFD7ED023A71EE887A18BFDFED5E3A2E
:10EF800070EEE86A5D49A9EE896A30EE81BA66EEF4
:10EF9000A76AF0EE447A70EEC10AB0EE667ADAEE55
:10EFA0008A7AAAEE8A6AA9EE897A31EEA41A71EEFB
:10EFB000E41A72EE022AF0EE674A36EE266AAAEEEC
:10EFC000CA7AE9EEC94A20EE466A77EEE67AABEEF7
:10EFD000016A37EE447A74EEA66A35EE684A27EE87
:10EFE000007A35EE285AB0EE461A66EE806A35EEA3
:10EFF000C86AE9EE897A82ED011AE5EE216AA4EE8B
:10F00000067A21EE015A75EE885A33EE038AB0EE85
:10F01000456A67EE807AC2ED036AF1EE668A82ED98
:10F02000007A97EE076AE0EEA57AA7EE075AB1EEEE
:10F03000470A61EE264AF0EE465AB1EE679AC2EDF3
:10F04000027A61EE270AE8EEA65A27EEA64AA9EE52
:10F05000275AF0EE609AF0EE441AA9EE276AE7EE1E
:10F06000269AE7EEA75AA8EEA65AE0EE011AF0EEAD
:10F07000648AE0EE260AA7EE014AE7EE278A25EE2B
:10F08000827A62EEA95AA6EEA66AE0EE274A21EE3F
:10F09000822AF0EE656AA8EE207AA3EE282AE3EE33
:10F0A000056A66EE237A34EE044A74EEA44AB0EEA2
:10F0B000006AA4EE237AE4EEA36AE2EE067A87ED14
:10F0C000017A81ED377AC1ED366AC7ED006A19E041
:10F0D000446E0408845901206C240120E42301209B
:10F0E00068A3012094A401201F85EB51781C012006
:10F0F00094000120CC00012000000000A421012088
:10F1000078350120C1ED387A0BB9C7ED027ABAF132
:10F11000000F40F0668116F039FD17B0BDEC088B8A
:10F12000BDE8F08FB54A1278960741F19F84B44A42
:10F13000127D042A41F29A8417F0AEFD079BB14A72
:10F140001B68B14E03F004030A92002B3FF4C0ACDD
:10F15000AE4C94F896305BB1089B1B78DB0707D563
:10F16000059BB3F90620069B5B8B9A4201F3018253
:10F170001121A7480DF0B8FF002800F09A8694F8F6
:10F180009A302BB994F8943013B93223A4F89830FC
:10F19000012384F89A309BE4089B1B78D9077FF5FC
:10F1A0009DAD4FF40F7028F057FC00283FF4F1ADEF
:10F1B0002DF08EFA4FF40F7028F0F0FB00283FF48A
:10F1C000E8AD2DF085FA4FF40F7028F0E7FB00282A
:10F1D000EED1DEE5DFF88492D9F8003099077FF5AB
:10F1E000DAAC3788FA073FF5F7AC47F001039F42E6
:10F1F00033803FF4F1AC874B02201421FF221870BA
:10F200000E2059709A7031F035FC3788E4E428F408
:10F2100080739BB2434533807FF43EAD7E4B1B78B9
:10F220000E2B7FF448AD328822F040039BB29A4205
:10F2300033803FF443AD774B02201421FF22187036
:10F240000E2059709A7031F015FC37E5069B5A8BE9
:10F250009142C0F2E784B1F5FA6FD4BFC2EB01016D
:10F26000C2F5FA614FF47A7303FB01F16B4BC2F5FF
:10F27000FA621878B1FBF2F100283FF425AE5B7812
:10F28000674A01FB03F182FB0123C917C1EB63113C
:10F290001AE6DFED647ADAE5DFED627ABAE5B1F518
:10F2A000FA6F80F2B8848B1A007AC2F5FA6203FB17
:10F2B00000F393FBF2F3C3F1640307EE903AF8EE28
:10F2C000E77A9FED597A594B67EE877AC3ED007A5A
:10F2D0007DE51B780793002B7FF467AD544A1268D5
:10F2E000002A3FF462AD534ADFF874B1114612F8B8
:10F2F000030CA2F1030908929BF8008016F0C6F9EE
:10F30000089A002800F00286079BB8F1000F41F030
:10F31000AF8509F1080199F8050016F0B7F9002842
:10F3200041F0DF85444999F80A0016F0AFF900284A
:10F3300000F00186B8F1020F41F0CF853F4999F8FE
:10F340000F0016F0A3F9002841F0C3853C4999F855
:10F35000140016F09BF9002800F00186B8F1040FA4
:10F3600041F0B385374999F8190016F08FF9002854
:10F3700041F0A785344999F81E0016F087F9002856
:10F3800000F00186B8F1060F41F097852F4999F8F2
:10F39000230016F07BF9002841F08B852C4999F861
:10F3A000280016F073F9002800F00186B8F1080F64
:10F3B00041F0A685274999F82D0016F067F9002835
:10F3C0003FF4F3AC0922134602EB82028BF80030C3
:10F3D000214B914499F8011099F8022019705A7044
:10F3E000E3E40C9B19780B9B01F0010118680BF00A
:10F3F0001BFA17B0BDEC088BBDE8F08F6E3D012005
:10F400004C5F0120743D01206C3D0120A4210120AE
:10F41000F43E0120E4280120A840012094A401200A
:10F420001F85EB51000000000AD7233CE423012094
:10F4300088590120AA280120B4280120B9280120D8
:10F44000BE280120C3280120C8280120CD28012082
:10F45000D2280120D72801208C590120143D0120F9
:10F460007600012013B90123099A93709F4B1B204A
:10F470001D460893099B93F8214016F02FF92D782B
:10F480008146012C05F0010800F0198705F00205FE
:10F49000099A974E92F820309346DFF86CA2954F68
:10F4A000CDF82890052B00F29780DFE803F0857BEC
:10F4B00003C5C8B9012C00F0F384B8F1000F00F0C7
:10F4C000C180069B00213588B3F918000A46DFF891
:10F4D0003C9260F30F0160F30F0265F31F41059D3D
:10F4E00060F31F42D9F800006960DBF814102A604D
:10F4F000814280F0E786032547F230510322CBF8A2
:10F500001C108BF82020022009F066FC2FF060FC14
:10F51000D9F80000DBF81C20042102448BF82010ED
:10F52000CBF81820012C40F0BE87D9F80020DBF87A
:10F530001810914250D29AF8000018B916F0CEF87F
:10F54000002849D13A6822F002023A60D9F8001046
:10F5500064207388002200FB03134FF480608BF853
:10F560002020CBF810308BF8032009F005FC9BF825
:10F57000203097E716F0B8F8012801F04D820A9B79
:10F5800013B1B379002B4ED1012C25D0DFF87C913B
:10F59000DBF81010D9F800209142C0F079870123E0
:10F5A0008BF82030012C3BD0F379012B4FD016F093
:10F5B0002BF89BF8203075E7B8F1000FDAD1DDF8B1
:10F5C00028904FF48060B9F1000F00F0418309F0FA
:10F5D000EBFB0023099A1361002D3FF42FA9284665
:10F5E00031F048FA079B1E6816F480573FF42CA9A7
:10F5F0001D2141480DF078FD00287FF425A93F4BDF
:10F6000003F1500903E00433994500F001871A78AB
:10F61000262AF8D19978DA789142F4D2FFF716B910
:10F62000DFF8E89092E715F0EFFF03224FF47A73CA
:10F630008BF82020CBF81C30DFF8D09063E7DFF8A0
:10F64000CC906FE7DFF8C490D9F8002054E715F0AC
:10F65000DBFF032240F6B833DFF8B0908BF82020B0
:10F66000CBF81C304FE7264F3B78002B56D0DFF805
:10F67000A0804FF47A79DFF89CB0224B4546DFF842
:10F6800098A05E46069326E0069A115D9847032CE3
:10F6900002B219DC0246B8B138F824E040F6CA01DB
:10F6A0006B88A0EB0E02A3EB0E0040F2EE2309FBE9
:10F6B00002F292FBF0F202F57A728A42A8BF0A4681
:10F6C0009A42B8BF1A4612B201343B782AF8022F88
:10F6D00004359C4224DA072C3046DBF80430E1B2D2
:10F6E000D2DD3046984702B2EEE700BF83590120D1
:10F6F00070350120683D0120F43E0120102E0120CC
:10F70000D82E0120384D0120DC0001203CC2012010
:10F71000EC2E0120543E0120A2210120914A0692A4
:10F72000914A42F20106914908980791A2FB002BE9
:10F730000A6816404FEA9B1B00F0B7838C488D493E
:10F7400090F800E08C4C08788C4984F800E0087050
:10F75000BEF1000F04D0894991F800E08EF0010E4F
:10F76000874C0F2084F82400002B00F03E85854B49
:10F7700012F4805F844904F1280212931B781090E0
:10F780001846069B94F825A0A1FB00C19D8C0F9004
:10F790004FF0000306984FEA5101CDF824E0B64639
:10F7A000B0F818C001EB41010698CDF844C0B0F89C
:10F7B00026C01198CDF838C08446744808BFAC46BE
:10F7C000CDF828A00590A2460F98CDF84CC00BF5B7
:10F7D000967C411A97F80080CDF82CC0C9B2DFF8AA
:10F7E000CCC16A4C0D910999002900F07B843AF94B
:10F7F000130059001FFA80F9A94503D30E9EB145A5
:10F8000040F2B0845CF82300834580F07384605E2E
:10F81000BEF1000F40F08784013360520632434549
:10F82000E1DB109A54465A4B0F2A84F82420DDF865
:10F8300028A00CBF0122002284F825A01A7000F035
:10F84000DB8401234B494D4A04200B70137009F0EF
:10F85000C3FADFF854B14F4BDBF800101C46099394
:10F860009B686268CB1AE160934202D9002384F856
:10F870002130079B3C781E68002C01F0EC81069A31
:10F8800016F48056444DB2F824E0178B40F0E08423
:10F8900032463E4928460DE0437803EB830303EBF1
:10F8A000830303F2EE239BB20132023021F8023BC4
:10F8B000A2420DD015F81230002B00F05884022B14
:10F8C000EAD00B880132023021F8023BA242F1D18A
:10F8D000129A137801331370FEF796BF1D212F483B
:10F8E0000DF002FC002840F033850D9B03E004334B
:10F8F000AB423FF40EAB19782629F8D19878DA7824
:10F900009042F4D2099BDB78002B7FF402AB2348B2
:10F910000DF0EAFBDFED227A002801F0A48138EE39
:10F92000678AC8F57A73104901201AB21D4BFDEEA3
:10F93000C87ACDED057A1870BDF914301B0381FB30
:10F940000301DB17C3EBA11302FB03F343F30F33F4
:10F95000434407EE903AF8EEE77AC7ED037AFFF7F3
:10F96000D8BA00BF384D0120D34D6210E0560120B7
:10F97000FC2B0120840001203D9201208500012004
:10F98000A4210120C52D0120ABAAAAAA247D012013
:10F99000963E01207C920120202F0120F43E012080
:10F9A00000007A44602401203CC20120C82D0120BF
:10F9B000DFF8F8B29846DFF8F8A24FF001090BF132
:10F9C0005A07A54C59461BF8010C15F05FFEF8B11B
:10F9D0009BF804209BF8023002EB420E9BF80300D8
:10F9E000013B09FA02F204EB8E0E03EB4303DEF84F
:10F9F000A01053448B420BD094F8CC108EF89C008E
:10FA000021EA0202CEF8A030CEF8A48084F8CC20FF
:10FA10000BF1060BBB45D5D1904B4FF0000A904A35
:10FA20001B78DFF890920B930A9BA9F19C0BD2F8FC
:10FA300000801B680C93D9F8043083B31C7874B32E
:10FA4000D9F80820A8EB0202002A0CDB01219BF860
:10FA5000CC2008F5FA7001FA0AF1C9F8080022EA88
:10FA600001028BF8CC200B9ACAB199F80020597882
:10FA70000432D2B2002940F0348206990598098BED
:10FA800030F9122001F1C800824240F3D3849BF880
:10FA9000CC109A7841FA0AF3DF0740F178850AF131
:10FAA000010A09F10C09BAF1040FC4D1FFF765B8D6
:10FAB0006C4B03E004339D423FF45AA81978232984
:10FAC000F8D19878DA789042F4D267480DF00CFBC0
:10FAD00000283FF44DA8654B1B6813F4003341F038
:10FAE000BF811846624AD15C0C33142900F0E587C7
:10FAF00001301828F7D1FFF73BB85E4B1B789C0705
:10FB000004D55D4C237D042B00F2D884B6F8008028
:10FB100018F0300F40F05982584FFFF7B1B8069AED
:10FB20000599537DD27D013B31F913301AB140F66E
:10FB3000B832D21A13B2A3F57A739FED517A40F21C
:10FB4000FF31504A07EE903AF8EEE77A67EE877A8F
:10FB5000FCEEE77ACDED0A7ABDF828308B4228BF5B
:10FB60000B461380FEF75EBE3B4C089AD4F88830F3
:10FB7000D31A002BFEF656AE434B40F2FF320698E6
:10FB8000597C424BDFED426A33F811300C999BB23D
:10FB90009FED406AC4F88810817D07EE903A07EE29
:10FBA000101AF8EEE77AC17DB8EEC77A67EE867A6A
:10FBB00027EE267AC7EE876AFCEEE67ACDED0A7A62
:10FBC000BDF82830934228BF134609B1D31A9BB21F
:10FBD000314D324E2878324C36F81070411C226874
:10FBE00001F00F0126F81030D21B29701344254A6A
:10FBF000190923601180FEF715BE0AF0B1FA294BEE
:10FC0000294A1B68C31A93427EF70CAE1D4B002293
:10FC10001A80FEF707BE037AC3F1640307EE903A39
:10FC2000FFF74DBB2146FFF721BB02210E480DF027
:10FC30005BFA00283EF4D0AF3480BB073EF5DDAF61
:10FC400047F00203BB4233807EF4CCAFFEF7D5BF52
:10FC500009F092F8BDE400BFA42101203D920120EB
:10FC60003CC20120102E0120F43E0120B4270120C7
:10FC7000184B04086E3D01204C5F0120403B0120E1
:10FC80006F12833F70920120AC5B0120CC5B01209E
:10FC90000000C84200008044F72C0120FC2C012009
:10FCA000F82C0120A822012060E31600C1270120C2
:10FCB000C444040840220120D64AB2F90030002B87
:10FCC000B8BF5B42B3F5E17FBEF6D2AFB2F9023006
:10FCD000002BB8BF5B42B3F5E17FBEF6C9AFCE4B98
:10FCE000B7EE007A93ED096AD3ED076AD3ED037A94
:10FCF00076EE866A93ED056A77EE867A76EEA66AE8
:10FD000077EEA77A37EE666AF0EEE75AB0EEC66A8B
:10FD100086FE255AB5EE405AF1EE10FA40F0008406
:10FD20009FEDBE7AB4EEE56AF1EE10FA03D59FEDD1
:10FD3000BC6A36EE477AB7EE006AF4EEC66AF1EEB8
:10FD400010FA00F38287F5EEC07ADFEDB57AF6EEB1
:10FD5000006AF1EE10FA48BFB1EE477A27EE667AF4
:10FD600077EE276ABDEEE66A16EE103A2033402B96
:10FD700040F2BA86DFEDAB6AAB4ADFEDAA7AC2ED9C
:10FD8000006AFDEEC76AC2ED017AC2ED027A16EE94
:10FD9000903A2033402B47D8DFEDA47AB4EEE77ACF
:10FDA000F1EE10FA41F32B819FEDA16ADFEDA16A1C
:10FDB000B4EEE67A77EE467AF1EE10FAB0EE677AB4
:10FDC000F6DC9FED9D7AF4EEC77AF1EE10FA41F180
:10FDD00012819FED976ADFED996AF4EEE67A37EECD
:10FDE000867AF1EE10FAF0EE477AF6D4DFED8C7AEF
:10FDF000B4EEE77AF1EE10FA40F3F586DFED8B7A98
:10FE000037EEC77A27EE076ADFED8D5ADFED8D6A90
:10FE1000DFED8D7AE6EE256A67EE065AE6EE267A83
:10FE2000A5EEA77AF0EE477A884BC2ED037A1B68FD
:10FE300013F4003340F0B9861846854AD15C0C3380
:10FE40000A2900F0908501301828F7D1FEF710BF7D
:10FE500024F040039BB2A34233803EF402AF7D4BBB
:10FE600002201421FF2218700E2059709A7030F071
:10FE700001FEFEF7F6BE338823F00404A4B2A342C9
:10FE800034803EF4E4AE734B02201421FF2218703C
:10FE90000E2059709A7030F0EDFD3488FEF7D7BE11
:10FEA00005238BF82030FFF708BB6B4991F800E081
:10FEB0004EE494F89430002B3EF40AAE089B1B7875
:10FEC00013F001037EF404AE012284F8943084F828
:10FED0009520FEF7FDBD614C012184F88C10FEF7E2
:10FEE00061BD012900F05B8501239BF8CC2009F15D
:10FEF0000C0903FA0AF30AF1010A1343BAF1040FD9
:10FF00008BF8CC307FF497ADFEF737BE511D99F8D2
:10FF1000050015F0BBFB00283FF404AAB8F1010F5F
:10FF200040F0DF8709F10D0199F80A0015F0AEFBEA
:10FF3000002840F0D2874A4999F80F0015F0A6FB37
:10FF400000283FF403AAB8F1030F40F0C2874549E7
:10FF500099F8140015F09AFB002840F0B687424942
:10FF600099F8190015F092FB00283FF403AAB8F1A4
:10FF7000050F40F0A6873D4999F81E0015F086FB55
:10FF8000002840F09A873A4999F8230015F07EFB43
:10FF900000283FF403AAB8F1070F40F08A873549DB
:10FFA00099F8280015F072FB002840F0A987324923
:10FFB00099F82D0015F06AFB00283EF4F6AEB8F172
:10FFC000090F3EF4F2AEFFF7FDB910202B4F08F0F9
:10FFD000D3FE202008F0D0FE294B0022B6F8008086
:10FFE0001A7000212748284B284A016011602848D0
:10FFF000284A196000234160816103608360436186
:020000040801F1
:10000000C36113605160936053619161D361FEF7E6
:1000100037BE00BF183D0120A4000120A7DFA8348F
:10002000DB0FC93F00000000781C0120DB0F4940B6
:10003000DB0FC940E4CB1641DB0F49C0E4CB16C14E
:1000400092E741B99730083C15A82ABEB427012091
:10005000184B0408E42801203D920120A42101202E
:10006000B9280120BE280120C3280120C82801206A
:10007000CD280120D2280120D7280120403B012093
:10008000D437012008240120C8240120C0380120D1
:1000900070380120983801205D2A00F07D825B2AAB
:1000A00000F0DD855E2A00F04786562A00F0F286D1
:1000B000972A00F01A87A72A00F03086B84E3388B6
:1000C000990740F0F985A2F1B703072B00F28C8263
:1000D000DFE813F083028A028A028A027C028A0223
:1000E0006D026D02002D3BD05CF823005900834562
:1000F000FFF48DABAB485FFA83F9AA4E405C0E4427
:10010000002841D0022851D1707800EB800000EB2C
:10011000800000F2EE2080B2032B3DDD00B2BEF184
:10012000000F3FF479AB0D9E22F816000A9E1EB90F
:100130000F9E022E7FF670AB0120B2F800909A4E0F
:100140000A9050884844B2F80490484400B286FBB4
:100150000069964E7052A9EBE07000B2FFF75CBBED
:10016000284659000B9E4CF82360FFF751BBD3B2D1
:10017000022B06D9032B73463FF496AB0B88FFF78F
:10018000A1BB3B46FFF790BBB9F1020F40F20484DC
:10019000B9F1030F0AD11398012600B206FA03F948
:1001A000109E26EA09061096FFF732BB605AB3E7A5
:1001B00031467F480CF098FF002800F0908084F8CA
:1001C00093602FF0C7FAFEF749BC44F04003A34206
:1001D00033807FF444AEFEF744BD44F004039C42F8
:1001E00033807FF450AEFEF732BD724B012272496C
:1001F0001A70724B129105931B216D480CF074FF1D
:1002000000287FF41EAB6E4BDFF8D0B1194609937E
:10021000DBF80030CA688B609B1AC82B00F230856F
:10022000079B1E6806F48056FFF752BB27F00103B8
:100230009BB2BB4233803FF400AD0E2084F80080B7
:1002400084F801B084F802A030F014FC3788F4E49C
:1002500000225A4928460EE0437803EB830303EB60
:10026000830303F2EE239BB2013221F8023B0230FA
:10027000A2423FF42DAB15F812301BB1022BEBD08C
:100280000B88F1E75FFA82FE3B46BEF1030FEBD924
:100290000B88E9E7B3F5FA7FFEF650AF94F89220A9
:1002A000002A7EF44BAF089A0121127884F892104C
:1002B0000A4000F0E2832EF08BFDFEF73FBF0025E1
:1002C000FFF7E6B83F4A1278002A7FF414A9012C00
:1002D00040F0F4869BF820300325FFF7E3B8089B35
:1002E000394A1B781060D8077EF5BDAB374B1B78B9
:1002F000002B3EF423AF099BDB78002B7EF41EAF6E
:1003000094F893300133DBB2032B84F893307EF6FC
:1003100015AF2F4B5B7813B9002D7EF40FAF2EF085
:1003200057FDFEF79BBBB3F5FA7FFEF607AF94F8D7
:100330009220002A7EF402AF089B01211B7884F8EA
:100340009210D90700F15D842FF004FAFEF7F6BE93
:10035000099BDB78002B7FF4C8AADFED1E7AC8F575
:10036000FA631D4938EE678A1AB2FDEEC87ACDED00
:10037000057ABDF914301B0381FB0301DB17C3EBC6
:10038000A11302FB03F343F30F33434407EE903A08
:100390000D9BB8EEE78A87ED038AFFF7ACBA00BF82
:1003A0006C3D0120202F0120565555551422012067
:1003B000F43E0120963E0120C52D0120247D012020
:1003C0007C92012024240120F8B701203D920120D5
:1003D00090A3012000007A44D34D62103CC201205A
:1003E000C04B47F6FF76C04A1968B4F99030C96926
:1003F00082FB0172C91792118F1A3E44B3423EF735
:1004000020AB521A13441BB2A4F89030FEF719BB6C
:10041000B64A069BD5881B8B059AB2F906105A1B63
:10042000914240F3A3802B449942B4BF002501259B
:10043000FEF715BAC8398A4263DA9BF8CC109A786D
:1004400041FA0AF3D8073FF52AAB524201200E9237
:1004500030F036FC631E0E9A162B00F21781DFE88F
:1004600013F0240238020D025D024C026F02E40117
:10047000D101BC01A701920115015D027F016F024C
:10048000E401D1016B012C011801F701EE0002011A
:1004900015F0BAF8032140F6B8328BF82010CBF8EB
:1004A0001C20FFF730B80999D9F80020CB69134414
:1004B0008B61002D3EF4C2A9FFF791B80A2015F018
:1004C0000DF9B6F800808146002800F0538318F03B
:1004D000100F00F0D084864C94F8D490B9F1000F3E
:1004E0007FF41AAB834F0D2030F0C4FA0123B6F825
:1004F000008084F8D430B9F1000F7FF472ADFEF7BC
:10050000BFBB01229BF8CC3008F5FA7102FA0AF25F
:10051000C9F8081023EA02038BF8CC30FFF7BFBA02
:1005200086FE654AC4EE054A9FED732A9FED735A15
:10053000DFED731ADFED732A9FED733ADFED733A47
:100540009FED734AA4EE825AE4EEE12AA4EE857A86
:10055000A4EEA23AB0EE475AB0EE637AA4EE837AE4
:10056000A4EE874A84EE057AFFF7DCBB0125FEF78F
:1005700076B9002167480CF0B7FD00287EF4F8AD8D
:10058000322384F89600A4F89830FEF7F1BD002AD3
:100590000CBF012002205AE75F4B002201205F4C74
:1005A0005F4922700B6030F08BFBFEF7C7BD5B4BE1
:1005B00002225C495A705C4B0A910B6015F0F2F80C
:1005C000079B1B6803F00403FEF77FBA534B00221E
:1005D00054495A700A91554BEFE7504B012251494B
:1005E0005A700A91524BE8E7792A00F0EA847A2A95
:1005F00000F0E0849E2A00F0D5849D2A00F0CA8491
:10060000AE2A00F0BF84AD2A00F0B484EF2A00F0D7
:100610009D84FD2A00F08684FB2A00F03885FE2A9E
:1006200000F03285F72A00F035857B2A7EF447AA50
:100630004FF4FA6102202FF0B7FCFEF740BADBF866
:10064000D0003C4F90F83710BB781144FE29A8BF6A
:10065000FE2121EAE17180F83710002B40F031854E
:1006600014F070F940E4DBF8D000324F90F8361007
:10067000BB7811446429A8BF642121EAE17180F8A4
:100680003610002BECD0172015F072F8DBF8D000F4
:10069000E6E7DBF8D000274F81781144C829A8BFCE
:1006A000C82121EAE1718170BB78002BD8D01420D9
:1006B00015F05EF8DBF8D000D2E7DBF8D0001D4F74
:1006C00041781144C829A8BFC82121EAE1714170CD
:1006D000BB78002BC4D0132015F04AF8DBF8D0000B
:1006E000BEE700BFA4A20120D34D621058350120FF
:1006F000A4210120403B012099FB243F69A2163E22
:1007000039094E3DE3B59E3E88FA163E45FE7F3FD1
:10071000A7DFA834F43E01207E440120D93D01200A
:10072000703D0120743D0120FE3D0120E63D012089
:10073000F23D01209E450120DBF8D000BC4F01783E
:100740001144C829A8BFC82121EAE1710170BB7812
:10075000002B85D0122015F00BF8DBF8D0007FE7D6
:10076000B34F0C98BB78417911446429A8BF642128
:1007700021EAE1714171002B88D00E2014F0F8FFBE
:10078000DBF8D0006CE7DBF8D000A94F017ABB782A
:100790001144C829A8BFC82121EAE1710172002BC8
:1007A0003FF45EAF0B2014F0E3FFDBF8D00057E717
:1007B000DBF8D0009E4FC179BB781144C829A8BF8F
:1007C000C82121EAE171C171002B3FF449AF0A2031
:1007D00014F0CEFFDBF8D00042E7DBF8D000944FF6
:1007E0008179BB781144C829A8BFC82121EAE171E9
:1007F0008171002B3FF434AF092014F0B9FFDBF80E
:10080000D0002DE7DBF8D000894F4179BB78114447
:10081000C829A8BFC82121EAE1714171002B40F02D
:100820001384112C7FF438AF1AE7DBF8D000804F27
:100830000179BB781144C829A8BFC82121EAE17118
:100840000171002B40F02984102C7FF439AF07E7A9
:100850000C98774F41781144B1F5967FA8BF4FF4BB
:10086000967121EAE1714170BB78002B3FF40EAF25
:10087000152014F07DFFDBF8D000F1E60C996C4FE9
:100880000C791444642CA8BF642424EAE4740C7129
:1008900014F088FFBB78002B3FF4F8AE032021460C
:1008A00014F066FFDBF8D000DAE60C98604F0178B0
:1008B0001144FA29A8BFFA2121EAE1710170BB783D
:1008C000002B3FF4E3AE012014F052FFDBF8D00020
:1008D000C6E60C98564F817811446429A8BF64215C
:1008E00021EAE1718170BB78002B3FF4CFAE02208A
:1008F00014F03EFFDBF8D000B2E60C984C4FC17903
:10090000BB78114481F30801C171002B3FF4BEAEE6
:10091000052014F02DFFDBF8D000A1E60C9B444F1E
:100920009979B87811446429A8BF642121EAE1715A
:100930009971002840F091830D2C7FF412AFA5E649
:10094000DBF8D0003A4FC178BB781144C829A8BF62
:10095000C82121EAE171C170002B40F0A7830F2C60
:100960007FF4EDAE7CE6334947000B683BB15C7821
:100970003B1802EB83035B78A342BEF479A90744DA
:100980002D4C0020D9F8003002EB87022B4F20803D
:100990000A603860FEF76EB91198FFF7BDBB987812
:1009A0004FF49661059B33F91230B3F5617F91FBEB
:1009B000F0F2C0F2318140F633019942A8BF1946E6
:1009C0000C2CA1F5617191FBF2F100F09D82182CC5
:1009D0007FF48AAAC9B2C8290B46A8BFC823DBF88E
:1009E000D020D8B2D47DA0423FF47EAA1B1B104F6A
:1009F000D07548BF0733DC10BB780134E4B23BB993
:100A0000002C3FF471AA204630F05AF9FFF76CBA77
:100A1000182014F0ADFEF3E7DFF82490642172880B
:100A2000D9F8003001FB0233CBF81030FEF7A7BD38
:100A30009E450120DC230120CC240120D02401206C
:100A40003CC20120BE4B4FF47A72BE491B68B2FB18
:100A5000F3F2079BC2EB42101B6802EB80021F06F9
:100A60004FEAC202A1F8AC203EF55CABB64A03F0F7
:100A70000403B64E0A92FEF728B8B549096811F486
:100A8000003140F0E7810846B24A555C0C310F2D29
:100A900000F0938001301828F7D1A3F1FA01002269
:100AA000079B84F892201B68A74AA4F8901003F0D3
:100AB0000403A64E0A92FEF708B8A74943000C6843
:100AC0003CB167781C1802EB84046478BC42BEF425
:100AD0004FA80344A14C002002EB8302A04B2080CE
:100AE0000A601860FEF744B8B4EEE77AF1EE10FA47
:100AF00040F37E82DFED9B5A9FED9B6AF4EEC66A5F
:100B000076EEE57AF1EE10FAF0EE676AF6DCDFEDEC
:100B1000976AF4EEE67AF1EE10FA40F16682DFEDC4
:100B2000915A9FED936AF4EEC67A77EEA56AF1EEDC
:100B300010FAF0EE667AF6D4DFED8E7AF4EEE76A1C
:100B4000F1EE10FA40F3AB80DFED8B7A77EEE66AD8
:100B500066EEA65A9FED895A9FED896ADFED897A84
:100B6000A5EE856A26EEA55AE5EE867AE5EE276AB9
:100B7000FFF702B918F0100F40F05B810B2014F062
:100B8000ADFD002840F01C817F4F18F0200F40F091
:100B9000BD817E4C94F8D430002B3FF4A4ACB9F165
:100BA000000F7FF41EAAFEF76BB8794B1B78032B5E
:100BB00000F0A2810023FFF73FB9674945000E68A6
:100BC0003EB177782E1802EB86067678BE42BFF4E7
:100BD00064AF0544614E002002EB8502604D308019
:100BE0000A60286059E7DFED6B7AB4EEE77AF1EE40
:100BF00010FA7FF507A9DFED5D7A37EEC77AFFF7C8
:100C000001B96549079B0A601B684F4A03F004035A
:100C10004E4E0A92FDF759BF0C2C40F0158100246E
:100C200021465E4B0E915B78A3423FF45DA95C4F79
:100C300020462FF025FA0E99BB781BB1C9B20C20C3
:100C400014F096FD0134E4B2DAE6DFED4B6A36EEDD
:100C5000C77AFFF778B806F48056FEF739BE514BD5
:100C6000012202209BE438EE678AC8F5FA634E49F8
:100C70001AB24E4BFDEEC87ACDED057AFEF75BBE9B
:100C800008464B4A0121136880F82110079923F088
:100C900004030E68136006F48056FEF719BEDFEDFC
:100CA0003D7AF4EEE76AF1EE10FA7FF551AFDFED31
:100CB0002F7A77EEE66A4BE70023BB2A149300F005
:100CC0008B81B72A00F08481BE2A00F08C81BD2A76
:100CD0007FF48AAC4FF6FE71364A1B48D5890A90DC
:100CE00090892B440144D381918111F0BBFC0BF01E
:100CF00013FA11F09FFC08F011FD01202FF0E0FF26
:100D0000B4F89020079B0021FA3A1B6884F89210EF
:100D100003F00403A4F89020FDF7D7BE2649079BF3
:100D20000A781B6842F00402074803F00403074EE8
:100D30000A900A70FDF7C9BE204B022203202EE460
:100D4000D0560120DC4E0120743D01206C3D012075
:100D5000B4270120184B0408DC230120CC240120F7
:100D6000D0240120DB0FC940E4CB1641DB0F49C082
:100D7000E4CB16C1DB0FC93FDB0F494092E741B915
:100D80009730083C15A82ABE403B0120A421012031
:100D900076920120DB0FC9BFF8B70120D93D0120B1
:100DA0009E450120CC440120D34D621060240120D7
:100DB000683D012070A301206E3D01201A450120ED
:100DC000C54BC64F5B8997ED007A07EE903AB0EEBF
:100DD000C77AF8EEE77AB4EEE77AF1EE10FA7FF52B
:100DE000D4AE97ED017AB0EEC77AF4EEC77AF1EEA1
:100DF00010FA7FF7CAAE18F0200F7FF4CAAE202099
:100E000007F0D2FFB64B60681946226841F8040F1C
:100E100018461A6019F0E6FAB24B01221A70B24C69
:100E200094F8D430002B00F05381B6F80080FFF71F
:100E3000D8B8102007F0A0FFAA4BB6F8008083F8BE
:100E400000904FF0010999E6182C7FF44DA800217D
:100E50000B46C4E5A549097803295ED0114612E680
:100E6000A24B1B78032B00F0BA800023FEF739BE9B
:100E70001A46FEF7A9BA1020984F07F095FF2020D8
:100E800007F07AFF9A49081F19F0ACFA954B022235
:100E90001A70C4E711F0E6FB0BF03EF911F0CAFB43
:100EA00008F03CFC01202FF00BFF94F88E20FFF798
:100EB000FFB807221346FEF787BA06221346FEF74D
:100EC00083BA05221346FEF77FBA04221346FEF7C3
:100ED0007BBA03221346FEF777BA02221346FEF7C7
:100EE00073BA01221346FEF76FBA824A4FF4C871F3
:100EF000079B11801B68B9E52FF0A0FDFDF7B8BE78
:100F000008221346FEF760BACCB28AE6202007F02A
:100F100033FF744B00221A7081E72FF08FFDB4F974
:100F20009030BAE5002101202FF03EF8B4F890206F
:100F3000079B0021963A1B68A4F890206E4A03F0A4
:100F4000040384F892100A92FDF7BFBD00216A4B9A
:100F500008460A932FF028F8B4F89020079B002148
:100F6000963A1B6884F8921003F00403A4F89020CA
:100F7000FDF7ABBDFF21002021F09CFD94F88E20F1
:100F8000FFF744BB0121002021F094FD94F88E204E
:100F9000FFF739BB0021FF2021F08CFD94F88E2053
:100FA000FFF72EBB0021012021F084FD94F88E2054
:100FB000FFF723BB514A137A43F001031372FDF785
:100FC0007EBD4E4A137A23F001031372FDF777BDFD
:100FD00019464FF6FE737FE6194602237CE62FF092
:100FE0002DFDFDF7C5BD022176E6F0EE676AA3E5AB
:100FF000F0EE667A8BE5B0EE677AFEF7F7BEF0EEBC
:10100000477AFEF7DEBE3C4B84F8941084F89500D6
:101010003B4E0A93FEF79DB8002D3DF46AAC324C6E
:1010200094F88D30002B3DF4C2AC2FF007FD002367
:1010300084F88D30FDF7BBBC2DF0CAFE2A4C00238E
:1010400084F88D30FDF7B3BC11200E9214F090FBA4
:10105000DBF8D0000E9AFFF7E4BB0D200E9214F0DF
:1010600087FB0E9A68E4002BD9D026494FF47A709A
:10107000254A096800FB03131360D0E70B20204EBC
:101080002FF0F8FCFDF71BBD002103204CE70021E9
:10109000022049E70021042046E710200E9214F0B8
:1010A00067FBDBF8D0000E9AFFF7CEBB0F200E9245
:1010B00014F05EFBDBF8D0000E9A50E40325FEF737
:1010C0008EBA162014F054FBDBF8D000FFF7C8BA34
:1010D0004FF00109FFF707BA64380120403B0120B7
:1010E0008C220120D4370120A421012076920120F6
:1010F000CC37012092350120743D0120E8380120D1
:101100006C3D01203CC20120F4B70120B0F9083049
:101110002DE9F04FDDB28DB00C461746442D0B8102
:1011200000F05084064643D9812D00F0828300F2FE
:101130009980542D00F0D08040F2DA806E2D00F0BE
:101140000F84802D40F0D780764B93F8009009F102
:10115000020919F0FF0900F09880734B0A25734FBC
:10116000994403F10108724EDFF8ECA117E0322D2B
:1011700001F0EE82A5F13C00C0B2132841F2F282E8
:1011800000232268C84502F1010121601570226820
:1011900002F101012160137077D018F8015B0A2D6C
:1011A000E5D1BAF80030FF2BA8BFFF23DBB2E8E798
:1011B000052D00F0F5831FD8022D00F0858040F248
:1011C0001A83032D00F0BC83042D40F094802A463E
:1011D000584920460BF074FA002120460BF0B4FA6F
:1011E000216801230020CD181A4625600870184692
:1011F00062810DB0BDE8F08F242D63D040F2A8824B
:10120000282D00F05F83382D75D10A68012005274D
:101210000A261318002548492360034610702068E9
:101220001A4600EB030EC4F800E007702068C718E8
:10123000276006702068C6182660057020680D7843
:10124000C6182660057020684D78C618266005709F
:1012500020688978C51825600170184662810DB034
:10126000BDE8F08FA02D17D040F29682B82D00F087
:101270006583FE2D3FD1314D05F1080635F8021B7F
:1012800020460BF061FAAE42F8D101231A46184607
:1012900062810DB0BDE8F08F294B084619680BF04C
:1012A0003DFA284B204619680BF038FA264B2046A9
:1012B00019680BF033FA01231A46184662810DB003
:1012C000BDE8F08F214BF2E70422214920460BF0C4
:1012D000F7F901231A46C0E7096801230020CD1859
:1012E0001A46256008702168CD1825600870B4E79B
:1012F000522D3FF475AF2146284606F075FC014695
:101300000028C2D1742D00F08A82772D26D133684F
:1013100072689A4240F062830E4A20462FF084FDA4
:10132000B3E700BF653901200C45040867666666AF
:101330003CA40120DF3D01206944012088390120BF
:10134000107AF01F147AF01F187AF01FB4450120AC
:10135000BC760408B100040864A40120F52D01F056
:101360009782762D00F03E83292D376801F05A824E
:10137000392D01F02C82212D01F06A8272680B3D1B
:10138000D31BEF2D00F2AC8501A050F825F000BF73
:1013900049220108E11E0108E11E0108E11E0108C1
:1013A000E11E0108E11E0108E11E0108E11E01081D
:1013B000E11E0108E11E0108E11E0108E11E01080D
:1013C000E11E0108E11E0108E11E0108E11E0108FD
:1013D000E11E0108E11E0108E11E0108E11E0108ED
:1013E000E11E0108E11E0108E11E0108E11E0108DD
:1013F000CF210108E11E0108B5210108E11E010805
:101400002F210108E11E0108E11E0108E11E01086B
:101410004D230108E11E0108D7220108E11E010841
:10142000A5220108E11E01087F220108E11E010832
:101430001D210108E11E0108BD200108E11E01086F
:101440006D200108E11E0108E11E0108E11E0108EE
:10145000E11E01088B120108E11E0108412001086C
:10146000E11E0108E11E010831260108E11E010804
:10147000751A0108E11E0108E11E0108E11E0108BC
:10148000E11E0108E11E0108E11E0108E11E01083C
:10149000E11E01084B260108E11E01088F25010805
:1014A000E11E0108E11E010839250108E11E0108BD
:1014B000E11E0108E11E0108E11E0108E11E01080C
:1014C000E11E0108E11E0108D5240108E11E010802
:1014D00023240108E11E010875230108E11E01080B
:1014E000A9260108E11E0108092601088B2601082A
:1014F00073250108E11E0108E11E0108E11E010833
:10150000E11E0108E11E0108E11E0108E11E0108BB
:10151000E11E0108E11E0108E11E0108E11E0108AB
:10152000E11E0108E11E0108E11E0108E11E01089B
:10153000E11E0108E11E0108E11E0108E11E01088B
:10154000E11E0108E11E0108E11E0108E11E01087B
:10155000E11E0108E11E0108E11E0108E11E01086B
:10156000E11E0108E11E0108E11E0108E11E01085B
:10157000E11E0108E11E0108E11E0108E11E01084B
:10158000E11E0108E11E0108E11E0108E11E01083B
:10159000E11E0108E11E0108E11E0108E11E01082B
:1015A000E11E0108E11E0108E11E0108E11E01081B
:1015B000E11E0108E11E0108E11E0108E11E01080B
:1015C000E11E0108E11E0108E11E0108E11E0108FB
:1015D000E11E0108E11E0108E11E0108E11E0108EB
:1015E000E11E0108E11E0108E11E0108E11E0108DB
:1015F000E11E0108E11E0108E11E0108E11E0108CB
:10160000E11E0108E11E0108E11E0108E11E0108BA
:10161000E11E0108E11E0108E11E0108E11E0108AA
:10162000E11E0108E11E0108E11E0108E11E01089A
:10163000E11E0108E11E0108E11E0108E11E01088A
:10164000DD250108E11E01082B2001080120010809
:10165000E11E0108E11E0108E11E0108E11E01086A
:10166000E11E0108E11E0108E11E0108E11E01085A
:10167000E11E0108E11E0108E11E0108E11E01084A
:10168000E11E0108A51F0108711E0108351E010891
:10169000E11E0108991D01083D1D0108211D0108D9
:1016A000E11E0108071D0108A31C01087B1C01089D
:1016B000C51A0108CF1A0108E11E01080D1F010813
:1016C000E11E0108E11E0108EB1E01084F1F010881
:1016D0003B1F01087D1F0108C31E0108591C01089A
:1016E000271C0108E11E0108E11E0108E11E010896
:1016F000E11E0108E11E0108E11E0108E11E0108CA
:10170000E11E0108E11E0108E11E0108E11E0108B9
:10171000E11E0108E11E0108E11E0108E11E0108A9
:101720000D1C0108E11E0108E11E0108AB1B0108A8
:10173000E11E0108E11E0108E11E0108471B010826
:10174000E11E0108E11E0108E11E01082D1B010830
:10175000202D7FF4D0AD0B680846B34D591C6A7834
:1017600021601A7023682A78591C21601A70236836
:10177000AA78591C21601A7029890AF0E5FF2168AE
:1017800001236879CE181A46266008702168A87966
:10179000CD182560087060E5822D7FF4ACAD0B6834
:1017A0000846A24A5E1CA24D11789F4A2660197015
:1017B00011890AF0C9FF9F4B226820461B88511CE3
:1017C000FF2B2160A8BFFF231370A96881F31001CC
:1017D00089B20AF0B9FF2968204601F30F0189B2E6
:1017E0000AF0B2FF2168944A01231078CD181A46F6
:1017F0002560087031E5012D7FF47DAD0968002674
:101800002B4625204F1C2A4627600E7021684E1C4F
:1018100026600D7021684D1C256008701DE5336839
:1018200072689A4240F0D680844A20462FF0FCFA33
:101830002BE5834B1E78033616F0FF063FF425ADEB
:10184000804B4FF00A08804F1E4403F1010920E04D
:10185000B8F1500F00F08387B8F1320F00F098878D
:10186000A8F13C00C0B2132840F298870025294611
:10187000236820465A1C226083F800800AF064FF27
:10188000294620460AF060FF4E453FF4FEAC19F8A9
:10189000018BB8F10A0FDBD16C498B684FF6FF72F0
:1018A000096803EB830391424FEA4305A8BF114641
:1018B000954221EAE171A8BF154689B225EAE5758E
:1018C000ADB2D5E70B68022101250627581C0A2274
:1018D000DFF89C8120602046197023685C4E5919FE
:1018E00021601F702368591921601A7023685A19E2
:1018F00022601D70B8F800100AF026FFB8F8021038
:1019000020460AF021FF23685021002203EB050E38
:101910002046C4F800E01F7023685F192760197023
:101920002368591921601A7031880AF00DFF7188F7
:1019300020460AF009FF2B462A468EE4454BB6E4C2
:10194000096801230020CE181A4626600D70216810
:10195000CE1826600D702168CD18256008707CE4D3
:10196000344B08460A681B88511C314DFF2B2160FF
:10197000A8BFFF231370A96881F3100189B20AF090
:10198000E3FE354B204619880AF0DEFE2968204622
:1019900001F30F0189B20AF0D7FE01231A465CE475
:1019A0000B222E4920460AF08BFE08222C492046A5
:1019B0000AF086FE07222B4920460AF081FE012309
:1019C0001A464AE4002A3FF460AC274A01233A60F1
:1019D0001A4642E45A1C3260197825E75A1C3260D4
:1019E000197899E433685A1C32601B78002B00F098
:1019F000A887102B00F0BE870E461C4D226820469B
:101A0000571C276013700AF089FE314620460AF001
:101A100085FEE96820460AF081FE002120460AF092
:101A200093FEFFF7D9BB00BF043D01203E3B0120E0
:101A3000D83A0120383B0120769201206501040844
:101A4000653901201C45040834A40120F0A30120BD
:101A500024A40120B427012070920120C476040838
:101A6000D0760408DC760408597901088822012020
:101A700060A301207A1CDFF818830021B64B326086
:101A800030463A78C8F800101A7030F080FF32689B
:101A9000D8F80030571CB1490343B14D3046C8F85F
:101AA0000030376013780B720AF0F8FD286030467A
:101AB0000AF0F4FD686030460AF0F0FDA860304698
:101AC0000AF0ECFD30460AF0E9FDFFF7DEBB0D2B16
:101AD00040F006827B1C33603D78072D00F20082C7
:101AE0000C27DFF8B082304607FB05F70AF0D6FD79
:101AF00008EB0705A88030460AF0D0FDE8803046A4
:101B00000AF0CCFD3368288130461A46591C3160F2
:101B100012F8021BA97232605B78EB7230F037FF6B
:101B2000012348F807001A46FFF797BB8D4B1B7837
:101B3000DB0700F1D58107F021FC07F0EFFD012361
:101B40001A46FFF78ABB30460AF0A8FD3368ADF8A5
:101B50000C0000211A465D1CD81C1F1D35605D1D40
:101B600012F802EB32608DF80EE05A78306003A86C
:101B70008DF80F209A7837608DF81020DA7835606C
:101B80008DF811201B79ADF814108DF812300AF081
:101B9000F1FC754A0123754D16681A46801B61F1E8
:101BA0000001C5E90601FFF758BB7B1C33603B7899
:101BB0000F2B00F29581BA1CC3EBC3036C49F81CD0
:101BC000326007F1040E7D78CA18CD547D1D306057
:101BD000B81DBB78F91D537007F10803C6F800E083
:101BE00097F803E082F802E035603D79D570306007
:101BF000787910713160B97951713360FB799371E3
:101C000022F05CFC01231A46FFF727BB594D3046F2
:101C10000AF044FDE88130460AF040FD0123A88126
:101C20001A46FFF71ABB3A467B1C5349FD1C33602A
:101C3000381D12F802EB012381F800E032601A46E9
:101C400097F801E081F801E03560BD788D70306073
:101C5000F878C870FFF701BB484D30460AF01EFD0A
:101C6000288230460AF01AFD688230460AF016FDD6
:101C70000123A8821A46FFF7F0BA7B1C336038783C
:101C8000060600F11D87374B1B78DD073FF5FDAADF
:101C9000032828BF002007F057FB01231A46FFF74F
:101CA000DCBA7B1C3046336097F8009030F06FFE52
:101CB0008046304630F06BFE0746304630F067FE17
:101CC000054630460AF0EAFC30460AF0E7FC3046AA
:101CD0000AF0F0FCB9F1000F00F0DD86B9F1100F49
:101CE0007FF4D3AA214BC3F804809F6005B1DD6067
:101CF00023490222234B081F1A7018F073FB01239B
:101D00001A46FFF7AABA174B1B78D8073FF5BDAAAA
:101D100008F0F0F807F002FD01231A46FFF79DBA1C
:101D2000104B1B78DA073FF5B0AA1748012301785A
:101D30001A4641F004010170FFF78FBA094B1B7876
:101D4000D9073FF5A2AA114A4FF4C87101231180A7
:101D50001A46FFF782BA00BFA8400120384D012083
:101D600060B60120835901203CC201208822012055
:101D7000C826012070A30120C4350120887E0120DF
:101D800090220120D43701206E3D012092350120A0
:101D9000B445012008260120092B40F3A1803B46D1
:101DA0007A1CDFF80884F81C391DD8F8005032601E
:101DB00013F8022B2A707A1D33607B78AB70306089
:101DC000B81DBB78642BA8BF64236B713160F91D0B
:101DD000FB78642BA8BF6423AB71326007F1080263
:101DE0003B79EB71306030467B79642BA8BF64236C
:101DF0002B723160BB79EB703260FB792B710AF08A
:101E00004DFC726833686881D11A00290CDD581CBA
:101E1000D8F80010121A30601878002A487203DDD2
:101E20009A1C32605B784B7013F0BCFC01231A469D
:101E3000FFF713BAC64AFB1C2137106802469D1EE5
:101E4000591E0332356013F8035C02F8035C3160FD
:101E500013F8021C02F8021C3360033313F8041C4D
:101E6000BB4202F8011CEAD112F06CFDFFF70DBA7B
:101E70007B1CB84A33603B78002B00F0F98513785F
:101E800043F00203B91C1370B34D304631607B78C8
:101E90002B7530F07CFD2860304630F078FD6860AE
:101EA00030460AF0FBFB28813046AC4E0AF0F6FBC8
:101EB00001233178E8811A4641F002013170FFF7C1
:101EC000CCB9791C3B46FA1C316013F8020B336025
:101ED00079783260BA7828F0A7F900287FF4D5A97C
:101EE0004FF0FF331A46FFF7B8B99D4D30460AF060
:101EF000D5FB288030460AF0D1FB688030460AF0D6
:101F0000CDFB0123A8801A46FFF7A7B9DFF8A0820E
:101F100098F80030002B3FF4B8A9924F00253046C6
:101F200001350AF0BBFB12F05FFE98F80030A7EC19
:101F3000010A9D42F3DBFFF7A8B9854B4E228A497F
:101F4000186831F08AF801231A46FFF786B93A4635
:101F5000781C864BF91C3060304612F8025B1D700D
:101F600032607A785A703160BA789A700AF096FBCB
:101F70007B4A0123D0801A46FFF76FB939467B1C94
:101F80007B4AF81C3360012311F8025B15701A4676
:101F9000316078497D788D7030607749B878887085
:101FA000FFF75BB9C3F34705122D99D8BDB10CAB50
:101FB0000DF10A0803EB45094746A9F12609304609
:101FC0000AF06CFB27F8020FB945F8D16B4B38F8D3
:101FD000022FB84523F8022FF9D1112D0AD86B0032
:101FE00067480021023B00F12202034423F8021F4C
:101FF0009A42FBD10122634913460A70FFF72DB9BB
:102000007B1C614933600A783B78002A40F03585B3
:1020100004220A709B005D4A138008F0A1F85C4A14
:10202000012310621A46FFF718B90023594D3046B4
:102030002B6030F0ACFC012328601A46FFF70DB985
:102040003B46781C5449306013F8020B8870934269
:102050003360787848703FF418A9FA1C4C49012382
:102060003260B8781A460875FFF7F7B80722B3FB55
:10207000F2F2C2EBC2055B1B7FF432AFD2B202F1C7
:10208000FF395FFA89F9002A3FF4FFA809F1010935
:102090001D46DFF808A17A1C404B4FF00008326063
:1020A00097F9001093F9022008338A4200F0678400
:1020B00008F10108B8F1060FF4D111E77B1C336079
:1020C00039780E293FF60CAFBB1C336078780328B3
:1020D0003FF606AF0623324AFD1C07F1040C03FB52
:1020E00001F307F1050ED11848713560BD1DB878B0
:1020F000D054F81DC6F800C00123FA784A701A4679
:10210000C6F800E097F804E081F802E035607D79D8
:10211000CD703060B8790871FFF79FB87A1C2149FB
:102120000123326038781A464875FFF796B81E4D7D
:1021300030460AF0B3FA286030460AF0AFFA686019
:1021400030460AF0ABFA0123A8601A46FFF785B8BB
:10215000703D01206E3D01204C5F0120D2370120EF
:102160005835012034290120605B040868A3012050
:10217000BC56012070A3012080A30120222C012045
:10218000242C0120482C0120F62C012070920120E3
:1021900088220120B427012090A30120644D012052
:1021A000C0270120384D012060B60120743D012078
:1021B00065390120BB4D002330462B6030F0E7FB32
:1021C0002A68012310431A462860FFF746B87B1C93
:1021D000019133603D78132D3FF682AEBB1C336016
:1021E00078782EF05BFE00283FF47AAE90F800E09D
:1021F000FA1CAD4B381D019903F825E003EB85056A
:1022000032607A1D97F802E085F801E0306003F152
:10221000500097F803E085F802E032603A79EA70FE
:1022200002E00433834207D01A78002AF9D19D785E
:10223000DA789542F5D201219C4A81F0010101230F
:1022400011701A46FFF709B8102B99494FF0000298
:1022500028BF10230A604A608A60CA600A74002B93
:102260003FF413A8326801391344013232609A42B4
:1022700012F8010C01F8010FF7D1FFF706B87A1C2C
:1022800032603D781F2D3FF62BAE052B7FF428AE34
:10229000304630F07CFB874B43F8250014F060FC9F
:1022A000FEF7F3BF834D05F14007304604350AF0D1
:1022B000F5F93368A5F87C00591C1A46316012F80C
:1022C000021B85F87E1032605B7885F87F30AF4264
:1022D000EBD1FEF7DABF7B1C774D304633603B789D
:1022E0002B720AF0DBF9A88330460AF0D7F928836D
:1022F00030460AF0D3F9336868835A1C32601B7881
:10230000EB7473689A1A032A00F3938331685A1A9C
:10231000052A0EDD4B1C304633600B78EB7230F033
:1023200036FB3368E8605A1C32601B782B7496E8E1
:102330000A005B1A002B7EF7A8AF4A1C012332600B
:102340001A46097885F82110FEF787BF7B1C5B4889
:102350003360D31A3A78002B02707EF796AFBA1C1E
:10236000012332601A467978003118BF012141708B
:10237000FEF773BF7B1C524DDFF85481304633604B
:10238000D5F800903B7888F805300AF087F9A9F86D
:10239000200030462F680AF081F996E80A00F88399
:1023A0005A1A072A15DD30460AF078F9A8F80A000B
:1023B00030460AF073F92F68A8F80C0030460AF08E
:1023C0006DF978842F6830460AF068F996E80A00BB
:1023D000B8845A1A032A0BDD30460AF05FF9A8F8D0
:1023E0000E0030460AF05AF996E80A00A8F81000E4
:1023F0005B1A002B05DD4A1C2B6832600A7883F8D3
:10240000262007F0EDF81EF03FFE2E4B1B68002B38
:1024100000F00483286811F0C7FE01231A46FEF776
:102420001CBF3B467A1CDFF8A880F91C32603A1DBD
:1024300013F8025B304688F802503360224D7B78F7
:102440002B703160214DBB782B713260FB78092BEA
:10245000A8BF0923AB700AF021F996E80A0028808A
:102460005A1A012A05DD30460AF018F996E80A00E2
:10247000E8818B4207D04B1C33600B78003318BFC8
:10248000012388F8073007F0ABF896E80A008B4282
:102490003EF4FBAE4A1C012332601A460978E9700B
:1024A000FEF7DBBEB4450120102E0120DC00012028
:1024B00044A30120C0900120384D0120A8400120F4
:1024C000703D0120A440012064A30120887E0120EA
:1024D000BC560120C64B1B68002B3EF4D6AE18F04C
:1024E0006DF8FF283EF4D1AE30460AF0D7F83F2809
:1024F00040F2F1820025BF4F72683D703368B880AA
:10250000D21A012A7EF7C1AE5D1C1A4600210CA822
:10251000356012F8025BBD7032605D7800F8241DF2
:1025200018F028F89DF80C30AB423EF4AEAE2846C9
:1025300030F04AFAFEF7A9BEAF4B1B78012B3EF6EE
:10254000A4AE7B1CF91C3846AC4D3360531A10F80E
:10255000022B012BAA70306097F801E0316040F344
:10256000C78230460AF09AF8012328801A46FEF7FF
:1025700074BE7B1C33603B78002B00F083824FF4E9
:10258000004006F029FC01231A46FEF766BE7B1CBC
:10259000336097F80080B8F1110F3FF6A1ACBB1C77
:1025A000974D3046336019267B7805F8183005EBD7
:1025B00048050AF073F840F6CA0340F2EE2298424A
:1025C000A8BF184601239042B8BF10461A46A0F291
:1025D000EE2191FBF6F16970FEF73FBE791C3B4698
:1025E000FA1C316013F8025B336078783260B97896
:1025F000002D00F08982012D7EF447AE2DF022FDE2
:102600002B462A46FEF729BE39467B1C7D4AF81C1C
:102610003360012311F8025BD5701A4631607A49A4
:102620007D784D7130607949B878C870FEF715BE75
:10263000774B07F1080201373760BA4217F8011CDF
:1026400003F8011FF7D1FEF720BE3B467A1C714DFF
:102650003046326013F8022B2A7133607B786B713D
:102660000AF01CF83368288030465A1C32601B7808
:10267000AB710AF013F8316801236880C8181A4654
:1026800030600978E971FEF7E8BD634B1B7813F001
:1026900001017FF425AC7B1C336038782DF084FC7D
:1026A00001231A46FEF7D9BD30465C4D09F0F6FF0E
:1026B000304609F0F3FF304609F0F0FF304609F0EC
:1026C000F9FF33682A68304619465F1C3760DF1C03
:1026D00011F802EB82F82CE03160597882F836105C
:1026E00037609B7882F8373009F0E4FF304609F014
:1026F000E1FF304609F0DEFF2F68304609F0CEFFDB
:10270000788730462F6809F0C9FF96E80A003887B5
:102710005A1A012A0ADD4A1C2B68304632600A78B0
:1027200083F82E2009F0C6FF96E80A005B1A032BF7
:102730000BDDD5F80080304609F0B0FF2F68A8F80F
:102740003200304609F0AAFFB8862868FFF78CBB34
:102750003388FF2BA8BFFF23DBB2FEF712BD304941
:10276000FFF79BB815F0B2FF00283EF409AD0378DF
:102770000A2B2AD8B0F9023087FB0312DB17C3EB10
:10278000A2039BB2FF2BA8BFFF23DBB2FEF7F9BC6D
:102790007B684FF6FF723968FFF783B815F096FF34
:1027A00000283FF463A803780A2B3FF65FA8B0F92E
:1027B0000430B0F9061003EB830321EAE17183F3DF
:1027C000500589B2ADB2FFF753B80023DDE77B1C9B
:1027D00033603B780A2B00F0BC80304609F06AFF7A
:1027E000304609F067FF304609F064FFFEF74DBD43
:1027F000885901208C5901209C4501209E450120CB
:10280000202F012070A3012094A2012080A3012089
:10281000374D01207035012083590120703D012082
:1028200028A401207B1C33603B780A2B00F08F80AA
:10283000502B7FF444A9B74D304609F02FFF288074
:10284000304609F02BFF012368801A46FEF705BDCC
:102850003B46791CB04DFA1C3160304613F8021B20
:10286000697033607B782B703260BB78AB7009F095
:1028700015FF316801232881CF1808461A463760B2
:1028800010F8027B6F7130604978A971FEF7E5BCE2
:10289000336872689A4240F09A80A04BFF221A7007
:1028A00000269F4D2CF058FA202231469D482E706C
:1028B00031F067FD8DF80C6032469DF80C30072B27
:1028C00032D8DFF89C82974E9DF80C3003EB43031F
:1028D00008EBC3035B7CEBB19DF80C30202103EBCC
:1028E000430308EBC3035B69A3B19DF80C3003EB12
:1028F000430308EBC3035B6946F82230184607F030
:1029000083FF2B7856F8230007F088FF2A780132DE
:10291000D2B22A709DF80C300133DBB28DF80C3046
:102920009DF80C30072BCFD92368591C21601A70F1
:10293000002F3EF4AAAC7C4A01233A601A46FEF707
:102940008CBC7A4A754D92E84200FFF757B8784D33
:1029500072E7BB1C7749FD1C381D336001237A7870
:102960000A701A463560BD784D703060F87888700E
:10297000FEF773BC694D6968AE68FFF73FB80AEBB4
:10298000C80B304601358BF8021009F087FE32681B
:102990002AF83800A945134602F1010002F10301AB
:1029A00002F10407306013F8020B8BF80300336068
:1029B00053788BF80430316093788BF806303760A9
:1029C000D3788BF805307FF466ABFEF75EBC5A1CFB
:1029D00019465248326011F8022B0270042A316005
:1029E0005B78437003D9FF2A7EF4FAAB58E752496B
:1029F0000978994205D8FF2B7EF4F2AB022A7EF4C7
:102A0000EFAB22680123D11821601370002F3EF430
:102A10003CAC4A491A463960FEF71FBC48490123BD
:102A2000484E494D1A464948316029600160FEF719
:102A300014BC304609F032FEA884304609F02EFE60
:102A400096E80A00E8845A1A032A7FF760AC0B461E
:102A50004A1C3046326013F8022BAA7733604B7859
:102A600085F8203009F01AFE96E80A0068844EE4E2
:102A7000137803F0FD03FFF705BA042A7EF405ACD2
:102A8000FFF7C8BA3248012301681A4621F4004111
:102A90000160FEF7E2BB254B1020C3F800805F60A9
:102AA00006F06AF92B4A137843F001031370002DE6
:102AB0003EF4EBAB194A0123D5601A46FEF7CDBBB5
:102AC00000F07F00032828BF00202DF0D9FA012351
:102AD0001A46FEF7C2BBC50800F007031E4F0135BA
:102AE0000133EDB219467B70284615F093FD03E5DE
:102AF0001A4A0123B87811881A4611FB0EF191FB8E
:102B0000F0F12980FEF7A9BB11F09EFD01231A46C2
:102B1000FEF7A3BB24A40120043D0120882201204C
:102B2000DD280120C82501209DE60108C8370120C5
:102B300060A30120694401206539012065790108FD
:102B400041B40108FC2F01205030012050340120F5
:102B5000683D01206E3D01208C5901202CA30120ED
:102B6000205801202DE9F04FDFF89CB32DED0C8BA0
:102B700093B0DBF80420059058469047002876D0A3
:102B80000021BBF8AC408BF85510002C41F0E083DD
:102B9000BBF94060DBF84C20DBF82450B31ABBF9DA
:102BA0003C40BBF93E0083EAE371641BDBF828502C
:102BB000A1EBE371CBF83040401BB1F5804FCBF86F
:102BC000340002DC3246CBF84C60DBF82C10DFF826
:102BD0003CA3521AB1489BF85610CBF838201BF092
:102BE000B5FADAF80020910041F1CB849BED0D7A23
:102BF000AB4CB8EEC78ADBED0C7A9BED0E7AD4F8BD
:102C00000C21F8EEE77AF8EEC78AA64994ED406AFF
:102C10000132D4ED416A94ED427A77EE867A096802
:102C200038EE268A78EE878A9F4B8A42C4ED407A36
:102C300084ED418AC4ED428AC4F80C21039302F06A
:102C4000468193F800E0BEF1140F03F0D380002317
:102C5000D4F814510493062D01F22581DFE815F014
:102C6000C11496152D1359149608A915B6138E4B39
:102C70008B4C1D780393072D01F0688194F828315F
:102C8000079353B1013B84F82831012D01F02A84C8
:102C900013B0BDEC0C8BBDE8F08F844A5279002A4A
:102CA00001F0B581824A1278013AD2B2072D84F838
:102CB000282102F0CE8100230993D4F83421B7EE05
:102CC000007A059800269FED7B6A821A94ED4CAA43
:102CD000DFF83C82354607EE902A774908F11C035D
:102CE00077EE4A8AF8EE677AD1ED006A0893734B63
:102CF00068EEA68A86EE279A714AD3F800A0714F33
:102D0000C8FEC78A704BDFF80C9294ED4BCADFED1A
:102D10006F9A9FED6FBADFED6FBADFED6FAA069283
:102D2000C4F8340104936D4B98ED008A3344D3ED1D
:102D3000007AF5EE407AF1EE10FA17D0684B334482
:102D400093ED007A78EE476AB0EEE66AF4EEC67A62
:102D5000F1EE10FA08D5F5EEC06AF1EE10FACCBF2C
:102D600037EE878A37EE678A83ED008A5D4B1A88D3
:102D700093073AD0022D38D05B489AF82E1030F9DC
:102D80001500089B07EE901A07EE100A68003344FE
:102D9000B8EEE76AB8EEC77AD3ED006A4B42A6EE0A
:102DA000267A07EE903AF8EEE77AB4EEE77AF1EE9B
:102DB00010FA05D407EE901AF8EE677AC7FEC77AC4
:102DC0004A4B4B490344085EB3F90C30C31AD00791
:102DD00007EE103AB8EEC77AE7EE697A41F1C080A3
:102DE000444B93ED008A27EE888A069B94F86C2169
:102DF000334493ED01DA78EE4DCA002A00F0D48016
:102E0000D4F870213C4B05991B688A1A9A4240F30A
:102E1000CB809AF84830022B02F07C81022D04F01E
:102E2000BF84364B1B68990776D4354BC7ED00BA83
:102E30001B689342C0F2A880F7EE007AB4EEE7AACE
:102E4000F1EE10FA40F1B080069A2E4BD2ED017AE5
:102E500093ED007AF0EEE77AF4EEC77AF1EE10FA2D
:102E600040F1A280D2ED027AF0EEE77AB4EEE77A92
:102E7000F1EE10FA40F39880D2ED037AF0EEE77AA3
:102E8000B4EEE77AF1EE10FA40F38E801B4B1B682C
:102E90009B0779D51649154B5DE000BF0C4F01200B
:102EA000B8220120B040012084390120BC56012005
:102EB00064A3012000247449A4340120703D012042
:102EC000D0560120083F0120FC3E0120CDCCCC3D56
:102ED000AE47813F000000000000C8429834012046
:102EE000FC2301206C3D01200824012070A3012057
:102EF000183D012080340120AC340120143D012014
:102F0000A8340120B4340120DC4E0120E056012019
:102F1000F0230120143F0120CE4BCF4903EB4500A5
:102F2000DFF8B8C331F915E0B0F90C009CED008A68
:102F3000A0EB0E0EC94828EE298AC7ED00BA07EEAD
:102F400090EA0068F8EEE77A904227EE888A78EEF9
:102F50004DCABFF671AFB3F90C20B1F900E0C0481B
:102F6000AEEB020E00688EEAEE72A2EBEE728242C7
:102F70001ADAB3F90E30B1F90220D21A82EAE273FA
:102F8000A3EBE27398420FDDB64A0023128884F85F
:102F90006C31002A43F0EA85B34AB44B11781868C3
:102FA00081F0010107F040FCB14B022D334493ED59
:102FB000000A049B2CEE000A20EE2C0AA3EC010A66
:102FC000049304F02584AB4BAB4AD3ED006AD2EDF9
:102FD000007AAA4B66EEA77A97ED006A334467EE53
:102FE000A87A93ED007AA64B67EE877AD3ED005A64
:102FF000B0EE467AF1EE656AACEEA77AF4EEC76AF7
:10300000F1EE10FA01DCC5FEC76AF7EE007A94ED26
:103010004C7AB4EEE77AF1EE10FAACBF012300234C
:1030200043B1B0EEC66AF0EEE67AF4EEC67AF1EE9F
:1030300010FA01D5C7ED006A022D65D0914AB0EEB5
:103040004D0A914B52F825001B6898478F4A904BC8
:1030500052F825001B6898479AF8373023B18D4BFA
:103060001B88002B01F07180B0EE6B8A8A4B38EE22
:10307000400A334493ED008A83ED000A30EE480A9B
:103080009AF8483020EE098A002B33D0834B1B7806
:1030900013F0010300F06486F7EE007A94F86C31C7
:1030A000B4EEE7AAF1EE10FAC1F2B784002B01F0FA
:1030B000F880D4F87031059AD31A794A12689A4286
:1030C00018DD784BF0EEECCAD3ED007AF4EEE7CAE7
:1030D000F1EE10FA42F12F80624A0023128884F840
:1030E0006C31002A00F048866F494A6912B10A68BB
:1030F00013604B746D4B334493ED000A2CEE000AC1
:1031000020EE088A89ED008A94F87C3133B9049B5B
:10311000C7ED00BA43ED01BAC9ED00BA013508F1B7
:103120000408043709F10409032D06F104067FF4AD
:10313000FAAD039B1A78072A01F08484012A01F072
:103140008D870023069394F88421002A41F0FE81A4
:10315000DFF88CA1564BDAF800201968D50491F8F5
:103160002C0001F11B80534B0125534A04935B8BC8
:10317000D2ED007A07EE103AD2ED013A13464F4AEB
:10318000F8EEC75A4E4E92ED037A4E4AD6ED006ADB
:1031900037EE657AD2ED005A4B4A75EEE64A93ED6A
:1031A000025A92ED006AC4ED656AC4ED636AC4ED2B
:1031B000624AC4ED665A84F89C51444BC7EE065AE5
:1031C0000A8D93ED006A424BDFED424A93ED007A9F
:1031D0005342B7EE004A36EE076A06EE903AF8EE32
:1031E000E66A36EE276A07EE902AB8EE677AB4EE02
:1031F000E66AF1EE10FAC5FEC45AC5FEA45AC4ED43
:10320000695A01F1088386FE476A304BDFED324A86
:10321000D3ED017A2E4B26EE246A93ED014A77EE28
:10322000847A77EEA37AF4EEE76AF1EE10FA01DC25
:10323000C7FE676A254B4A8DD3ED027A53429FED54
:10324000267A75EE277A04EE903A66EE876AF8EEF3
:10325000E44A47E070A30120183D0120A834012072
:10326000B034012054C2012056C2012058C20120AE
:1032700054340120F82F012078000120603401200F
:10328000C834012000300120FC2F012054300120DF
:10329000503001206C3D01202C2401208359012055
:1032A000AC340120B83401205CC201206C34012010
:1032B000703D0120384D0120083F0120403B012096
:1032C0003CA3012040A3012060350120FC3E0120E9
:1032D000143F0120000000006F12833A8034012067
:1032E000E0560120F4EEE47AF1EE10FA05D407EE90
:1032F000102AF8EE474AC4FEE74AE84ADFEDE87ACA
:10330000527864EEA74A0AB9F1EE644A002841F007
:10331000AC85F7EE003AE34D2A78002A02F01B86CE
:10332000E1499FEDE24A91ED025A91ED017A26EED4
:10333000855AD1ED037AA6EE075AA4EEA75A23EEDA
:10334000855AB4EEC45A85FE447A8DED0A5AC5FEFC
:10335000047AF1EE10FA88BFB0EE447A012A02F046
:103360004B8691ED064AD1ED052A26EE844A91ED71
:10337000073AA6EE224AA4EE834A23EE844AB4EE2C
:10338000E74A8DED0B4AC4FE277A84FE474AF1EEE8
:1033900010FA98BFB0EE447A022A00F0AD8091EDA9
:1033A0000A4AD1ED092A26EE844A91ED0B3AA6EE9F
:1033B000224AA4EE834A23EE844AB4EEE74A8DED16
:1033C0000C4AC4FE277A84FE474AF1EE10FA98BFF1
:1033D000B0EE447A032A00F08F8091ED0E4AD1EDD1
:1033E0000D2A26EE844A91ED0F3AA6EE224AA4EE6B
:1033F000834A23EE844AB4EEE74A8DED0D4AC4FEBB
:10340000277A84FE474AF1EE10FA98BFB0EE447A6C
:10341000042A71D091ED124AD1ED112A26EE844A88
:1034200091ED133AA6EE224AA4EE834A23EE844A93
:10343000B4EEE74A8DED0E4AC4FE277A84FE474A71
:10344000F1EE10FA98BFB0EE447A052A54D091ED0F
:10345000164AD1ED152A26EE844A91ED173AA6EECA
:10346000224AA4EE834A23EE844AB4EEE74A8DED65
:103470000F4AC4FE277A84FE474AF1EE10FA98BF3D
:10348000B0EE447A062A37D091ED1A4AD1ED192AC6
:1034900026EE844A91ED1B3AA6EE224AA4EE834A18
:1034A00023EE844AB4EEE74A8DED104AC4FE277A33
:1034B00084FE474AF1EE10FA98BFB0EE447A072A2C
:1034C0001AD091ED1E4A91ED1D3A66EE846A91ED97
:1034D0001F4AE6EE036AE4EE246A66EEA36AF4EE9F
:1034E000E76ACDED116AC6FEA77AC6FEC76AF1EE9D
:1034F00010FA98BFB0EE667A77EEC77AF7EE006AF8
:10350000C4ED4C7AF4EEE67AF1EE10FA43F37C86E1
:1035100086EEA77ADDED0B7A022A27EE055A67EED2
:10352000877A8DED0A5ACDED0B7A2DD0DDED0C7A30
:10353000032A67EE877ACDED0C7A25D0DDED0D7A82
:10354000042A67EE877ACDED0D7A1DD0DDED0E7A77
:10355000052A67EE877ACDED0E7A15D0DDED0F7A6C
:10356000062A67EE877ACDED0F7A0DD0DDED107A61
:10357000072A67EE877ACDED107A05D0DDED117A56
:1035800027EE877A8DED117A4949096811F0805349
:10359000089301F0EA81F6EE005AC4ED695A002A58
:1035A00002F0F8844349D4ED667A434BFDEEE77AA6
:1035B000CE7894F99C1194ED656A1B7807EE101A89
:1035C000DFF804E117EE909ADAF80010FDEEC67A03
:1035D0003A4F03F0010801F01000394B01F4805C10
:1035E0009EED005A01F48001B7F906E0049FB8EEA1
:1035F000C77A099117EE901A1B78D4ED626AD4ED60
:10360000637A7F8B002E40F0EB87274E002841F035
:103610000F8396ED006A9DED0A5A25EE866A2948C9
:10362000A5EE076AB0EE675AA6EE265ABDEEC56A49
:1036300016EE10EA16EE107ACE45A8BF4F46714539
:10364000C8BF0F46012A06EE107AB8EEC66A80EDB2
:10365000006A00F0F68096ED046A9DED0B5A25EEA7
:10366000866AA5EE076AB0EE675AA6EE265ABDEE48
:10367000C56A16EE10EA16EE107ACE45A8BF4F4680
:103680007145C8BF0F46022A06EE107AB8EEC66A28
:1036900080ED016A00F0D58018E000BFA84001204D
:1036A0006F12833A65390120D034012000000000F8
:1036B000F43E01207C92012083590120247D0120C9
:1036C000AC7E0120303F0120CC34012096ED086A09
:1036D0009DED0C5A25EE866AA5EE076AB0EE675A94
:1036E000A6EE265ABDEEC56A16EE10EA16EE107A60
:1036F000CE45A8BF4F467145C8BF0F46032A06EE08
:10370000107AB8EEC66A80ED026A00F09A8096EDF3
:103710000C6A9DED0D5A25EE866AA5EE076AB0EE9D
:10372000675AA6EE265ABDEEC56A16EE10EA16EEE8
:10373000107ACE45A8BF4F467145C8BF0F46042A30
:1037400006EE107AB8EEC66A80ED036A79D096ED7F
:10375000106A9DED0E5A25EE866AA5EE076AB0EE58
:10376000675AA6EE265ABDEEC56A16EE10EA16EEA8
:10377000107ACE45A8BF4F467145C8BF0F46052AEF
:1037800006EE107AB8EEC66A80ED046A59D096ED5E
:10379000146A9DED0F5A25EE866AA5EE076AB0EE13
:1037A000675AA6EE265ABDEEC56A16EE10EA16EE68
:1037B000107ACE45A8BF4F467145C8BF0F46062AAE
:1037C00006EE107AB8EEC66A80ED056A39D096ED3D
:1037D000186A9DED105A25EE866AA5EE076AB0EECE
:1037E000675AA6EE265ABDEEC56A16EE10EA16EE28
:1037F000107ACE45A8BF4F467145C8BF0F4606EEAA
:10380000107A072AB8EEC66A80ED066A19D096EDDE
:103810001C6A9DED115A65EE865AE7EE055AE6EEF2
:10382000A57AFDEEE77A17EE906AB145A8BFB146DA
:10383000B142D8BF494607EE901AF8EEE77AC0EDDC
:10384000077AB8F1000F00F0D887CD4A1268002A35
:1038500040F09386CB4A127892B1287868B1CA4F6B
:103860000026DFF84883F0B2D8F80030B7EC010A40
:103870000136984728788642F5DBC44A126890479B
:10388000039B1A78072A01F0CD804FF00009DAF87F
:103890000020550500F1C387BD4B1B78BBB1BD4A65
:1038A000049BB2F906205B8B9A4210DCBA4B1B7862
:1038B000012B01F0F383192B01F0F0830E2B06D0BE
:1038C000082B04D00023B54AC4F84031936094F823
:1038D000AE5125B1B24B1B88980741F0A48394F8F0
:1038E000B451002D40F0A687049B9E7F002E00F06F
:1038F000F085022E01F0E482032E41F0DD8293F880
:103900002030C3EB431203EB8203DB009BB2049A2B
:10391000D77F0237FFB2002B00F03786002D00F072
:103920003486A04A1668B3FBF6F31EB2A4F8E4612D
:10393000B7B307EE906AF7EE005A984A012FB8EE37
:10394000E76AD4ED7E6AD2ED007A85EE867A77EE6C
:10395000E67A67EE877AC4ED7A7A21D0D2ED017AE1
:10396000022FD4ED7F6A77EEE67A67EE877AC4EDB0
:103970007B7A15D0D2ED027A032FD4ED806A77EEF0
:10398000E67A67EE877AC4ED7C7A09D0D2ED037AC5
:10399000D4ED816A77EEE67A67EE877AC4ED7D7AB8
:1039A000039B1B78092B03F06082002E40F3938564
:1039B000002F02F02F8294ED7E7A012FD4ED7A7AD7
:1039C000764A77EE877AC4ED7E7AC2ED007A21D00E
:1039D00094ED7F7A022FD4ED7B7A77EE877AC4ED6F
:1039E0007F7AC2ED017A15D094ED807A032FD4ED61
:1039F0007C7A77EE877AC4ED807AC2ED027A09D0BC
:103A0000D4ED817A94ED7D7A77EE877AC4ED817A70
:103A1000C2ED037A013F022FB8BF0227FBB2079322
:103A2000002D079D18BF02255F4BB0EE007A039969
:103A30001B6808781978DFED626A07EE901A9978AA
:103A4000F8EEE77A67EEA67AF4EEC77AF1EE10FAAE
:103A500040F3DD8637EEC77ADFED566AB0EE676A6F
:103A6000A7EE266AF0EE466A9FED536A92ED007A61
:103A700027EE067AB0EEC76A84ED557A84ED586A6F
:103A800099B105EE901A9FED4E4A67EE074AB8EEDF
:103A9000E55AF7EE005A64EE864A25EE045A75EEB2
:103AA000C55AE4EE855A27EE257ADFED445A5F7950
:103AB00066EEA56A26EE877ACFB19FED415A06EEF3
:103AC000907ADFED405AF8EEE66A26EE056A26EEB9
:103AD000266AB4EEE56AF1EE10FA01F3BE81F7EE64
:103AE000005A35EEC66AC5EE866A27EE267A0C289D
:103AF00000F07D879FED348ADFED346A87FE488AC7
:103B000088FE268A84ED4E8A002D00F0F380B0EE08
:103B1000007AF4EEC77AF1EE10FA05DD37EEC77AD7
:103B2000DFED246AE7EE267A92ED017ADFED226A74
:103B300027EE267AF0EEC75A84ED567AC4ED595A2C
:103B400099B106EE901ADFED1E4A27EE075AF8EEFD
:103B5000E66AB7EE006A25EE255A66EEA46A36EEEE
:103B6000666AA5EE266A27EE067ADFED146A997971
:103B700067EEA67A67EE877A00293FD028E000BF7B
:103B8000A05B0120F48F0120303F0120A87E01209E
:103B9000DC000120247D0120A8400120403B0120C1
:103BA0006C3D0120A4400120743D0120A07E012035
:103BB0000000C842D7A368416F12033B000048438E
:103BC0000AD7233CA4707D3F00C0F94400C0F9C46B
:103BD00007EE101A1FED066AF8EEC76A1FED077AA6
:103BE00066EEA56A66EE866AF4EEC76AF1EE10FA32
:103BF00041F325811FED127A67EE877A0C2800F0D9
:103C0000D9865FED0F6A012D1FED107AC7FEE67AA7
:103C1000C7FE877AC4ED4F7A6CDD5978B0EE007A32
:103C20005FED196A07EE901A597AF8EEE77A67EEB7
:103C3000A67AF4EEC77AF1EE10FA05DD37EEC77A10
:103C40005FED246AE7EE267A92ED027A5FED266A4E
:103C500027EE267AB0EEC75A84ED577A84ED5A5A89
:103C600099B106EE901A5FED2A4AF7EE005AB8EEC7
:103C7000E66A67EE076A26EE246A66EE856A75EEE6
:103C8000C65AE6EE865A27EE257A5FED346ADB796E
:103C900067EEA67A67EE877AFBB107EE103A1FED62
:103CA000386AF8EEC76A1FED397A66EE856A66EE05
:103CB000866AF4EEC76AF1EE10FA01F3D280F5EEEF
:103CC000C06AF1EE10FA02F16283B7EE006A76EE96
:103CD000666A86EE267A67EE877A0C2800F07F8681
:103CE0005FED476A1FED477AC7FEE67AC7FE877A1F
:103CF000C4ED507A092800F02B86049B93F82150DC
:103D0000002D40F0F385002384F8B431C14B1B68CB
:103D1000980609D5C04B1B8803F0300323B1BF4B75
:103D20001B78D90702F1A28018F024FC002840F08B
:103D3000E683BB4B1B7823B9BA4B9B78002B41F031
:103D40006D81039B1D78072D7EF49FAF06F008FA66
:103D5000039BA0EB09001D78B34BD880FEF795BFFD
:103D600094F86C21002A3FF4C5A9B04A84F86C315C
:103D70001288002A7FF4B8A9AD4AAE4B11781868B2
:103D800081F0010106F050FDFFF7B4B9AA4A11789D
:103D9000D4F81871A94BFE009FEDA97A9A1982ED0B
:103DA000007A002974D0B0EE476AA648F0EE476A60
:103DB00000220132F0EC017A05EE902A67EEA77A34
:103DC0009142F8EEE55A87FE277A76EEA76AA7EECB
:103DD000A56AEED1F5EEC06A9A1982ED007AF1EE8D
:103DE00010FA55DDC6EE265A9749984AD1ED007A69
:103DF0001188B7EE007A75EEC75A65EEA77AFDEE28
:103E0000E77A17EE902A812A42F32F828A42A8BFCE
:103E10000A4607EE902AF8EEE77AF0198C4A02EB90
:103E2000800292ED007A92ED056A92ED015AA7EEBA
:103E3000276AD2ED066A92ED047AE5EE276AD2EDA2
:103E4000034A92ED025A27EE467ABDEEC64AE6EEE6
:103E5000646AA5EE277A14EE100A8128C2ED056A7D
:103E600082ED067A42F3FE818142A8BF014607EE49
:103E7000901AF8EEE77AFCEEE77ACDED067ABDF817
:103E8000182099198A801FB9BEF1130F03F0A6817B
:103E9000BEF1150F41F067821E44D4F81451624BF5
:103EA000B28823F8172001356A4981FB0531EA17EA
:103EB0002944C2EBA102C2EBC202AD1AC4F81451EC
:103EC000D4F81C216448059B01689A1A634DC4F814
:103ED0001C3111442D780160002D40F0D38007EE95
:103EE000902A5F4EDFF89891B8EEE78A06F24475A3
:103EF00006F5F6685B4FF6EC017A28469BED080A5A
:103F0000F8EEE77ADBF8703727EE800A9847A5F1DC
:103F1000E000DBF890369847A5F17000DBF8003739
:103F200024359847D6F85006DBF8B0309847D7EDDF
:103F3000007AA845A9EC010AE0EE087AE7EC017ADC
:103F4000D9D1039B1D78072D7EF498AE06F008F9B1
:103F5000059A354B801A039A18801578FEF78EBEA5
:103F6000B1F90020B1F9021082EAE27394ED587AB7
:103F7000D4ED596AA3EBE27381EAE17286FE876AA7
:103F8000A2EBE17238499342B8BF13460A7807EEB4
:103F9000103AB8EEC77A27EE297A002A40F0588105
:103FA000324BD3ED005AF4EECB5AF1EE10FA41F158
:103FB0001A80B7EE005ADFED2E6ADFED2E4A36EE9C
:103FC000C77A2D4B35EE655AD3ED006A25EE245A9B
:103FD000E7EE055A65EEA65AF5EEC05AF1EE10FA74
:103FE00040F2BF84CAEEA56AB7EE007AF0EE475AF7
:103FF000E6EE665AC5FEC76AC6FEAB6A1F4B93ED76
:10400000007A67EE877AA7EEA68AFEF7EEBE012257
:10401000FEF74CBE143D01206C3D01206E3D012099
:10402000C73701209E4501208839012054C2012054
:1040300056C2012058C20120B6400120AC430120E5
:1040400000000000B8220120B8400120B440012047
:10405000D442012093244992BC2F0120AA40012080
:104060000C4F0120C02F01208C34012094340120FA
:1040700000003443610BB63B8834012084340120B6
:10408000D45601209C4B07EE902A9C4D00270493A8
:1040900099469B4BF8EEE78A069405F2D466DFF862
:1040A000AC821C46039B1B78172B69D095ED007AD8
:1040B000082BDBED087AB8EEC78A28EE278A07D1ED
:1040C000B0EE480A07932FF09FF9079BA9F800006C
:1040D000DAF8002092000BD5002F03F0D583B0EE64
:1040E000480ADBF8703706F170009847B0EE408A56
:1040F000B0EE480ADBF89036A6F170009847DBF87E
:10410000003730469847039BB0EE408A1B78032B5C
:1041100031D0D5F85406B0EE480ADBF8B03001379C
:104120009847D8ED007A032F06F12406E0EE287AAE
:1041300009F10209A4EC010A05F10405E8EC017A91
:10414000B0D1039B069C1D78FDE66E4BF7EE006A2E
:104150006D4A3344D2ED007A93ED007A6B4B67EEF3
:10416000277A93ED007AC7FEE67A67EE877A27EE24
:10417000888AFEF77BBF2FF047F9A9F80000C8E74F
:1041800095ED007A0BEB4702DBED087AB8EEC78AB3
:10419000928FA9F8002028EE278A99E75C4B1A78BD
:1041A0005C4BD207049302D41A8BA4F890215A4D89
:1041B0005A4A2D88D2ED037A07EE105AB8EEC77A24
:1041C000F4EEC77AF1EE10FA41F2E485544A13880E
:1041D00007EE103AB8EEC77AF4EEC77AF1EE10FAAD
:1041E000C0F268874F4A504D92ED006AD5ED006AE3
:1041F00094F99C2176EE665AC4ED656A012AC4EDF5
:10420000636A84ED666AC4ED625A01F07784059BA7
:104210000025C4F8A03137EEC77A0127FCEEE77A13
:10422000424E84F89C7184ED697A17EE902A96EDDF
:10423000006AA4F890213E4A954241F298853D4B90
:10424000D3ED007AD3ED013A93ED025AFEF7B5BFF4
:10425000394BD3ED005AF5EEC05AF1EE10FA40F3A7
:104260008083364B93ED005AB5EEC05AF1EE10FA4A
:1042700040F3778326EE6A6A35EE477AF7EE004A16
:10428000C6EE256A87EE056A76EEA46A86FE646A43
:1042900086FE2B6A66EE266AC6FEE46AC6FEAB6A36
:1042A000ACE6274AF0EEC87A92ED007AF4EEC77ACF
:1042B000F1EE10FA7EF71EAF224AF0EEEC7A92EDA4
:1042C000007AF4EEC77AF1EE10FA7EF713AFD8ED6C
:1042D000007A1D4AF0EEE77A92ED007AF4EEC77AA2
:1042E000F1EE10FA7EF506AF0122059984F86C21F3
:1042F000C4F87011FEF7E1BE883901200C4F01208F
:10430000D4560120182401207C3401207834012067
:1043100083590120384D012064350120403B0120A4
:104320006635012040A30120503501206C35012065
:104330008FD00300083F01208834012090340120F1
:10434000BC340120B8340120C0340120C02F01202A
:10435000924B4FF47A76924D1A680693914B92489D
:10436000039304951D788E4B4778B3F90600B6FB8E
:10437000F2F2C2EB421602EB8602D600B6B2B442AB
:1043800001F07787DBF88030BBF93CC0DBF86420B4
:10439000591C07EE90CA62440129F8EEE77ACBF87F
:1043A0008010CBF8642001F071879BED1C5A07EE5A
:1043B000101ADBED1E6A012C77EEC55AB8EEC76AFB
:1043C00085EE867A37EE057A77EEC77A8BED1D7A21
:1043D0008BED1C7AE7EEA56AF0EE667ACBED1F6AEC
:1043E000CBED1E6A02F00C82DBF89430BBF93EC0C4
:1043F000DBF86820591C07EE90CA62440129B8EE28
:10440000E77ACBF89410CBF8682001F05A879BED3F
:10441000215A07EE901ADBED236A012C77EE455AFC
:10442000B8EEE76AC5EE867A77EE857A37EE677A78
:10443000CBED227ACBED217AF0EE667AE7EE257AA3
:10444000CBED247ACBED237A02F05B83DBF8A83046
:10445000BBF940C0DBF86C20591C07EE90CA6244DF
:104460000129B8EEE77ACBF8A810CBF86C2001F060
:1044700043879BED265A07EE901ADBED286A012C44
:1044800077EE455AB8EEE76AC5EE867A77EE857A1A
:1044900037EE677ACBED277ACBED267AF0EE667AA7
:1044A000E5EE877ACBED297ACBED287A02F01D83F1
:1044B0003B4B3E4CD880BBF8AC20039B013A1D78A7
:1044C000ABF8AC20002206994A608A60CA60FEF709
:1044D000D2BBA4F8E461002D3FF418AC0225344AA5
:1044E000FFF7A2BA334B344A196812882C4BC969BA
:1044F0005A80198013B0BDEC0C8BBDE8F08F2F4CA7
:1045000017F032FF6378022B00F0BA85032B7FF49B
:1045100010AC41F2B813E35C002B41F0E08241F2B1
:10452000A403E35C002B41F0E48241F2E803E35C86
:10453000002B41F0D98241F22C13E35C002B3FF4B5
:10454000F8AB1F4821F0C8F9FFF7F3BB1D4B1E4D18
:104550001A7812F0010F2A7840F0888222B1920076
:104560001A491B482EF079FD1A4A1B4B1268DFF8D6
:104570006CA00493002A3FF46DA91FF0DDFBFFF748
:1045800069B9084B094C03939AE4B4F8E461013E1D
:1045900036B2A4F8E461FFF708BA00BFD056012094
:1045A0008839012084390120BC560120B82201201D
:1045B000403B0120A4A201205E2A0120645F01206B
:1045C0009070012083590120653901203429012090
:1045D000303F0120A05B0120384D0120E056012032
:1045E000002801F03881B8F1000F42F0CF82E24E8E
:1045F000002B42F02C81BDEEC56A9DED0A5ADF48C2
:1046000016EE101A96ED006A25EE866AA5EE076A88
:10461000B0EE675AA6EE265ABDEEC56A16EE10EA4F
:1046200016EE107ACE45A8BF4F467145C8BF0F465B
:10463000012A06EE107AB8EEC66A80ED006A00F034
:10464000DF8096ED046A9DED0B5A25EE866AA5EE95
:10465000076AB0EE675AA6EE265ABDEEC56A16EE98
:1046600010EA16EE107ACE45A8BF4F468E45B8BF69
:104670000F46022A06EE107AB8EEC66A80ED016A8D
:1046800000F0BE8096ED086A9DED0C5A25EE866A14
:10469000A5EE076AB0EE675AA6EE265ABDEEC56AC9
:1046A00016EE10EA16EE107ACE45A8BF4F468E459C
:1046B000B8BF0F46032A06EE107AB8EEC66A80ED40
:1046C000026A00F09D8096ED0C6A9DED0D5A25EE74
:1046D000866AA5EE076AB0EE675AA6EE265ABDEEC8
:1046E000C56A16EE10EA16EE107ACE45A8BF4F4600
:1046F0008E45B8BF0F46042A06EE107AB8EEC66A99
:1047000080ED036A7CD096ED106A9DED0E5A25EE81
:10471000866AA5EE076AB0EE675AA6EE265ABDEE87
:10472000C56A16EE10EA16EE107ACE45A8BF4F46BF
:104730008E45B8BF0F46052A06EE107AB8EEC66A57
:1047400080ED046A5CD096ED146A9DED0F5A25EE5B
:10475000866AA5EE076AB0EE675AA6EE265ABDEE47
:10476000C56A16EE10EA16EE107ACE45A8BF4F467F
:104770008E45B8BF0F46062A06EE107AB8EEC66A16
:1047800080ED056A3CD096ED186A9DED105A25EE35
:10479000866AA5EE076AB0EE675AA6EE265ABDEE07
:1047A000C56A16EE10EA16EE107ACE45A8BF4F463F
:1047B0008E45B8BF0F46072A06EE107AB8EEC66AD5
:1047C00080ED066A1CD096ED1C6A9DED115A65EECF
:1047D000865AE7EE055AE6EEA57AFDEEE77A17EE81
:1047E000906AB145A8BFB146B142D8BF494607EE6D
:1047F000901AF8EEE77AC0ED077A002A3FF425A870
:1048000092005F495D482EF028FCFFF71EB8F0EEDD
:10481000676AFFF729B9B0EE666AFEF7F6BCDBF807
:104820000830002B3FF438A85649A1F150009847B2
:10483000FFF732B8544B44F62061544AD3F8EC30B9
:1048400012688B42A8BF0B46B3F57A7FB8BF4FF40E
:104850007A7312F0100FDAF800209BB2A4F8B63188
:1048600000F02384D20441F12886494A17687E8EDD
:10487000760848486421484AA0FB0303D4F8B801ED
:10488000D2ED037A9A09431CBDEEE77A04EB4000AF
:10489000C4F8B83191FBF2F2142A17EE10EAA8BF5F
:1048A0001422A0F8BCE1934203DB00221346C4F8B3
:1048B000B82104EB4303B3F9BC3107EE103AB8EE6C
:1048C000C77A77EEC77AFDEEE77ACDED067ABDF9C5
:1048D000182082EAE273A3EBE273B34201F360872C
:1048E0004FF07E532D4A1360FEF7FEBF1E2127486E
:1048F00008F0FAFB00283FF406AA294B1B885E0645
:104900003FF501AA94F80832AB4242F0DF82234B14
:10491000D4ED837AD3ED016A94ED505A28EE277ACC
:10492000DFED235A67EEC57A9FED1E6AA5EE267A63
:10493000E8EE267A87FE657A87FE067A84ED507A5D
:10494000C7FEE57AC7FE867AC4ED4E7AFFF7DBB97B
:10495000FDEEC87A144A968017EE903AD380FFF79E
:10496000CCB9DFED126AFFF749BBDAF800104B0251
:104970003EF511AEFEF713BED0340120303F0120CA
:10498000342901202C4F012058170120F43E01202A
:10499000703D0120D34D6210403B01207800012082
:1049A0006C3D012000C0F9C48839012000000000DE
:1049B00000C0F944BDEEE77A5FED036A9449012D2A
:1049C000C7FEE67A17EE107A9FED927A4F80C7FE07
:1049D000877AC4ED4F7A3FF720A9FFF78EB9BDEE75
:1049E000E77A8B4A17EE103A9380FFF779B9FDEE1C
:1049F000C76A9FED898A864F87FE488A16EE90EA3D
:104A0000DFED846AA7F800E088FE268A84ED4E8AEE
:104A1000002D7FF47CA8FFF770B9002B3EF46AAB41
:104A2000FEF747BB05F09CFB069B7949C01A039B28
:104A30001A788880072A7EF428AF05F091FB81461A
:104A4000FEF725BF05F08CFB039A099B1278C01A6C
:104A50006F4B012A0493588000F00283072A7EF4EA
:104A600070AB05F07DFB0690FEF76DBB002A3FF4AE
:104A70007BADD4ED593AF3EE046A94ED586AD4ED67
:104A8000637AF4EEC63A654937EEA65A94ED627A37
:104A9000D1ED005AF1EE10FA94ED564AD4ED554A94
:104AA0005F4E604800F1568396ED026AF0EE674A69
:104AB00026EE446AE6EE074AF4EEC54A34EEE66AAC
:104AC000F1EE10FA48BFB0EE656A012A80ED006A87
:104AD0003FF44AAD96ED066AF0EE674A26EE446A68
:104AE000E6EE074AF4EEC54A34EEE66AF1EE10FA55
:104AF00048BFB0EE656A022A80ED016A3FF434AD2A
:104B000096ED0A6AF0EE674A26EE446AE6EE074A38
:104B1000F4EEC54A34EEE66AF1EE10FA48BFB0EEA4
:104B2000656A032A80ED026A3FF41EAD96ED0E6AB7
:104B3000F0EE674A26EE446AE6EE074AF4EEC54A0E
:104B400034EEE66AF1EE10FA48BFB0EE656A042A68
:104B500080ED036A3FF408AD96ED126AF0EE674A05
:104B600026EE446AE6EE074AF4EEC54A34EEE66AFB
:104B7000F1EE10FA48BFB0EE656A052A80ED046ACE
:104B80003FF4F2AC96ED166AF0EE674A26EE446A00
:104B9000E6EE074AF4EEC54A74EEE66AF1EE10FA64
:104BA00048BFF0EE656A062AC0ED056A3FF4DCAC4A
:104BB000D6ED1A6AF0EE674AB3EE046A66EEC46A8E
:104BC000E6EE874AF4EEC54A74EEC66AF1EE10FAD4
:104BD00048BFF0EE656A072AC0ED066A3FF4C4AC30
:104BE000D6ED1E6A104B26EEC44ADFF840A00493AF
:104BF000E4EE077AB4EEE75A77EEC67AF1EE10FAF1
:104C0000C8BFF0EE657AC0ED077AFEF71EBE00BFA2
:104C10008839012000C0F9C400C0F944CC34012017
:104C2000D0340120303F0120384D0120E0560120D2
:104C3000B8F1000F41F00E8296ED006A9DED0A5A20
:104C400025EE866AEA48A5EE076AB0EE675AA6EE38
:104C5000265ABDEEC56A16EE10EA16EE107ACE455B
:104C6000A8BF4F467145C8BF0F46012A06EE107A0D
:104C7000B8EEC66A80ED006A3FF4C2AD96ED046AF4
:104C80009DED0B5A25EE866AA5EE076AB0EE675ACF
:104C9000A6EE265ABDEEC56A16EE10EA16EE107A9A
:104CA000CE45A8BF4F467145C8BF0F46022A06EE43
:104CB000107AB8EEC66A80ED016A3FF4A1AD96EDB8
:104CC000086A9DED0C5A25EE866AA5EE076AB0EEDD
:104CD000675AA6EE265ABDEEC56A16EE10EA16EE23
:104CE000107ACE45A8BF4F467145C8BF0F46032A6C
:104CF00006EE107AB8EEC66A80ED026A3FF480AD27
:104D000096ED0C6A9DED0D5A25EE866AA5EE076AB2
:104D1000B0EE675AA6EE265ABDEEC56A16EE10EA48
:104D200016EE107ACE45A8BF4F467145C8BF0F4654
:104D3000042A06EE107AB8EEC66A80ED036A3FF4E4
:104D40005FAD96ED106A9DED0E5A25EE866AA5EED2
:104D5000076AB0EE675AA6EE265ABDEEC56A16EE91
:104D600010EA16EE107ACE45A8BF4F467145C8BF6F
:104D70000F46052A06EE107AB8EEC66A80ED046A80
:104D80003FF43EAD96ED146A9DED0F5A25EE866A0E
:104D9000A5EE076AB0EE675AA6EE265ABDEEC56AC2
:104DA00016EE10EA16EE107ACE45A8BF4F467145B2
:104DB000C8BF0F46062A06EE107AB8EEC66A80ED26
:104DC000056A3FF41DAD96ED186A9DED105A25EE6B
:104DD000866AA5EE076AB0EE675AA6EE265ABDEEC1
:104DE000C56A16EE10EA16EE107ACE45A8BF4F46F9
:104DF0007145C8BF0F46072A06EE107AB8EEC66A9C
:104E000080ED066A3FF4FCAC96ED1C6A9DED115AEC
:104E100065EE865AE7EE055AE6EEA57AFDEEE77AEC
:104E200017EE906AB145A8BFB146B142C8BF8946E6
:104E300007EE909AF8EEE77AC0ED077ADDE4F5EE3A
:104E4000C06AF1EE10FA01F1A682B7EE006A76EEC2
:104E5000666A86EE267AFEF7CFBEDFED666AFEF75B
:104E600044BE9FED647AFEF736BF63494A79002A53
:104E70003EF44FAA614A1278002A3EF44AAA0B78FF
:104E800007EE902A5E4AB7EE005A07EE103AF8EEA7
:104E9000E77A1288B8EE477A9FED5A4A67EE277A8A
:104EA00007EE102AB8EE477AC7EE873AC3FEC43A37
:104EB000C3FE853AFEF72FBA534B5B88FEF727BD3A
:104EC000B4F8B63103F57A739BB2FEF720BD07EE56
:104ED000102A1A78F7EE006A4C4BB8EEC77A002118
:104EE000132A0493C4F80C1186EE879AB3F90400D0
:104EF000B4F810619BED080A01F06482444A454908
:104F000067EE897AD2ED006A29EE088A92ED053AB9
:104F100069EE288A92ED097AD2ED0E3AA6EEA73A0A
:104F200092ED174A01EB8605D2ED126AE7EE083AD8
:104F3000D2ED064A2F4692ED017AA6EEA84A92EDEE
:104F40000A6AD2ED0F5AE7EE274AD2ED186A92EDBF
:104F5000137AE6EE085A92ED045AE7EE286A92EDCB
:104F60000D6A92ED167A25EE435A92ED032A26EE4B
:104F7000636AD2ED022A27EE447AD2ED0C1AE2EEF1
:104F8000434AA2EEA75A92ED0B2AD2ED152AE1EE82
:104F9000E35AD2ED147AA2EE086AE2EEC46A85ED15
:104FA000003AA7EEA87A0025C2ED054A82ED065A1E
:104FB000C2ED0E5AC7ED203A82ED0F6A87ED404AE6
:104FC000C2ED176A82ED187AC4F80051C4F8045192
:104FD000C4F80851721C9880039B02F01F02A4F8C9
:104FE0001021FDF72EBE0C4BD3ED005AFEF7F4BF97
:104FF000303F01200000C842043D01203E3B01201B
:10500000383B0120713DAA3F543E012088390120E0
:1050100040430120D440012088340120059825F028
:10502000CFFDFEF78EBED74B9FEDD77AD3ED087A32
:10503000F4EEC77AF1EE10FA00F2F6849FEDD37A1F
:10504000D34AD2ED037A77EE877AC2ED037AFEF780
:1050500046BC05F085F80990FDF72FBECD4B0493B3
:1050600005F07EF8D4F88021CB49821A0690C4F866
:105070008001096804988280521AC280FEF763B8E2
:10508000A378072B3EF655AEDFE813F07A054D0600
:1050900092054206DF05C805D2057605BF4A927B18
:1050A000002A7EF414ACFEF709BCD1003FF5DAAB60
:1050B000FEF71ABCB4F89021AA4240F2FF8494F89B
:1050C000A851002D40F06C87B54AB64E92ED007A9B
:1050D000D6ED007A94F99C2177EE676AC4ED657A83
:1050E000012AC4ED637A84ED667AC4ED626A02F047
:1050F0008580059BC4F8A031DFEDA47A0122AA4E79
:10510000B0EE677AC4ED697A96ED006A84F89C2166
:10511000FFF791B8A54B1B88002B40F01B85A44AD4
:10512000A44B1178186805F07FFBD4F87021059B1B
:105130009A1AFDF773BED8ED007A9F4BF0EEE77A2E
:1051400093ED007AF4EEC77AF1EE10FA7DF7D2AF64
:10515000FDF7C2BF96ED016AB0EE674A26EE646ABB
:10516000A6EE074AB4EEC54A34EE666AF1EE10FACE
:1051700048BFB0EE656A012A80ED006A3FF4F4A9E9
:1051800096ED056AB0EE674A26EE646AA6EE074A17
:10519000B4EEC54A34EE666AF1EE10FA48BFB0EEDE
:1051A000656A022A80ED016A3FF4DEA996ED096A7C
:1051B000B0EE674A26EE646AA6EE074AB4EEC54A28
:1051C00034EE666AF1EE10FA48BFB0EE656A032A63
:1051D00080ED026A3FF4C8A996ED0D6AB0EE674A09
:1051E00026EE646AA6EE074AB4EEC54A34EE666A55
:1051F000F1EE10FA48BFB0EE656A042A80ED036A4A
:105200003FF4B2A996ED116AB0EE674A26EE646AE1
:10521000A6EE074AB4EEC54A34EE666AF1EE10FA1D
:1052200048BFB0EE656A052A80ED046A3FF49CA988
:1052300096ED156AB0EE674A26EE646AA6EE074A56
:10524000B4EEC54A74EE666AF1EE10FA48BFF0EEAD
:10525000656A062AC0ED056A3FF486A9D6ED196A8B
:10526000B0EE674AB3EE046A66EEE46AA6EE874AD9
:10527000B4EEC54A74EE466AF1EE10FA48BFF0EE9D
:10528000656A072AC0ED066A3FF46EA9D6ED1D6A6D
:105290004A4B66EEE44ADFF830A10493E4EE877AE5
:1052A000F4EEC57A77EEC67AF1EE10FAB8BFF0EEFA
:1052B000657AC0ED077AFEF7C8BA414ED4ED017A9F
:1052C000B0EE006AD4ED005AF6EE006A77EEA77AE7
:1052D00032887169561EB0EE664AB0EE677A1031B8
:1052E000D5EE867A04EBC602A5EE867A083A67EE1A
:1052F000A67A27EE267AC4ED217A84ED207A314C05
:10530000274604F1800092ED036A013ED7ED036A5F
:10531000A2F1080292ED047A07F1080776EEC65A68
:10532000D7ED007A11ED015A76EE266A77EE674ADC
:1053300011ED026A77EE277A01F10801B0EE657A85
:1053400000F10800E6EE247AA5EE247AE5EE267A4E
:10535000A6EE667A67EE847A27EE047AC0ED007ACC
:1053600080ED017ACFD1BEF1140F7EF49CAD04F034
:10537000F7FE049BD4F81451C01A064B5880FEF770
:1053800092BD00BF942F01208FC2753C0000000029
:10539000403B012088390120A44001200C4E01200F
:1053A00040A30120503501206C35012054C201205A
:1053B00056C2012058C20120C0340120384D0120BE
:1053C000BC400120B8220120E0560120D4F81891F9
:1053D000B4F810C1E54ACCF120030CEB4917DBB25D
:1053E00002EB87079E0801F00487013607F11002DF
:1053F000DF483601DF4907EB060812ED025A10328A
:1054000010ED027A103152ED075A103050ED077A44
:1054100025EE075A12ED056A12ED087A65EEA75AD5
:1054200050ED056A904550ED087A66EE266A01ED6A
:10543000065A67EE277A41ED075A41ED056A41EDBC
:10544000087ADAD1103ECC48374400EB0608A1199F
:1054500013F0030209D0B7EC017A013AF8EC017AB3
:1054600067EE277AE1EC017AF5D1BCF1000F3FF449
:105470007AAF9F00BD4B5FEA9C0600EB070803EB89
:10548000C919274402F05680013609F1100208F1CB
:10549000100007F11001330109EB030612ED025A67
:1054A000103210ED027A103152ED075A103050EDE3
:1054B000077A25EE075A12ED056A12ED087A65EEB5
:1054C000A75A50ED056A964250ED087A66EE266AB4
:1054D00001ED065A67EE277A41ED075A41ED056A5C
:1054E00041ED087ADAD1A3F11006B14408EB0600C9
:1054F00037441CF0030C3FF436AFB9EC017ABCF131
:10550000010CF0EC017A67EE277AE7EC017AF4D12E
:1055100029E7DFF8749299F800108F0801F0B3873B
:1055200007F10108954E4FEA481806F12002A6F14E
:10553000700006EB080C52ED077A203252ED0D6A2E
:10554000103012ED0B7A27EEA76A52ED097A66EE5B
:10555000A66A52ED105A27EE077A67EEA77A52ED47
:105560000E4A12ED0C5AA5EEA56A52ED0A5AE4EE67
:10557000A46AA5EE057A9445E5EEA57AF1EEC65A41
:10558000B1EEE66AF1EEC76AB1EEE77A40ED085A8D
:1055900000ED076A40ED066A00ED057ACBD1A8F16F
:1055A000200204EB0717324411F0030010D0083238
:1055B00052ED017A013812ED027A02F1080267EE2B
:1055C000A77AE7EE077AB1EEE77AA7EC017AEFD196
:1055D000BEF1140F01F092860135C4F81451FEF7A4
:1055E000D7BB674E328873684FEA520904EB8205D5
:1055F0004FEA8901D20804EB010E00F0A180501C93
:1056000010310EF110025B4F0EEB001C294403F128
:10561000100E05F1100050ED047A103217ED047AE7
:105620000EF1100E12ED085A103751ED041A37EE34
:10563000271A11ED032A77EE670A50ED034A75EE3B
:10564000218A50ED023A71EEC51A11ED026A10304E
:1056500011ED017A103150ED055A52ED072A52ED45
:10566000066A52ED057A32EE828A17ED074A36EE67
:10567000860A17ED063A72EE622A17ED055A34EEE5
:10568000249A07ED081A74EE644A33EE231A37EEB3
:10569000874A07ED079A35EE252A07ED061A77EEB9
:1056A000677A33EE631A07ED052A76EE666A02ED35
:1056B000054A75EE655A42ED088A02ED078A02ED49
:1056C000060A94451EED077A1EED086A64EE873AD5
:1056D00027EE603A26EE624A21EE865AA4EE863A1A
:1056E000F0EE634AA2EE875AE0EE864AB0EE446AD4
:1056F00000ED073AA1EE876A40ED084A01ED075A2E
:1057000001ED086A1EED057A1EED066A65EE873A20
:1057100027EE414A66EE674A26EE865AA5EE864A8D
:10572000E1EE063AE6EE874AA7EE875A40ED063AE2
:1057300000ED054A41ED064A01ED055A7FF46BAFD5
:105740001FFA89F91A460F48494621F04FFA726844
:105750004946284621F04AFA039B1A78142A3FF456
:1057600006AED4F81451FEF79EBB00BFD440012012
:1057700064420120C8220120544201203823012024
:10578000BC400120B8220120B6400120DE4EDF4897
:10579000B268B1892CF0ECF9039B93F800E0BEF1FC
:1057A000140F01F0BA85D4F814510135C4F814511E
:1057B00084E5D4F81811D648CA00D64BD64D10440B
:1057C0000A441968838805EB8205A3F1640200EEA0
:1057D000103A2846D5F81490C82AB8EEC07AB8EE28
:1057E000400AD5F81880A8BFC822EF692E6A782A27
:1057F000B8BF782207EE902AF8EEE77A77EE670ACC
:1058000077EE876A67EE877A20EEA67AC7EE870A78
:105810001AF088FC039BC5F8149093F800E0C5F8D3
:105820001880BEF1140FEF612E6201F0F984D4F8F4
:105830001821BA490132D4F8145181FB0213013501
:10584000A3EBE279C4F8145109EB4903A2EB030975
:10585000C4F81891BCE5B24E002B40F03486BDEE82
:10586000C56A9DED0A5AAF4816EE101A96ED006A09
:1058700025EE866AA5EE076AB0EE675AA6EE265AAE
:10588000BDEEC56A16EE10EA16EE107ACE45A8BF38
:105890004F467145C8BF0F46012A06EE107AB8EE92
:1058A000C66A80ED006A3DF4CCAF96ED046A9DEDCA
:1058B0000B5A25EE866AA5EE076AB0EE675AA6EE89
:1058C000265ABDEEC56A16EE10EA16EE107ACE45DF
:1058D000A8BF4F468E45B8BF0F46022A06EE107A83
:1058E000B8EEC66A80ED016A3DF4ABAF96ED086A8A
:1058F0009DED0C5A25EE866AA5EE076AB0EE675A52
:10590000A6EE265ABDEEC56A16EE10EA16EE107A1D
:10591000CE45A8BF4F468E45B8BF0F46032A06EEB8
:10592000107AB8EEC66A80ED026A3DF48AAF96ED51
:105930000C6A9DED0D5A25EE866AA5EE076AB0EE5B
:10594000675AA6EE265ABDEEC56A16EE10EA16EEA6
:10595000107ACE45A8BF4F468E45B8BF0F46042AE1
:1059600006EE107AB8EEC66A80ED036A3DF469AFC0
:1059700096ED106A9DED0E5A25EE866AA5EE076A31
:10598000B0EE675AA6EE265ABDEEC56A16EE10EACC
:1059900016EE107ACE45A8BF4F468E45B8BF0F46CB
:1059A000052A06EE107AB8EEC66A80ED046A3DF468
:1059B00048AF96ED146A9DED0F5A25EE866AA5EE66
:1059C000076AB0EE675AA6EE265ABDEEC56A16EE15
:1059D00010EA16EE107ACE45A8BF4F468E45B8BFE6
:1059E0000F46062A06EE107AB8EEC66A80ED056A02
:1059F0003DF427AF96ED186A9DED105A25EE866AA4
:105A0000A5EE076AB0EE675AA6EE265ABDEEC56A45
:105A100016EE10EA16EE107ACE45A8BF4F468E4518
:105A2000B8BF0F46FDF7EBBEF0EEE76A9FED3E7A9A
:105A3000B7EE005ADFED3D5A9FED3D6AF5EEC07AB4
:105A4000E6EE875A9FED3B7A35EE665AF1EE10FA94
:105A5000F1EEC54AA6EEA56AA6EE867A27EE247A6E
:105A600003D5DFED357A37EEC77A94ED6C0A27EE71
:105A7000000A2DF0C9FCB0F5617F00F3A78607EEA0
:105A8000900A9FED2E7AF8EEE76A07EE905AF8EE4C
:105A9000E77A66EE876ABDEEE67A17EE103A2033B3
:105AA000402B41F202859FED260A2DF0ADFC00B29D
:105AB00007EE900AB8EEE77AFFF7C2BA214A02F180
:105AC000500503E00432954200F06A821378262BD9
:105AD000F8D19678D3789E42F4D2FFF7F0BA1A48FC
:105AE0001FF0FAFEFEF71BBD18481FF0F5FEFEF78B
:105AF00022BD17481FF0F0FEFEF717BDD4F8A051E5
:105B0000059B5D1BFEF787BBBC400120B82201202E
:105B1000AC430120D0560120505601205655555512
:105B2000D0340120303F0120306E99BC2716983DBB
:105B3000843459BEA40DC93FDB0F4940D06D393ABA
:105B400000000000102E01201C7101204C7001206B
:105B500008700120B1494B69002B3DF45FA9B048A2
:105B60004FF0010EAF4B008893FBF0F00B6818600C
:105B700081F811E0FDF752B903236370FEF7D9B83D
:105B800000230AAD09222946184615F0BBFB01285F
:105B90007EF4CFA80A9B93F8FE21552A01F06C836E
:105BA00041F2B41202210123A1546370FEF7C1B87F
:105BB0009D490320302305220091A0709B499C48F9
:105BC00016F00EFFFEF7B5B823690622652BA2700A
:105BD0002ED92278653B032A15BF6FF0FF016FF0C5
:105BE0007F014FF4807280220B4001339A4223617F
:105BF0001ED23268E66802329F19974281F0808592
:105C00008C4A05206660D16FA76049021660A070BB
:105C100003FB01F342F81C3C42F8183CA268012047
:105C2000854915F06FFD012841F060850623A370BA
:105C300000217F4815F0A2FC012841F05785A37888
:105C40000133DBB2A370FFF71CBA2278237D032A4D
:105C50007A4EDFF8E48114BF4FF480778027002B61
:105C600042D0012BFBD1764B4FF0FF3160684FF0F3
:105C7000000B1A68824633685202981CB1FBF2F19D
:105C80001AEB01024FF000014BF1000399426D49FC
:105C900008BF904238BF0246022015F059FE032883
:105CA00001F2BB8201A353F820F000BF333D01088D
:105CB000BD5C0108333D0108BD5C0108A368626852
:105CC0002569991AA94201D9E260216103283FF4AC
:105CD0007BAF0133B3FBF7F207FB12320AB13B444F
:105CE0009B1A00226360227532684146002002320E
:105CF00015F02EFE032801F2908201A353F820F044
:105D0000333D0108615D0108333D0108C95B0108AD
:105D100041F27013E35C002B3EF40BA844481FF0E3
:105D2000DBFDFEF706B80AAD41F2FC16294600235A
:105D30000922A05915F0E6FA01287DF4FAAF0023F4
:105D40000A9A2370B2F80B30B3F5007F01F06E842D
:105D500041F2B41203210123A1546370FDF7E9BF9E
:105D600063684FF0010201332275A3607BE7DFED2A
:105D7000367A364B94ED697AB0EE675AC3ED007A05
:105D8000F0EE673AC3ED017AC3ED027A304B196841
:105D9000FDF713BA2F4A304DD2ED006A2F4A95ED28
:105DA000006A1278C4ED656A84ED666A002A00F024
:105DB0007F8376EE665A94F99C21C4ED625A0132D3
:105DC000C4ED636A00F0DC86059B0025C4F8A031B1
:105DD00037EE677AFF27FCEEE77A214E84F89C7154
:105DE00084ED697A17EE902A96ED006AA4F8902166
:105DF000FEF721BA04F0B4F9039B049093F800E095
:105E0000D4F81451BEF1140F7CF425AF154B1D804E
:105E1000FCF721BF144AFDF703BE00BF5CC201209E
:105E200074C2012020A10700DDAF0208E876040853
:105E3000D4700120F8700120685F01206C7101208E
:105E4000747101206C5F012000000000083F0120F8
:105E5000703D01203CA3012054350120AC7E01207F
:105E60006835012088390120403B01206B4B6C4A8A
:105E7000B3F90430DFED6B7A82FB0312DB17C3EB5F
:105E8000A2031BB208EE103AB8EEC88A28EE278AA1
:105E9000B0EE480A06F060FFF0EE408AB0EE480A25
:105EA00006F0E2FE604BD878002800F04A845F4993
:105EB00044F25065B4F91222B1F902309B1AAB4298
:105EC00040F3BE87A3F50C43A03B45429D4200F33F
:105ED000C9878342A8BF03461344B1F90020B4F92F
:105EE000101244F250661BB2521AA4F81232B24297
:105EF00040F3AF87A2F50C42A03A954203DC9042F2
:105F0000A8BF10460546294407EE903A9FED486A1F
:105F10000BB2B8EEE77A07EE903AA4F81032F8EE3A
:105F2000E77A67EEE86A60EE277AE0EE076AE8EE65
:105F3000877A26EE867A67EE867ABDEEC77AFDEE20
:105F4000E77A17EE102A17EE903AA4F85021A4F839
:105F50005231FDF7E9BE3749DFED377A0968C4ED04
:105F60004C7A11F08053089340F02884DAF800103E
:105F70004E0200F14F87B6EE007AF4EEC75AF1EE0A
:105F800010FACCBF01210021002940F0438708917D
:105F9000FDF705BB294B1B7803F00108FDF751BC49
:105FA000274A284DD2ED007A274A95ED007A1278DB
:105FB000C4ED657A84ED667A002A00F0DD8377EE21
:105FC000676A94F99C21C4ED626A0132C4ED637A78
:105FD00000F03087059B0025C4F8A031DFED1B7A67
:105FE000FF261B4A84F89C61B0EE677AC4ED697A9B
:105FF00092ED006AFEF71FB977EEC77AB7EE007A26
:10600000C4ED4C7AF4EEC77AF1EE10FA41F3FC805D
:1060100085EE277A8DED0A7AFDF7B6BA183D012094
:106020006766666635FA8E3C64380120C038012008
:10603000CDCCCC3DF43E01200000008083590120EE
:106040003CA3012054350120AC7E0120000000005B
:1060500068350120BCF1000F00F0A58796ED006ABD
:106060009DED0A5A25EE866ACD48A5EE076AB0EE88
:10607000675AA6EE265ABDEEC56A16EE10EA16EE6F
:10608000107ACE45A8BF4F467145C8BF0F46012ABA
:1060900006EE107AB8EEC66A80ED006A3DF4D5AB24
:1060A00096ED046A9DED0B5A25EE866AA5EE076A09
:1060B000B0EE675AA6EE265ABDEEC56A16EE10EA95
:1060C00016EE107ACE45A8BF4F467145C8BF0F46A1
:1060D000022A06EE107AB8EEC66A80ED016A3DF437
:1060E000B4AB96ED086A9DED0C5A25EE866AA5EED6
:1060F000076AB0EE675AA6EE265ABDEEC56A16EEDE
:1061000010EA16EE107ACE45A8BF4F467145C8BFBB
:106110000F46032A06EE107AB8EEC66A80ED026AD0
:106120003DF493AB96ED0C6A9DED0D5A25EE866A13
:10613000A5EE076AB0EE675AA6EE265ABDEEC56A0E
:1061400016EE10EA16EE107ACE45A8BF4F467145FE
:10615000C8BF0F46042A06EE107AB8EEC66A80ED74
:10616000036A3DF472AB96ED106A9DED0E5A25EE72
:10617000866AA5EE076AB0EE675AA6EE265ABDEE0D
:10618000C56A16EE10EA16EE107ACE45A8BF4F4645
:106190007145C8BF0F46052A06EE107AB8EEC66AEA
:1061A00080ED046A3DF451AB96ED146A9DED0F5AF3
:1061B00025EE866AA5EE076AB0EE675AA6EE265A65
:1061C000BDEEC56A16EE10EA16EE107ACE45A8BFEF
:1061D0004F467145C8BF0F46062A06EE107AB8EE44
:1061E000C66A80ED056A3DF430AB96ED186A9DED08
:1061F000105A25EE866AA5EE076AB0EE675AA6EE3B
:10620000265ABDEEC56A16EE10EA16EE107ACE4595
:10621000A8BF4F467145C8BF0F46072A06EE107A41
:10622000B8EEC66A80ED066A3DF40FAB96ED1C6AC7
:106230009DED115A65EE865AE5EE075AE6EEA57A0F
:10624000FDEEE77A17EE902A9145A8BF91468A4263
:10625000A8BF494607EE901AF8EEE77AC0ED077A34
:10626000FDF7F3BA8222FDF70CBEDFED4E7AFDF7A3
:10627000D4BDBBF93C200123CBF8241007EE902AB3
:10628000CBF86420CBF88030F8EEE77A0022012CBE
:10629000CBED1D7ACBED1C7ACBF8782001F0EF80A6
:1062A000B4427EF4A1A8BBF93E200023012107EEF1
:1062B000902ACBF82830CBF86820B8EEE77ACBF8F4
:1062C00094100022012C8BED227A8BED217ACBF8F1
:1062D0008C2001F0D080B4427EF4B8A8BBF94020F5
:1062E000002107EE902ACBF86C200122CBF82C106D
:1062F000B8EEE77ACBF8A8200022012C8BED277AA4
:106300008BED267ACBF8A0207EF4D2A89FED268ACA
:10631000032D36D04FB107EE907AF8EEE77AF4EE1F
:10632000C87AF1EE10FA01F15A81DBF86C200021F5
:106330001E4B02EB56021E4CD8801E4892FBF6F60E
:10634000026894F82001CBF82C6091621163D1624D
:1063500028B1194A126832F480637EF4ACA8174A57
:10636000126812F4003240F0F1871046144DAB5C15
:106370000C32012B00F0368501301828F7D1FEF7DA
:106380009AB8B0EE480A2DF03FF800B2C2E7B7EE77
:10639000007AFDF7A0BCB7EE007AFDF72DBC00BF78
:1063A000303F012000000243000000008839012036
:1063B000B8220120A4A20120683D0120B4270120B9
:1063C000184B0408EF4D67EE897AEF4F29EE088AE3
:1063D000D5ED006A69EE288A95ED057A07EB86020D
:1063E000D5ED015AA6EEA77A95ED066AD5ED046AB9
:1063F000A5EEA76A95ED035AD5ED025A66EEC76A77
:1064000082ED007A20EE070AA5EE476AE5EEA76A5C
:1064100085ED056AC5ED066A2CF0F6FF95ED097A63
:1064200095ED0E5A07EB8602D5ED127A00B2D5ED46
:10643000175AA7EE085AD5ED0A6A1746E8EEA75A8A
:1064400095ED0F6AD5ED137A95ED187AA6EE886A68
:10645000D5ED0D6AA8EEA77AD5ED167A66EEC56A77
:1064600095ED0C3A67EEE57AD5ED0B3A95ED154AC8
:10647000D5ED144AA3EE456AE3EE886A82ED205A10
:10648000A5EEC47A0022E8EEA47AC7ED405AC4F81B
:106490000021C4F8042185ED0E6AC5ED0F6A85ED73
:1064A000177AC5ED187AC4F80821049BFEF792BD4F
:1064B00076EEC65AF0EE466A7DE4B44A1768B7F93C
:1064C0003260FEF7D6B9FDEEC54A9DED0A4AB048E6
:1064D00014EE901AD6ED004A65EEA44AE4EE074A9F
:1064E000B0EE674AA4EEA64AB4EEC46AF0EE444A9F
:1064F000F1EE10FA88BFF0EE454AFDEEE44A14EEE4
:1065000090EA14EE907ACE45A8BF4F467145C8BFB9
:106510000F46012A04EE907AF8EEE44AC0ED004AF4
:106520003DF48FA9D6ED044A9DED0B4A65EEA44AD1
:10653000E4EE074AB0EE674AA4EEA64AB4EEC46A97
:10654000F0EE444AF1EE10FA88BFF0EE454AFDEE57
:10655000E44A14EE90EA14EE907ACE45A8BF4F4676
:106560008E45B8BF0F46022A04EE907AF8EEE44A50
:10657000C0ED014A3DF465A9D6ED084A9DED0C4AEF
:1065800065EEA44AE4EE074AB0EE674AA4EEA64AD6
:10659000B4EEC46AF0EE444AF1EE10FA88BFF0EEB1
:1065A000454AFDEEE44A14EE90EA14EE907ACE45A8
:1065B000A8BF4F468E45B8BF0F46032A04EE907A17
:1065C000F8EEE44AC0ED024A3DF43BA9D6ED0C4A90
:1065D0009DED0D4A65EEA44AE4EE074AB0EE674A27
:1065E000A4EEA64AB4EEC46AF0EE444AF1EE10FA04
:1065F00088BFF0EE454AFDEEE44A14EE90EA14EE50
:10660000907ACE45A8BF4F468E45B8BF0F46042AA4
:1066100004EE907AF8EEE44AC0ED034A3DF411A985
:10662000D6ED104A9DED0E4A65EEA44AE4EE074A07
:10663000B0EE674AA4EEA64AB4EEC46AF0EE444A4D
:10664000F1EE10FA88BFF0EE454AFDEEE44A14EE92
:1066500090EA14EE907ACE45A8BF4F468E45B8BF5B
:106660000F46052A04EE907AF8EEE44AC0ED044A9B
:106670003DF4E7A8D6ED144A9DED0F4A65EEA44A15
:10668000E4EE074AB0EE674AA4EEA64AB4EEC46A46
:10669000F0EE444AF1EE10FA88BFF0EE454AFDEE06
:1066A000E44A14EE90EA14EE907ACE45A8BF4F4625
:1066B0008E45B8BF0F46062A04EE907AF8EEE44AFB
:1066C000C0ED054A3DF4BDA8D6ED184A9DED104A2F
:1066D00065EEA44AE4EE074AB0EE674AA4EEA64A85
:1066E000B4EEC46AF0EE444AF1EE10FA88BFF0EE60
:1066F000454AFDEEE44A14EE90EA14EE907ACE4557
:10670000A8BF4F468E45B8BF0F46072A04EE907AC1
:10671000F8EEE44AC0ED064A3DF493A8D6ED1C4AD3
:106720009DED114A65EEA45AE7EE045AE6EEA57A0D
:10673000B4EEE76AF1EE10FAC8BFF0EE457AFDF765
:1067400070B8144B9FED146AB3F90020B3F902300E
:1067500007EE902A06EE903AF8EEE77AF8EEE66A4F
:1067600027EEE87A60EE277AA0EE267AE8EEA67A9F
:1067700027EE067AFFF7DFBB77EEC76AF0EE477ABF
:106780001FE400BF40430120D4400120703D0120A0
:10679000303F0120C0380120CDCCCC3D6F12833A70
:1067A000BB8E1FED027A07EE903AEA4BF8EEE77ADD
:1067B00067EE877AC3ED007AFDF796B8B7EE007AF8
:1067C00077EE677AC5FEE75AFCF7E7BE07EE905A08
:1067D000DFEDE16AF8EEE77A66EEA65A9FEDDF5A42
:1067E0009FEDDF6A9FEDDF7AA5EE856A26EEA55A5A
:1067F000A5EE867AE5EE076A26EEA70AFFF755B9F9
:10680000012940F33C8607EE103AB8EEC77AC7EE8E
:10681000876AB1EEE68A032D13D04FB107EE907A66
:10682000F8EEE77AF4EEC87AF1EE10FA00F1D786C6
:10683000DBF8642002EB560292FBF6F2CBF8242040
:106840002EE5B0EE480A2CF0DFFD00B2E5E7FDEEE4
:10685000C54A9DED0A4AC44814EE907AD6ED004A26
:1068600065EEA44AE4EE074AB0EE674AA4EEA64AF3
:10687000B4EEC46AF0EE444AF1EE10FA88BFF0EECE
:10688000454AFDEEE44A14EE90EA14EE901ACE4525
:10689000A8BF49467745C8BF3946012A04EE901A79
:1068A000F8EEE44AC0ED004A3DF4AAAFD6ED044A42
:1068B0009DED0B4A65EEA44AE4EE074AB0EE674A46
:1068C000A4EEA64AB4EEC46AF0EE444AF1EE10FA21
:1068D00088BFF0EE454AFDEEE44A14EE90EA14EE6D
:1068E000901ACE45A8BF4946BE45B8BF3946022AD0
:1068F00004EE901AF8EEE44AC0ED014A3DF480AF90
:10690000D6ED084A9DED0C4A65EEA44AE4EE074A2E
:10691000B0EE674AA4EEA64AB4EEC46AF0EE444A6A
:10692000F1EE10FA88BFF0EE454AFDEEE44A14EEAF
:1069300090EA14EE901ACE45A8BF4946BE45B8BFAE
:106940003946032A04EE901AF8EEE44AC0ED024AF2
:106950003DF456AFD6ED0C4A9DED0D4A65EEA44AC6
:10696000E4EE074AB0EE674AA4EEA64AB4EEC46A63
:10697000F0EE444AF1EE10FA88BFF0EE454AFDEE23
:10698000E44A14EE90EA14EE901ACE45A8BF4946A8
:10699000BE45B8BF3946042A04EE901AF8EEE44A20
:1069A000C0ED034A3DF42CAFD6ED104A9DED0E4AE2
:1069B00065EEA44AE4EE074AB0EE674AA4EEA64AA2
:1069C000B4EEC46AF0EE444AF1EE10FA88BFF0EE7D
:1069D000454AFDEEE44A14EE90EA14EE901ACE45D4
:1069E000A8BF4946BE45B8BF3946052A04EE901AED
:1069F000F8EEE44AC0ED044A3DF402AFD6ED144A85
:106A00009DED0F4A65EEA44AE4EE074AB0EE674AF0
:106A1000A4EEA64AB4EEC46AF0EE444AF1EE10FACF
:106A200088BFF0EE454AFDEEE44A14EE90EA14EE1B
:106A3000901ACE45A8BF4946BE45B8BF3946062A7A
:106A400004EE901AF8EEE44AC0ED054A3DF4D8AEE3
:106A5000D6ED184A9DED104A65EEA44AE4EE074AC9
:106A6000B0EE674AA4EEA64AB4EEC46AF0EE444A19
:106A7000F1EE10FA88BFF0EE454AFDEEE44A14EE5E
:106A800090EA14EE901ACE45A8BF4946BE45B8BF5D
:106A90003946072A04EE901AF8EEE44AC0ED064A99
:106AA0003DF4AEAED6ED1C4A9DED114A65EEA45AFA
:106AB000E7EE045AE6EEA57AB4EEE76AF1EE10FAD4
:106AC000C8BFF0EE457AFDEEE77A17EE901A8945D9
:106AD000A8BF89468F42D8BF4F4607EE907AF8EE9E
:106AE000E77AC0ED077AFDF788BE01297FF70EAC83
:106AF00007EE103AB8EEC77AC7EE876AB1EEE68ABB
:106B000006E4012940F3B78407EE103AB8EEC77ADD
:106B1000C7EE876AB1EEE68A032D14D04FB107EEB7
:106B2000907AF8EEE77AF4EEC87AF1EE10FA00F116
:106B30005685DBF8682002EB560292FBF6F2CBF8A2
:106B40002820FFF7C8BBB0EE480A2CF05DFC00B26D
:106B5000E4E700BF7800012084F9223F92E741B9C1
:106B60009730083C15A82ABE303F0120CC494A691D
:106B7000002A3CF419AA0A6813604B74FCF714BA93
:106B8000D4F8A051059B5D1BFFF722B9BCF1000FA3
:106B900000F0E483C34E9DED0A4AD6ED004A65EE4F
:106BA000A44AE4EE074AB0EE674AA4EEA64AF0EE25
:106BB000444A33B1B4EE446AF1EE10FAC8BFF0EEC5
:106BC000454ABDEEC55A15EE108ABDEEE45A474659
:106BD00015EE101A884500F3FF844945A8BF4946C1
:106BE00005EE101AB048012AB8EEC55A80ED005AD9
:106BF0003CF42BAE96ED045ADDED0B4A25EE855A9A
:106C0000A4EE875AF0EE674AE5EE264AB0EE645AE3
:106C1000002B00F0D784B4EEE46AF1EE10FA40F3F2
:106C2000D18441464945A8BF494605EE101A022ABB
:106C3000B8EEC55A80ED015A3CF407AE96ED085AFD
:106C4000DDED0C4A25EE855AA4EE875AF0EE674A30
:106C5000E5EE264AB0EE645A002B00F0A984B4EEAB
:106C6000E46AF1EE10FA40F3A38441464945A8BF17
:106C7000494605EE101A032AB8EEC55A80ED025AAD
:106C80003CF4E3AD96ED0C5ADDED0D4A25EE855A48
:106C9000A4EE875AF0EE674AE5EE264AB0EE645A53
:106CA000002B00F07B84B4EEE46AF1EE10FA40F3BE
:106CB000758441464945A8BF494605EE101A042A85
:106CC000B8EEC55A80ED035A3CF4BFAD96ED105AAC
:106CD000DDED0E4A25EE855AA4EE875AF0EE674A9E
:106CE000E5EE264AB0EE645A002B00F04D84B4EE77
:106CF000E46AF1EE10FA40F3478441464945A8BFE3
:106D0000494605EE101A052AB8EEC55A80ED045A18
:106D10003CF49BAD96ED145ADDED0F4A25EE855AF5
:106D2000A4EE875AF0EE674AE5EE264AB0EE645AC2
:106D3000002B00F01F84B4EEE46AF1EE10FA40F389
:106D4000198441464945A8BF494605EE101A062A4E
:106D5000B8EEC55A80ED055A3CF477AD96ED185A59
:106D6000DDED104A25EE855AA4EE875AF0EE674A0B
:106D7000E5EE264AB0EE645A002B00F0F283B4EE42
:106D8000E46AF1EE10FA40F3EC8341464945A8BFAE
:106D9000494605EE101A072AB8EEC55A80ED065A84
:106DA0003CF453AD96ED1C5ADDED114A65EE855A63
:106DB000E4EE875AE5EEA67A002B00F0CA83F4EEE3
:106DC000C67AF1EE10FA40F1C48342464A45A8BFA4
:106DD0004A46174607EE907AF8EEE77AC0ED077A52
:106DE000FCF733BDD4F8242141003AB156780A1893
:106DF00005EB82025278B242BDF45DAB0144002043
:106E000005EB8101A4F81402C4F81802C4F8241197
:106E1000FDF751BB00230893B6EE007A67EE877A40
:106E2000F4EEE57AF1EE10FA7FF7C8ACF0EE675AAF
:106E3000FCF7B3BBD4F8A051059B5D1BFFF7CEB8A0
:106E40001A4DAB42BFF641A803F50C43A033FFF740
:106E50003CB8164EB242BFF650A802F50C42A03222
:106E6000FFF74BB82B46FFF737B8114A92ED000AEF
:106E70002CF0CAFA0F4B104AD3F8EC300F4982FBC2
:106E800003E2DB170880C3EBA21307EE903AF8EE9B
:106E9000E77AFDEEE77A17EE903A4B80FCF785BD76
:106EA0005CC20120D0340120303F0120B0B9FFFF87
:106EB000403B012058170120D34D62108839012032
:106EC00035FA8E3CDB0FC93F0000000007EE905AF8
:106ED0005FED056A1FED057AF8EEE77A84F808524F
:106EE00067EEA67A77EE876ABDEEE66A16EE103A8E
:106EF0002033402B40F27B825FED0D6ABDEEE77AD6
:106F0000CD4BC3ED016A17EE103A2033402B00F24F
:106F10006B829FEDCA7AF4EEC77AF1EE10FA40F375
:106F20000184DFEDC75A9FEDC76AF4EEC67A37EEEB
:106F3000E57AF1EE10FAF0EE477AF6DCDFEDC27A90
:106F4000B4EEE77AF1EE10FA40F1E983DFEDBC5AD6
:106F50009FEDBE6AB4EEC67A77EE257AF1EE10FAAE
:106F6000B0EE677AF6D49FEDBA7AF4EEC77AF1EE16
:106F700010FA40F38D829FEDB17A77EE677A67EE73
:106F8000A75A9FEDB45A9FEDB46A9FEDB47AA5EE6F
:106F9000856A27EEA55AA5EE867AE5EE077AC4ED56
:106FA000837AFDF7B9BC96ED006ADDED0A4A25EE5D
:106FB000866AA4EE876AF0EE674AE6EE264ABDEEE0
:106FC000E46A16EE100A814200F3BE814845A8BF6C
:106FD000484606EE100A089BB8EEC66A002B00F081
:106FE0000D849F48012A80ED006A3CF42EAC96ED9A
:106FF000046ADDED0B4A25EE866AA4EE876AF0EEA0
:10700000674AE6EE264ABDEEE46A16EE10CA61450E
:1070100000F39881CC45A8BFCC4606EE10CA089B69
:10702000B8EEC66A002B00F0E083022A80ED016A08
:107030003CF40BAC96ED086ADDED0C4A25EE866A51
:10704000A4EE876AF0EE674AE6EE264ABDEEE46AF1
:1070500016EE10CA614500F37381CC45A8BFCC463B
:1070600006EE10CA089BB8EEC66A002B00F06D83CE
:10707000032A80ED026A3CF4E8AB96ED0C6ADDED84
:107080000D4A25EE866AA4EE876AF0EE674AE6EEC0
:10709000264ABDEEE46A16EE10CA614500F34E8141
:1070A000CC45A8BFCC4606EE10CA089BB8EEC66A0F
:1070B000002B00F04183042A80ED036A3CF4C5AB49
:1070C00096ED106ADDED0E4A25EE866AA4EE876A1B
:1070D000F0EE674AE6EE264ABDEEE46A16EE10CA06
:1070E000614500F32981CC45A8BFCC4606EE10CA05
:1070F000089BB8EEC66A002B00F03983052A80EDA4
:10710000046A3CF4A2AB96ED146ADDED0F4A25EE5D
:10711000866AA4EE876AF0EE674AE6EE264ABDEE7E
:10712000E46A16EE10CA614500F30481CC45A8BF9D
:10713000CC4606EE10CA089BB8EEC66A002B00F0DB
:107140000D83062A80ED056A3CF47FAB96ED186A44
:10715000DDED104A25EE866AA4EE876AF0EE674AF6
:10716000E6EE264ABDEEE46A16EE10CA614500F36B
:10717000DF80CC45A8BFCC4606EE10CA089BB8EE0F
:10718000C66A002B00F00383072A80ED066A3CF4F0
:107190005CAB96ED1C6ADDED114A65EE865AE7EEB2
:1071A000245AE5EEA67AFDEEE77A17EE902A914290
:1071B00003DC4A45A8BF4A46114607EE901A089BD1
:1071C000F8EEE77A002B7FF409AE099B002B7FF4E1
:1071D00005AEBE45B8BFF0EE457AFFE5214B9FED09
:1071E000220A1D4625EE800A2CF00EF9E880FEF7F3
:1071F000B8BA1E481E498046FEF72AB9D4F8A051F5
:10720000059B5D1BFDF778BF1A49096811F0805393
:1072100008937FF401AEFEF7A9BE237DFEF71FBDE4
:1072200002F09EFF049A0F4B801A039A588092F83E
:1072300000E0FEF7FCBA00BF78000120DB0F4940F8
:10724000DB0FC940E4CB1641DB0F49C0E4CB16C1CC
:10725000DB0FC93F92E741B99730083C15A82ABE19
:10726000303F0120883901200000C84254420120EB
:10727000B8220120F43E012093F8FF21AA2A7EF4CF
:107280008FACD3F8C61149B193F8C221A2F10B001B
:1072900001282CD902F0F702062A28D0D3F8D611FB
:1072A00049B193F8D221A2F10B0001281FD902F0B5
:1072B000F702062A1BD0D3F8E61141B193F8E22178
:1072C00002F0F700062812D00B3A012A0FD9D3F8A2
:1072D000F61100293EF464AC93F8F231A3F10B02ED
:1072E000012A04D903F0F703062B7EF459AC41F2CE
:1072F000FC120123A150A370FEF716BD02F030FF6F
:10730000049ABA4B801A99F80010D4F81451988056
:10731000039B93F800E0FEF75FB902F021FF049AA7
:10732000B24B801A039A588092F800E0FEF73BBAFD
:107330008C4621E78C46FCE68C46D7E68C46B2E6C6
:107340008C468DE68C4668E6084642E6A84A1278E6
:10735000032A00F0DA810022FFF707B80AA9FDEE40
:10736000C54AA44801EB8202A34E14EE908A9446CB
:107370001A46089B089405E0614500F11000E6EC10
:10738000014A2ED0D0ED004AB1EC014A65EEA44A84
:10739000E7EE044AB0EE674AA6EEA44A32B1B4EE74
:1073A000446AF1EE10FAC8BFB0EE454ABDEEC44AD9
:1073B00004EE908A14EE104AA04506DC14EE104A42
:1073C0004C45A8BF4C4604EE904AF8EEE44A002B28
:1073D000D2D1099C002CCFD1BE45B8BFF0EE454AB2
:1073E000CAE7089CFCF731BADFED847AD7E5F4EE02
:1073F000C77AF1EE10FA40F38C81DFED815A9FEDF0
:10740000816AF4EEC66A36EEE57AF1EE10FAF0EE35
:10741000476AF6DCDFED7C6AB4EEE67AF1EE10FA4C
:1074200040F17A81DFED765A9FED786AB4EEC67A44
:1074300077EE256AF1EE10FAB0EE667AF6D49FED9B
:10744000747AF4EEC76AF1EE10FA76DD9FED717A88
:1074500077EE666A66EEA65A9FED6F5A9FED6F6AE9
:107460009FED6F7AA5EE856A26EEA55AA5EE867A7F
:10747000E5EE076A42E59FED618AFFF74DBB9FEDA0
:107480005F8AFFF7C8B9674F07F18002FEF78CB833
:107490009FED657AF4EEC77AF1EE10FA7FF56FADE5
:1074A0009FED597A77EE677A69E59FED5A7AF4EEA7
:1074B000C76AF1EE10FA40F33881DFED515A9FEDC3
:1074C000516AF4EEC66A36EEE57AF1EE10FAF0EEA5
:1074D000476AF6DCDFED4C6AB4EEE67AF1EE10FABC
:1074E00040F15281DFED465A9FED486AB4EEC67A0C
:1074F00077EE256AF1EE10FAB0EE667AF6D49FEDDB
:10750000447AF4EEC76AF1EE10FA05DD9FED417A98
:1075100077EE666AFFF760B99FED437AF4EEC76ACB
:10752000F1EE10FA7FF558A99FED377A77EE666A8B
:10753000FFF752B94046FDF7DCBF9FED3B7AF4EE12
:10754000C76AF1EE10FA85D59FED2F7A77EE666A5D
:1075500080E7FDEEE77A17EE902A4245FFF63AAC57
:1075600034E4BDEEC55A15EE101A4145BFF60EAC17
:1075700041460EE4BDEEC55A15EE101A4145BFF660
:10758000E1AB4146FFF7E1BBBDEEC55A15EE101A5F
:107590004145BFF6B3AB4146FFF7B3BBBDEEC55A9D
:1075A00015EE101A4145BFF685AB4146FFF785BB86
:1075B000BDEEC55A15EE101A4145BFF657AB414610
